:020000040800F2
:1000000000000120B5400008B5270008B727000808
:10001000B9270008BB270008BD2700080000000022
:10002000000000000000000000000000BF270008E2
:10003000C127000800000000C3270008C5270008EA
:100040000541000805410008C927000805410008CE
:100050000541000805410008D5270008DB270008F6
:1000600005410008054100080D2800080541000869
:10007000E1270008E3270008E5270008F12700082A
:10008000FD2700080928000805410008054100086F
:1000900000000000054100080F2800080541000885
:1000A0000541000805410008054100080541000818
:1000B0000541000805410008054100080541000808
:1000C00005410008054100080541000805410008F8
:1000D00005410008152800080541000805410008F1
:1000E00005410008112800082128000805410008E2
:1000F0000541000800000000000000000541000864
:1001000005410008054100082D28000805410008A8
:1001100005410008054100080541000805410008A7
:100120000541000805410008054100080541000897
:0801300005410008054100082B
:1001380010B5054C237833B9044B13B10448AFF319
:1001480000800123237010BD4C0100200000000036
:10015800E00E010808B5034B1BB103490348AFF390
:10016800008008BD0000000050010020E00E0108DA
:1001780014214160704714207047406A704700009E
:10018800790100087F01000883010008990100082F
:1001980010B5044604F1100000F05CFCC4F8F80047
:1001A8000148C4F87C0110BD88010008F8B5E6B024
:1001B80004460D4616461F460A4906A800F0CAFE20
:1001C80070996F9A05910492009733466E996D9ACB
:1001D800039102922A466C990191214600F060F839
:1001E80067B0F0BD94010008F8B5E6B004460D46C6
:1001F80016461F46094906A800F0ACFE6F996E9A8C
:100208000491039200976D996C9A0291019233467A
:100218002A46214600F087F867B0F0BD940100082F
:1002280038B500281CBF01680029184A23D1184B8B
:100238001C684FF6F0710C404CF24025AC421FBFD1
:100248001B6819404CF27024A14212D1114D296843
:1002580079B911490B68C3F30B03B3F58A6F1FBF54
:100268000968C1F30B0140F28343994204BF01219D
:10027800117028B905E0094B994204BF012111709A
:100288004068BDE8324001F09FBE00BF6801002011
:1002980000ED00E0002004E00010005C000037489A
:1002A8002DE9F04104460D46216816464A681F4666
:1002B80090478046B8F5403F2ED122680A99936846
:1002C800204698478046B8F5403F25D12368089ACC
:1002D8000799D3F80CC02046E0478046B8F5403F60
:1002E8001AD12368069A39461F692046B8478046BE
:1002F800B8F5403F10D1236829465D69324620464B
:10030800A8478046B8F5403F06D123680B9A09995B
:100318009D692046A847804621680A68204690477C
:100328004046BDE8F0812DE9F04104460D462168BC
:1003380016464A681F4690478046B8F5403F2ED17A
:1003480022680A999368204698478046B8F5403F46
:1003580025D12368089A0799D3F80CC02046E047AE
:100368008046B8F5403F1AD12368069A39461F6976
:100378002046B8478046B8F5403F10D12368294643
:100388005D6932462046A8478046B8F5403F06D109
:1003980023680999DD6900222046A847804621681C
:1003A8000A68204690474046BDE8F0814FF4403047
:1003B80070470000F0B50C4685B0114600281A4673
:1003C8001CBF0568002D0B4B11D082B104B971B95F
:1003D8000D9860B10F9E0E9F0A9B0290049603979A
:1003E8000B980C9E009001962046A8470346184695
:1003F80005B0F0BD020003002DE9F04F0646D0B06D
:100408000868F56DD6F860E0726EB76EF36E00BAE4
:1004180000906C46486800BA60600DF14008886832
:1004280000BAA060C86800BAE060086900BA206134
:10043800486900BA6061886900BAA061C86900BAF1
:10044800E061086A00BA2062486A00BA6062886A95
:1004580000BAA062C86A00BAE062086B00BA2063FA
:10046800486B00BA6063886B00BAA063C86B00BAB7
:10047800E063402058F80C1C58F820CC58F838ACE9
:100488008CEA010158F840CC8AEA01018CEA01099A
:100498004FEAF979401E48F8049BEBD187EA02003D
:1004A80000EA0E00784010EBF5610098DFF824C4EC
:1004B80041186144C81882EABE032B404FEAF06134
:1004C80053405918636859186144CF194FEAB50366
:1004D80083EABE01014081EABE0111EBF765A1681C
:1004E8004D196544A91883EAB0023A404FEAF1650C
:1004F8005A405519E26855194FEAB70282EAB0071F
:1005080065440F4005EBBE0E97EAB00717EBFE6592
:1005180027697D194FEAB10782EA0701654401EAB4
:100528000E01EB18514011EBF36561694D194FEA63
:10053800BE0187EA010E65440EEA030E15EBB00012
:100548008EEA070E0EEBF065D4F818E075446544A2
:10055800AA1881EAB30505404FEAF26E4D40AE4451
:10056800E569AE44E64477444FEAB00080EAB30E4A
:100578000EEA020E8EEAB30E0EEBF765D4F820E011
:1005880075446544691880EAB2053D404FEAF16E4A
:100598004540AE44656AAE44E6440EEBB3034FEA09
:1005A800B70787EAB20E0EEA010E8EEAB20E0EEB1C
:1005B800F365D4F828E075446544281887EAB1053E
:1005C8001D404FEAF06E7D40AE44E56AAE44E64415
:1005D8000EEBB2024FEAB30383EAB10E0EEA000E45
:1005E8008EEAB10E0EEBF265D4F830E0754465443E
:1005F800EF1983EAB00515404FEAF76E5D40AE4447
:10060800656BAE44E6440EEBB1014FEAB20282EAF2
:10061800B00E0EEA070E8EEAB00E0EEBF165D4F8B6
:1006280038E075446544EB1882EAB7050D404FEA97
:10063800F36E5540AE44E56BAE44E6440EEBB000B5
:100648004FEAB10181EAB70E0EEA030E8EEAB70E41
:100658000EEBF065D4F840E07544654481EAB30ECA
:10066800AA180EEA000E4FEAF2658EEA010E7544EA
:10067800DDF844E04FEAB000754480EAB30E654403
:100688000EEA020E15EBB7078EEAB30E0EEBF7650E
:10069800DDF848E04FEAB202754480EA020E65448C
:1006A8000EEA070E69188EEA000E0EEBF165DDF80A
:1006B8004CE07544654405EBB3034FEAB70E1427C5
:1006C8000DF1500CDFF810528EEA010B82EA0B0B89
:1006D8000BEBF36A5CF804BBDA44AA44504483EA9F
:1006E800B10B4FEAF06A8EEA0B0BDA445CF804BBF4
:1006F800DA44AA44524480EAB30B4FEAF26A8BEA1E
:10070800B10BDA445CF804BBDA444FEAB000AA44FF
:1007180080EA020BD6448BEAB30B0BEBFE6A5CF85B
:1007280004BBDA444FEAB202AA4482EA0E0B0AEB8F
:10073800B10180EA0B0B0BEBF16A5CF804BBDA44FD
:100748007F1DAA44282F0AEBB3034FEABE0EBBD382
:100758003C2F61D3502F4DD204EB870CC7F15407BF
:100768005E4CA7FB04A504465D4FA8088EEA010A63
:1007780082EA0A0A5CF804BB0AEBF3655D447D195A
:100788002C1983EAB10A4FEAF4658EEA0A0A55443D
:100798005CF804AB5CF804BB55447D19AA1884EADC
:1007A800B30A4FEAF2658AEAB10A55445D444FEA52
:1007B800B4047D1984EA020AAE448AEAB30A0AEB51
:1007C800FE655CF804AB55444FEAB2027D1982EA33
:1007D8000E0A15EBB10184EA0A0A5CF804BB0AEBBD
:1007E800F1655D447D1915EBB303401E4FEABE0E5B
:1007F800BCD12046F46D1B19F365336EC9183166F8
:10080800716E71447166B36ED218B266F16E40189B
:10081800F06650B0BDE8F08F4EEA010B0EEA010A0F
:100828000BEA020B4BEA0A0A0AEBF36554F827A015
:10083800DFF8B0C0554443EAB10B654403EAB10A96
:100848000BEA0E0B28184BEA0A0A7F1C0AEBF06524
:1008580054F827A0554440EAB30B654400EAB30AAC
:100868000BEAB10BAA184BEA0A0A7F1C0AEBF265DD
:1008780054F827A055444FEAB00040EA020B6544FB
:1008880000EA020A0BEAB30BAE444BEA0A0A7F1CE1
:100898000AEBFE6554F827A055444FEAB20242EA33
:1008A8000E0B654402EA0E0A0BEA000B15EBB101C8
:1008B8004BEA0A0A7F1C0AEBF16554F827A0554455
:1008C8007F1C65443C2F05EBB3034FEABE0EA3D350
:1008D80040E700BF9979825AA1EBD96ECDCCCCCC38
:1008E800D6C162CADCBC1B8F00B581B00168074A5B
:1008F800914200D110B9064801B000BD7C2110F02A
:1009080055FA4FF4003001B000BD00BFFC090008E3
:10091800030002002DE9F0410B4A92E8F85188B033
:10092800694681E8F8510268084B9A4200D118B923
:10093800074808B0BDE8F0811422083000F04FFBEA
:1009480008B0BDE8F08100BFDC090008FC09000818
:1009580003000200152904D20268044B9A4200D110
:1009680008B903487047083000F048BBFC09000884
:100978000300020010B481B013460268074CA2427B
:1009880000D118B901B010BC0548704701B000F19A
:10099800240210BC083000F035BB00BFFC09000879
:1009A8000300020010B481B013460268074CA2424B
:1009B80000D118B901B010BC054870470A4601B00B
:1009C80000F1240110BC083000F070BBFC090008DD
:1009D800030002000123456789ABCDEFFEDCBA981E
:1009E80076543210F0E1D2C300000000000000008D
:1009F80000000000F10800081D0900085D09000852
:100A08007D090008AD09000801040008790F0008F5
:100A1800C50F0008810F0008F0B5A3B004460B48C5
:100A280002900D4616461F46094B0822402104A88D
:100A380000F0D1FA28980190009733462A462146BB
:100A480002A800F01BF823B0F0BD00BFFC090008A5
:100A5800100A000810B5040008BF002408D0054893
:100A6800054B20600822402104F1080000F0B3FA89
:100A7800204610BDFC090008100A00082DE9F041C5
:100A880004460E46216817464A681D469047804628
:100A9800B8F5003F19D1226806999368204698470F
:100AA8008046B8F5003F10D123683146DE683A46E3
:100AB8002046B0478046B8F5003F06D12368079A1C
:100AC80029461D692046A847804621680A682046AD
:100AD80090474046BDE8F08110B500F033FA4FF476
:100AE800403400280EBF034C4FF4C07110F05EF97B
:100AF800204610BD0200030010B5044600F022FA9B
:100B080008B9054810BD0021A160D0F87C21116802
:100B180088474FF4403010BD0200030070B504460A
:100B28000D4600F00FFA064E40B1D0F87C0141683E
:100B38008847A84224BF65604FF44036304670BDF0
:100B4800020003002DE9FF4715000C4600D02CB128
:100B5800064600F0F7F95FEA000801D16448C3E0EF
:100B6800D8F8F80001684A689047B0F5003F17D1F7
:100B7800D8F87C118A68404690478146B9F1810FC0
:100B880080F09E80A94508F1FC0A17D2D8F8F80031
:100B98000368D3F80CC02A462146E047B0F5003F69
:100BA80040F08E80D8F8F8000368D3F810C06A4681
:100BB8005146E047B0F5003F76D10AE0002004E056
:100BC800215C0AF800100098401C00900098A84288
:100BD800F6D34FF0000C4749474A484B01AC009800
:100BE800844558D2D3E9007001ADC5E9007010788A
:100BF80000281ABF042086464FF0000E085854F803
:100C08000E5028443E4D05600127D0F800E087606B
:100C1800019D4F681AF80C007D408EEA050585F0A5
:100C2800040E65680F687D4085F0FC05754485F005
:100C3800A30568400AF80C000CF1010CCFE7D3E9D2
:100C4800004501A8C0E9004510782E4D002814BFC2
:100C58004FF0040E4FF0000E01A8744651F80EE054
:100C68000459A6440127CEF80050DEF80040CEF81B
:100C780008704D68019F40687D406C400D68684071
:100C880084F0040480F0FC00041984F057040AF886
:100C98000C400CF1010CCC45D1D3D8F8F800016810
:100CA8004A689047B0F5003F0AD1D8F8F8000368C1
:100CB800D3F80C804A465146C047B0F5003F01D0F2
:100CC800114811E0002006E05AF8201081F06A313E
:100CD8004AF82010401CB0EB990FF5D3B06840F0EB
:100CE8000100B0604FF4403004B0BDE8F08700BFA9
:100CF80002000300780F010868010020240F000893
:100D0800ADBE4ED70DBE75A10100030038B50C4627
:100D1800017A1546CA0702D500F014F908B908483F
:100D280032BDD0F8F80003682146DC682A46A0479F
:100D3800B0F5003F01D0034832BD4FF4403032BD1A
:100D480002000300010003002DE9F84191B00546B7
:100D58000E461746402101A810F028F8297AC8073E
:100D680004D5284600F0EEF8040002D1DFF8A4808C
:100D78004BE0D4F8F800DFF8A0800368D3F810C07F
:100D88006A4601A9E047B0F5003F3ED1D4F8F80023
:100D980001684A689047B0F5003F36D1D4F87C1115
:100DA8008A6820469047D4F8F830024618461B68EF
:100DB800D3F80CC004F1FC01E047B0F5003F24D1A2
:100DC800D4F87C0141688847D4F8F83002461846C0
:100DD8001B68D3F80CC001A9E047B0F5003F14D157
:100DE800D4F8F8000268696893689847B0F5003F3E
:100DF8000BD1D4F8F80003681C693A463146A0477D
:100E0800B0F5003F08BF4FF44038404612B0BDE887
:100E1800F08100BF02000300010003002DE9F84142
:100E2800A5B0074688461646402115A80FF0BEFF14
:100E380000220492402105A80FF0B8FF387AC107B4
:100E48005ED5384600F07EF8050059D0D5F8F80090
:100E58002D4C0368D3F810C06A4605A9E047B0F5E1
:100E6800003F3CD1D5F8F80001684A689047B0F5D2
:100E7800003F34D1D5F87C118A6828469047D5F8C8
:100E8800F830024618461B68D3F80CC005F1FC017F
:100E9800E047B0F5003F22D1D5F87C01416888478A
:100EA800D5F8F830024618461B68D3F80CC005A9D7
:100EB800E047B0F5003F12D1D5F8F800026879682C
:100EC80093689847B0F5003F09D1D5F8F800036852
:100ED8001D6904AA15A9A847B0F5003F01D020460E
:100EE8000FE00A4B0A490B4A0396029101924046C9
:100EF8001C68049B009415AA796800F0E5F900E0E5
:100F0800054826B0BDE8F08101000300800F010804
:100F1800936E030026C703000200030004B001011A
:100F280000170145E10A0008010B0008250B00081D
:100F3800B50300084D0B0008150D0008510D0008F9
:100F4800250E00080168024A914218BF0020704728
:100F58002C0F000810B5040008BF002404D0034873
:100F68002060204609688847204610BD2C0F0008DD
:100F780020225C300FF018BFF0B58468A308002267
:100F880004F0030407E000F15C0555F8226035BA67
:100F980041F82250521C9A42F5D300220BE000F18E
:100FA8005C0502EB830755F82360D500C5F11805E9
:100FB800EE40CE55521CA242F1D3F0BD30B5C46804
:100FC80003690022E31AD5188C5C0544521C082AD0
:100FD8002C77F8D330BD0360C1600261704738B523
:100FE800044615460022626023685A68904700202C
:100FF8006061A061A5604FF4003032BD81604FF49C
:10100800003070472DE9F84304462079D4F80C8065
:10101800450748BF244845D466691D46A8F1010024
:1010280000EAD60306EBC506B6EBC50F666102D229
:10103800A669761CA6611746A66906EB5576A661D1
:101048000E46E918884225D2A8EB03094A463146DC
:10105800F8180FF0A9FE2268136839460FE04246D7
:1010680038460FF0A1FE23681A6839462046904793
:1010780007E0311811F00300F1D122681368204607
:101088009847484600EB0809A9F10101A942F0D3A5
:10109800002300E000202A1A3118F8180FF084FE07
:1010A8004FF40030BDE8F283040002002DE9FC4F44
:1010B800024685B0D0681369DFF86CC1DFF86C812F
:1010C800A0EB030A506840F004005060002703A812
:1010D80002900DF10C0ED8E9003403A8544DC0E974
:1010E80000342878534D00280CBF00230423994668
:1010F8005CF803305EF80940234401261D601C6833
:101108009E60DCF80430039DDCF80090DEF8046093
:101118005D406540484C654089EA0606474C664094
:101128007519474C6540D8E9006B03AC0028C4E941
:10113800006B0EBF002404200424029E5CF800000B
:10114800345920183F4C04600126046886600398CF
:10115800029E43406340384C7068634089EA00004F
:10116800364C6040034438484340280018BF0120EB
:101178005B1E9B41042F2CBFC0B2D80F02F1140391
:1011880053F8200007F00303C3F10303DB00D84042
:101198000DF807007F1C082F9DD315460C466A6979
:1011A800AB69E868D20842EA4372401E00EA0207C7
:1011B800002302409B420AD8524508D28020E055BD
:1011C8007F1C574516D2AAEB0701E01910E08020D2
:1011D800E05500E0E355E8687F1C8742FAD32A68A7
:1011E800136828469847BAF1000F03D051462046A5
:1011F8000FF0DCFD2A68069E059F9368694628461D
:1012080098472A68D2F8009021462846C8472B6894
:10121800DA683946284690470EB1A86830604FF41E
:10122800003007B0BDE8F08F780F010854120008AD
:10123800680100205FC5109304850012FC68017ADC
:10124800C0F524FF24AF33D426AF698B04B0010165
:1012580000170145F8B501240094002300240DE08F
:10126800009D065D0F5D7E40F643761CF60F86F006
:10127800010635400095641C009DEB189442EFD39D
:101288001846F2BDF8B5002301240094002A11E0A5
:10129800009C85188F1815F8016C17F8015C6E40D2
:1012A800F643761CF60F86F0010634400094009C45
:1012B800E318521EECD11846F2BD00005D1200087A
:1012C8008D120008010000002DE9F84F1D46DDF8D9
:1012D80028900B9F0D9C4FF0FF3300930E469246CB
:1012E800D9F800B0804632465146D847834664B3A1
:1012F800D9F8043032465146404698476FEA0B0207
:10130800521C42EA0B0200996FEAD2735B1C194027
:10131800C2430091521C024300996FEAD2735B1CCE
:101328001940009186F05531484087EA000181F064
:101338005531216080F05531C943491C0843009A52
:101348006FEAD070401C82430092D9F80800012847
:1013580009D17540E943491C0D4300986FEAD572DD
:10136800521C90430AE0F11C85EA9102D243521CB8
:10137800154300986FEAD5735B1C984386F0AA362C
:10138800009086EA0B0686F0AA33F243DB430C98FA
:10139800C2F3C0725B1C42EAD3720099D243521C5A
:1013A80091430091774000998843009987F0AA37C4
:1013B8000F403843BDE8F28F034613F8012B002A8B
:1013C800FBD1181A0138704781F0004102E000BFD4
:1013D80083F0004330B54FEA41044FEA430594EAED
:1013E800050F08BF90EA020F1FBF54EA000C55EA28
:1013F800020C7FEA645C7FEA655C00F0E2804FEAF9
:101408005454D4EB5555B8BF6D420CDD2C4480EADA
:10141800020281EA030382EA000083EA010180EA0A
:10142800020281EA0303362D88BF30BD11F0004F58
:101438004FEA01314FF4801C4CEA113102D040428E
:1014480061EB410113F0004F4FEA03334CEA1333C9
:1014580002D0524263EB430394EA050F00F0A780E1
:10146800A4F10104D5F1200E0DDB02FA0EFC22FADC
:1014780005F2801841F1000103FA0EF2801843FAD0
:1014880005F359410EE0A5F120050EF1200E012AC1
:1014980003FA0EFC28BF4CF0020C43FA05F3C018FF
:1014A80051EBE37101F0004507D54FF0000EDCF178
:1014B800000C7EEB00006EEB0101B1F5801F1BD321
:1014C800B1F5001F0CD349085FEA30004FEA3C0C25
:1014D80004F101044FEA445212F5800F80F09A801B
:1014E800BCF1004F08BF5FEA500C50F1000041EB1F
:1014F800045141EA050130BD5FEA4C0C404141EB23
:101508000101013C28BFB1F5801FE9D291F0000F1D
:1015180004BF01460020B1FA81F308BF2033A3F1CC
:101528000B03B3F120020CDA0C3208DD02F1140CC3
:10153800C2F10C0201FA0CF021FA02F10CE002F1FE
:101548001402D8BFC2F1200C01FA02F120FA0CFCF7
:10155800DCBF41EA0C019040E41AA2BF01EB045140
:10156800294330BD6FEA04041F3C1CDA0C340EDC3E
:1015780004F11404C4F1200220FA04F001FA02F381
:1015880040EA030021FA04F345EA030130BDC4F13F
:101598000C04C4F1200220FA02F001FA04F340EA34
:1015A8000300294630BD21FA04F0294630BD94F0E5
:1015B800000F83F4801306BF81F480110134013DCC
:1015C8004EE77FEA645C18BF7FEA655C29D094EA3D
:1015D800050F08BF90EA020F05D054EA000C04BFBB
:1015E8001946104630BD91EA030F1EBF00210020A6
:1015F80030BD5FEA545C05D14000494128BF41F045
:10160800004130BD14F580043CBF01F5801130BDA8
:1016180001F0004545F0FE4141F470014FF0000033
:1016280030BD7FEA645C1ABF194610467FEA655CE4
:101638001CBF0B46024650EA013406BF52EA033586
:1016480091EA030F41F4002130BD00BF90F0000F74
:1016580004BF0021704730B54FF4806404F13204B0
:101668004FF000054FF0000150E700BF90F0000F69
:1016780004BF0021704730B54FF4806404F1320490
:1016880010F0004548BF40424FF000013EE700BF60
:1016980042004FEAE2014FEA31014FEA02701FBFF0
:1016A80012F07F4393F07F4F81F06051704732F022
:1016B8007F4208BF704793F07F4F04BF41F4002179
:1016C800704730B54FF4607401F0004521F00041D7
:1016D8001CE700BF50EA010208BF704730B54FF061
:1016E80000050AE050EA010208BF704730B511F062
:1016F800004502D5404261EB41014FF4806404F19A
:1017080032045FEA915C3FF4D8AE4FF003025FEA1F
:10171800DC0C18BF03325FEADC0C18BF033202EBA3
:10172800DC02C2F1200300FA03FC20FA02F001FAFD
:1017380003FE40EA0E0021FA02F11444BDE600BFA0
:101748004FF0FF3C06E000BF4FF0010C02E000BF85
:101758004FF0010C4DF804CD4FEA410C7FEA6C5C68
:101768004FEA430C18BF7FEA6C5C1BD001B050EA0B
:10177800410C0CBF52EA430C91EA030F02BF90EAF6
:10178800020F0020704710F1000F91EA030F58BFB5
:10179800994208BF90422CBFD8176FEAE37040F017
:1017A800010070474FEA410C7FEA6C5C02D150EAB5
:1017B800013C07D14FEA430C7FEA6C5CD6D152EA70
:1017C800033CD3D05DF8040B704700BF8446104635
:1017D80062468C461946634600E000BF01B5FFF734
:1017E800B7FF002848BF10F1000F01BD4DF808ED04
:1017F800FFF7F4FF0CBF012000205DF808FB00BFD5
:101808004DF808EDFFF7EAFF34BF012000205DF82E
:1018180008FB00BF4DF808EDFFF7E0FF94BF01207B
:1018280000205DF808FB00BF4DF808EDFFF7CEFF7C
:1018380094BF012000205DF808FB00BF4DF808EDBB
:10184800FFF7C4FF34BF012000205DF808FB00BF8C
:101858004FEA410212F5001215D211D56FF47873D0
:10186800B3EB625212D94FEAC12343F0004343EA73
:10187800505311F0004F23FA02F018BF404270474E
:101888004FF00000704750EA013005D111F00040D8
:1018980008BF6FF0004070474FF00000704700BF6E
:1018A80080F0004002E000BF81F0004142001FBF0D
:1018B8005FEA410392EA030F7FEA226C7FEA236C16
:1018C8006AD04FEA1262D2EB1363C1BFD21841400B
:1018D80048404140B8BF5B42192B88BF704710F0A1
:1018E800004F40F4000020F07F4018BF404211F044
:1018F800004F41F4000121F07F4118BF494292EAAC
:10190800030F3FD0A2F1010241FA03FC10EB0C00D7
:10191800C3F1200301FA03F100F0004302D5494264
:1019280060EB4000B0F5000F13D3B0F1807F06D311
:1019380040084FEA310102F10102FE2A51D2B1F109
:10194800004F40EBC25008BF20F0010040EA0300FE
:101958007047490040EB0000013A28BFB0F5000F7E
:10196800EDD2B0FA80FCACF1080CB2EB0C0200FA34
:101978000CF0AABF00EBC25052421843BCBFD04083
:101988001843704792F0000F81F4000106BF80F4FD
:1019980000000132013BB5E74FEA41037FEA226CC0
:1019A80018BF7FEA236C21D092EA030F04D092F08B
:1019B800000F08BF0846704790EA010F1CBF0020BF
:1019C800704712F07F4F04D1400028BF40F000401C
:1019D800704712F100723CBF00F50000704700F03C
:1019E800004343F0FE4040F4000070477FEA226263
:1019F80016BF08467FEA23630146420206BF5FEA34
:101A0800412390EA010F40F4800070474FF0000333
:101A180004E000BF10F0004348BF40425FEA000CFA
:101A280008BF704743F0964301464FF000001CE0A2
:101A380050EA010208BF70474FF000030AE000BFF8
:101A480050EA010208BF704711F0004302D5404236
:101A580061EB41015FEA010C02BF844601460020A8
:101A680043F0B64308BFA3F18053A3F50003BCFAC3
:101A78008CF2083AA3EBC25310DB01FA02FC634470
:101A880000FA02FCC2F12002BCF1004F20FA02F277
:101A980043EB020008BF20F00100704702F120026A
:101AA80001FA02FCC2F1200250EA4C0021FA02F2CB
:101AB80043EB020008BF20EADC7070474FEA40029F
:101AC800B2F1FE4F0FD34FF09E03B3EB12620DD964
:101AD8004FEA002343F0004310F0004F23FA02F0CE
:101AE80018BF404270474FF00000704712F1610F75
:101AF80001D1420205D110F0004008BF6FF000404C
:101B080070474FF00000704753B94AB9002908BF21
:101B180000281CBF4FF0FF314FF0FF3000F070B9C4
:101B2800ADF1080C6DE904CE00F006F8DDF804E02C
:101B3800DDE9022304B070472DE9F047089E0D4601
:101B480004460F46002B4AD18A42944665D9B2FA18
:101B580082F343B102FA03FCC3F120029F4020FA4A
:101B680002F217439C404FEA1C4E1FFA8CF5B7FB54
:101B7800FEF1220C0EFB117742EA074201FB05F049
:101B880090420AD91CEB020201F1FF3780F01B8159
:101B9800904240F2188102396244121AA4B2B2FB90
:101BA800FEF00EFB102244EA024400FB05F5A542B4
:101BB8000AD91CEB040400F1FF3280F00681A5422B
:101BC80040F203816444023840EA0140641B00216A
:101BD8001EB1DC400023C6E90043BDE8F0878B4214
:101BE80008D9002E00F0EC800021C6E9000508465F
:101BF800BDE8F087B3FA83F1002949D1AB4202D39B
:101C0800824200F2F780841A65EB0302012017462E
:101C1800002EE2D0C6E90047DFE702B9FFDEB2FADC
:101C280082F3002B40F08F808A1A4FEA1C471FFA74
:101C38008CFE0121B2FBF7F507FB1520220C42EAC6
:101C480000420EFB05F0904208D91CEB020205F198
:101C5800FF3802D2904200F2CA804546121AA4B256
:101C6800B2FBF7F007FB102244EA02440EFB00FE29
:101C7800A64508D91CEB040400F1FF3202D2A645A0
:101C880000F2BA801046A4EB0E0440EA05409FE734
:101C9800C1F120078B4022FA07FC4CEA030C05FA35
:101CA80001F420FA07F3FD40234300FA01F94FEA53
:101CB8001C401FFA8CFEB5FBF0F81C0C00FB1855F5
:101CC80044EA054408FB0EF5A54202FA01F20BD9D5
:101CD8001CEB040408F1FF3A80F08780A54240F22B
:101CE8008480A8F102086444641B9DB2B4FBF0F33D
:101CF80000FB134445EA044403FB0EFEA64508D93D
:101D08001CEB040403F1FF306BD2A64569D9023BF2
:101D1800644443EA0840A0FB0283A4EB0E049C42FF
:101D2800C6461D4655D352D056B1B9EB0E0364EBE7
:101D3800050404FA07F7CB40CC401F43C6E90074FA
:101D48000021BDE8F087C3F1200102FA03FC20FA64
:101D580001F225FA01F19D402A434FEA1C471FFA78
:101D68008CFEB1FBF7F007FB1015110C41EA054199
:101D780000FB0EF58D4204FA03F408D91CEB0101AF
:101D880000F1FF382FD28D422DD902386144491B0A
:101D980092B2B1FBF7F507FB151142EA014205FBC8
:101DA8000EF1914208D91CEB020205F1FF3816D258
:101DB800914214D9023D6244521A45EA004139E77A
:101DC8003146304609E73946E7E61046FCE6C145A4
:101DD800AAD2B8EB020E63EB0C050138A4E745461E
:101DE800EAE7034695E74046D1E7D0467CE7023D5F
:101DF800624433E708460BE76444023843E700BF10
:101E0800704700BF1348144A08B54FF00043C0E9B3
:101E180000230422002342610122C2614FF4805151
:101E280007220383C0E90233C0E90933C0E90C1271
:101E38000361837680F8203080F82C30826380F844
:101E48003C30C36402F0B0F918B1BDE8084000F0B6
:101E580009BC08BD6C010020002401400268084B41
:101E68009A4282B00AD14FF0B0431A6E42F400721F
:101E78001A661B6E03F400730193019B02B070474E
:101E8800002401400268054B9A4201BF4FF0B0425E
:101E9800136E23F400731366704700BF00240140DB
:101EA80030B585B000240546CDE901440394FFF719
:101EB800A9FF144802F010FD08B100F0D3FB114847
:101EC800039401A9CDE9015402F0CCFA08B100F05D
:101ED800C9FB0C4802F02AFC08B100F0C3FB4FF024
:101EE800FF31084802F060FA064802F0D7FC0548BE
:101EF80002F0B4FA0446034802F07AFC204605B022
:101F080030BD00BF6C010020014B024A1A607047C7
:101F18006C0100200024014008B50948FFF7C0FF04
:101F280068B1084BB3F8AA304FF6FF72934216BF58
:101F380040F6E442044B5343B3FBF0F398B208BDB8
:101F4800002000B40075FF1FD8084C0013B500230B
:101F5800ADF80630FFF7E0FF04461948FFF7A0FF89
:101F6800184BB3F8C820B3F8A8108A4204FB00F055
:101F780018D040F6E443B0FBF3F364205B1A434304
:101F8800521A93FBF2F31E331BB2ADF80630BDF8BC
:101F980006305BB21B02ADF80630BDF8060000B291
:101FA80002B010BD4FF47A7240F6FF73B0FBF3F342
:101FB8005343A3F53923A3F50C6340F6C412E0E7B5
:101FC800001000B00075FF1F4FF0B04382B09A6A4E
:101FD80022F480529A629A6C42F480529A649B6C02
:101FE80003F480530193019B002002B070474FF027
:101FF800B04382B09A6C02439A649B6C034001938D
:10200800019B02B0704708B50420FFF7F0FF0120DC
:10201800FFF7EDFF0220FFF7EAFF002211460B2031
:1020280002F0F8FC0B2002F027FD002211460C20DC
:1020380002F0F0FC0C2002F01FFD002211460D20DA
:1020480002F0E8FC0D2002F017FD002211460E20D8
:1020580002F0E0FC0E2002F00FFD002211460F20D6
:1020680002F0D8FC0F2002F007FD002211461020D4
:1020780002F0D0FC102002F0FFFC002211461120D3
:1020880002F0C8FC112002F0F7FC002236201146AD
:1020980002F0C0FCBDE80840362002F0EDBC0000AC
:1020A80008B502F031FF10B16FF0040008BD064B0F
:1020B8009A6942F040429A614CF2FA321A6102F08F
:1020C80035FF0028F2D0EFE700400058F0B585B0A2
:1020D80000230C4600930646A8B3FFF7E1FF054628
:1020E80070BB02F011FF88BB1A481B4A02230193F8
:1020F800D0F8E01506F1784302EA8121B3FBF1F745
:1021080001FB1733DB0A0293D0F8E00504F17841AC
:102118000139314402EA8022B1FBF2F002FB1011CE
:10212800C3EBD1230133694601A8039302F07EFF74
:1021380020B102280CBF01256FF0010502F0F6FE60
:10214800284605B0F0BD6FF00505F9E76FF0040506
:10215800F6E700BF0070FF1F00FCFF03014B18608B
:1021680000207047D00100202DE9F04F89B0B0F170
:10217800006F06460F460092C0F0C580DFF89881D0
:10218800664DD8F8E03505EA832303F10063013B87
:10219800984200F2B880002800F0B880002900F0CA
:1021A800B58040EA02035B0740F0B080FFF778FF94
:1021B8000446A0BB02F0A8FE002840F0AA80D8F888
:1021C800E01506F1784205EA8121B2FBF1F301FB43
:1021D8001322009B03F17843013B3344B3FBF1F036
:1021E80001FB1033DB0A01334FEAD22AA3EBD222D8
:1021F800012A039388BFC6F30A050AF58038C6F199
:10220800080398BF009D069388BFC5F500654FEA8F
:10221800C828B346039B9A4505D302F087FE20469B
:1022280009B0BDE8F08FA6F10803069A1A44954252
:1022380019D804950197CDF814B04FF00009059B03
:1022480009EB0301049B99453ED3009BAB442F4403
:102258005D1BB5F5006F28BF4FF400650AF1010A50
:1022680008F50068D6E753F8081F5A68B2F1FF3F2F
:1022780008BFB1F1FF3FD8D0294B186810B96FF0EB
:102288000504CAE7B8F1000F04D04FF400624146D4
:102298000EF026F9DFF88890D9F80030CBF30A0061
:1022A80039461844AAB20EF01BF94FF400614046B3
:1022B800FFF70CFF08BBD9F8003001934FF4006317
:1022C800CDF814800493B8E7019B07914B4402931F
:1022D8000120D3E9002302F063FE88B90799019B26
:1022E800D1E9000259F80310029B5B689A4208BFC3
:1022F800884205D109F10809A1E76FF001048CE7CC
:102308006FF0030489E74FF0FF3488E76FF00504A6
:1023180085E76FF0040482E70070FF1F00FCFF03ED
:10232800D0010020B1F1006F70B511D30B4BD3F879
:10233800E0650B4B03EA862303F10063013B9942F6
:1023480006D840B139B192B20EF0CAF8002070BD7B
:102358004FF0FF30FBE76FF00500F8E70070FF1F54
:1023680000FCFF03B0F1006F10B40DD3084BD3F895
:10237800E045084B03EA842303F10063013B9842DC
:1023880002D810BCFFF7A2BE4FF0FF3010BC704758
:102398000070FF1F00FCFF034FF0B04382B0DA6CFF
:1023A8000243DA64DB6C03400193019B02B070477F
:1023B80070B5012086B00024CDE90444FFF7ECFF96
:1023C8000220FFF7E9FF0420FFF7E6FF01250222BC
:1023D8000DEB00014FF404134FF09040CDE90123B9
:1023E800204E039502F070FE4FF4441301A94FF0FC
:1023F8009040CDE90235019502F066FE04230DEB0D
:1024080003013046CDE90135CDE9034402F05CFE15
:1024180022463046082102F07DFF4FF4806301A96F
:102428004FF09040CDE90134039402F04DFE0823AB
:1024380001A93046CDE90135CDE9034402F044FE57
:1024480022462146062002F0E5FA062002F014FB97
:1024580022462146072002F0DDFA072002F00CFB95
:1024680006B070BD0004004808B51248124A134B64
:10247800C0E9002300230122C0E90232C0E9043385
:10248800C0E90633036202F057FF08B100F0EAF82A
:102498000848002102F0A1FF08B100F0E3F8054860
:1024A800002102F0C0FF18B1BDE8084000F0DAB81A
:1024B80008BD00BF94020020005800405D3E302057
:1024C80070B596B005461422002103A80EF040FC12
:1024D8003822002108A80EF03BFC2A68304B9A42AB
:1024E8005BD18023089308A84FF440230E9303F090
:1024F800F5FC08B100F0B6F84FF0B0444FF4C05006
:10250800E36C43F00103E364E36C03F0010302931B
:10251800029B12230026CDE903030323CDE90563BB
:102528004FF09040042303A9079302F0CDFDA36D5B
:10253800DFF870C043F48003A365A36D1A4C03F45D
:1025480080030193019B26620D23C4E900C3204642
:102558008023C4E90266C4E90436C4E9066602F0C9
:10256800EBFA08B100F07EF8104AEC63A562104C53
:102578000E23C4E900231021002380222046C4E949
:102588000213C4E90423C4E90633236202F0D4FA2F
:1025980008B100F067F8AC63A56216B070BD00BF63
:1025A8000058004044000240D40100205800024076
:1025B8003402002000B59BB04822002108A80EF084
:1025C800C7FB1822002102A80EF0C2FB02F050FF40
:1025D8004FF0B0420120D2F8903023F01803C2F82F
:1025E8009030D2F8003423F4C06343F40073C2F887
:1025F8000034D2F8003403F4C0630193019B242310
:10260800089381230B930023CDE91003B02208A877
:10261800CDE9122303F0A4F808B172B6FEE74F2300
:10262800CDE90230CDE90400CDE90600022102A877
:1026380003F030FB08B172B6FEE71BB05DF804FB8F
:1026480008B501F05FFDFFF7B5FFFFF7B1FEFFF733
:10265800DAFC00F0CAFD40F6B83000F03FFA00F0AE
:10266800CBFDFCE772B6FEE700B58DB02C22002149
:1026780001A80EF06DFB1748174B03601F238360FA
:102688004FF080420023C0E90433C0E90723836187
:102698004FF48073436203F0A7FD08B1FFF7E2FF30
:1026A8000C4803F0CDFE08B1FFF7DCFF4FF00053F4
:1026B80000220793074808924FF4807301A90292F9
:1026C80006920B9303F0F0FD08B1FFF7CBFF0DB0B6
:1026D8005DF804FBE80200200028004010B504461D
:1026E80090B03822002102A80EF032FB2268194B64
:1026F8009A422CD14FF48033029302A84FF480738E
:102708000F9303F0EBFB08B1FFF7ACFF4FF0B043BA
:102718000220D3F8902042F40042C3F890209A6D2A
:1027280042F480629A659B6D002203F4806311462F
:102738000193019B02F06EF9022002F09DF900223C
:102748002A20114602F066F92A2002F095F910B005
:1027580010BD00BF002800407047000008B501F018
:10276800E7FC044B0120C3F88800BDE8084002F0EC
:10277800D7BE00BF0004005801F0E1BC08B501F065
:10278800DEFC00F059FCFFF713FEFFF73CFCBDE848
:102798000840FFF769BE08B501F0CAFCBDE808406B
:1027A8000121002002F06CBE70477047FEE7FEE78B
:1027B800FEE7FEE7FEE77047704770477047000086
:1027C800014803F063BE00BFE8020020012002F0C8
:1027D800A7BD022002F0A4BD70477047014802F06F
:1027E80025BB00BFD4010020014802F01FBB00BF79
:1027F800C0030020014802F019BB00BF600300209D
:10280800FFF7F2BF7047704770470000014804F0B7
:1028180001BA00BF20040020014803F069BC00BFD2
:10282800E8020020014804F05CB800BF4C03002017
:102838002DE9F04389B080460020109E0790894614
:1028480015461F46FDF7ECFCF0B9104CCDE9009099
:10285800CDE9020407AB0E480593142304933A46C6
:10286800434629460068FDF7A5FD2346324604F194
:10287800140153F8044B42F8044B8B42F9D1079BDF
:10288800337509B0BDE8F0830120FAE72003002082
:10289800740F01081FB50E4C00233C2202A8CDE995
:1028A80002336275237500F0BBF8042303AA009471
:1028B80012210848FFF7BCFF0749142220460EF0F2
:1028C80037FAB0FA80F35B09637504B010BD00BF36
:1028D800340300209C0F0108DE060020054808B5D7
:1028E8000823036003F018FE18B1BDE80840FFF79D
:1028F800B9BE08BD4C0300204FF0B04307B55A6E6F
:1029080042F001025A665B6E002203F00103019354
:1029180011463220019B02F07DF8322003B05DF8A9
:1029280004EB02F0A9B800000CB407B5054A05ABE2
:10293800102101930EF0DEF803B05DF804EB02B04D
:10294800704700BFAE0F010830B585B0044602A835
:102958000D460DF0FBFEBDF90C30064A0093102120
:10296800029B2046FFF7E0FF2046FEF725FD288062
:1029780005B030BDAE0F01084FF0B04210B59368F6
:1029880023F4004393600DF069FF0F4B01241C7082
:1029980000F0B8F80DF032FC0C480DF049FC0C4B77
:1029A8004FF400421A6120460DF048FCFFF7ACFADC
:1029B80000F014F900F00CFC0DF03CFD2146204617
:1029C800BDE810400DF056BD5803002051290008FD
:1029D800004000580DF064BD08B5FFF79DFA40F6B9
:1029E800B83398420CD8B0F5E16F0BD3FE23A0F5AD
:1029F800E16058434FF49663B0FBF3F0C0B208BDF2
:102A0800FE20FCE70020FAE77FB5684600F0CAF828
:102A18000198FFF753F800B207B05DF804FB000017
:102A2800194A38B5D2F88035591C044619D101F035
:102A38008DFB054601F096FB054401F08DFB2B0E3E
:102A4800E3712B0CA3712B0A6371030EE370C0F3BF
:102A58000742C0F307232571C0B2A27063702070CB
:102A680038BD190AC3718171190C1B0E41710371AC
:102A7800D2F88435C370D2F88405C0F30722C0F3B6
:102A88000743000EE9E700BF0070FF1F38B5094B88
:102A9800D3F8803503600133054609D101F056FBB0
:102AA800044601F059FB444001F05CFB44402C60B3
:102AB80038BD00BF0070FF1F012102200DF0C4BC0B
:102AC800002102200DF0C0BC00207047024B18788E
:102AD80008B100F0BBB870475803002082B00190DD
:102AE800019802B000F04EB94FF0B04382B0DA6CF2
:102AF80042F00202DA64DB6C03F002030193019BEB
:102B080002B070472DE9F043254C87B001F030FB47
:102B180001F036FB01F03CFB0123002502934FF442
:102B28008059032301A9204604934FF400580395C4
:102B38000595FFF7D9FFFFF7D7FFFFF7D5FFFFF799
:102B4800D3FFCDF8049002F0BFFA01A920464FF454
:102B58000067CDF8048002F0B7FA01A920464FF4C7
:102B68000046019702F0B0FA01A92046019602F04A
:102B7800ABFA2A464946204602F0CCFB2A46414693
:102B8800204602F0C7FB2A463946204602F0C2FB1F
:102B98002A463146204602F0BDFB07B0BDE8F08367
:102BA8000004004810B50446FFF7D0F9074BA360AE
:102BB80040F30F20FEF72EFF054B064A2360064B15
:102BC8006060C4E90323002010BD00BF0000484234
:102BD80000007A440D093E00AB0305000020704751
:102BE800014B1868704700BF5C0300200320704742
:102BF80008B501464FF47A7200238002890DFEF76A
:102C080083FF08BD4FF47A73A0FB0303800A40EAF0
:102C180083507047034B98689A689042FBD1C04331
:102C2800704700BF0028004008B5FFF7F3FF014BCD
:102C3800186008BD5C03002008B5FFF7EBFF024BE6
:102C48001B68C01A08BD00BF5C030020024B18783F
:102C580008B1FFF7DFBF70475903002010B5074BD5
:102C6800074C0122DA654FF48071204603F006FA1A
:102C78004FF0FF332363002010BD00BF0028004041
:102C8800E802002002460021014803F010BC00BF02
:102C9800E802002002460121014803F008BC00BFF9
:102CA800E802002010B58CB02C220021044601A8AF
:102CB8000EF04EF8FFF7D2FF0C4B0D481B681C4472
:102CC8000023089306934FF00053E443079301222F
:102CD8004FF4807301A902940B9303F0E5FA08B14D
:102CE800FFF7C0FC00200CB010BD00BF5C03002043
:102CF800E802002038B50546FFF78CFF022104469C
:102D0800074803F0DBFBC4F309024FF47A71A2FB16
:102D18000121920AA30A2A8043EA805038BD00BFE5
:102D2800E80200200148002103F0C8BBE8020020A7
:102D38000148012103F0C2BBE8020020F8B50F4D9D
:102D48002E78CEB90E4C4FF0FF372763FFF78CFC77
:102D5800FFF784FF4FF48071204603F08FF9204677
:102D6800276303F04FFB32462046022103F09FFB06
:102D7800FFF75AFF01232B700020F8BD59030020EC
:102D8800E8020020014610B54FF47A720023800251
:102D9800890DFEF7B9FE0146FFF73CFF0446FFF731
:102DA80039FF031B8B4200D310BD00BFF7E70DF0BE
:102DB8005DBE000010B5064C0221204603F07EFBE4
:102DC8000221421C2046BDE8104003F070BB00BF42
:102DD800E80200201648174A08B54FF4E133C0E965
:102DE800002300230C22C0E90233C0E90523C0E90F
:102DF8000733C0E90933036104F0EDFC08B1FFF7BC
:102E080031FC0B48002104F062FE08B1FFF72AFCF0
:102E18000748002104F07BFE08B1FFF723FC0448B3
:102E280004F035FE18B1BDE80840FFF71BBC08BD2B
:102E3800200400200044004070B596B005461422D6
:102E4800002103A80DF084FF3822002108A80DF006
:102E58007FFF2A68334B9A4261D10223089308A85E
:102E6800314B0A9303F03AF808B1FFF7FBFB4FF038
:102E7800B0430C219A6D2D4C42F400329A659A6D3C
:102E880002F400320292029ADA6C42F00102DA6429
:102E9800DB6C03F001030193019B02230026CDE9BB
:102EA80003130323CDE905634FF09040072303A9DB
:102EB800079302F009F91E4826621423C4E90003A7
:102EC8001023C4E9023620468023C4E90436C4E945
:102ED800066601F031FE08B1FFF7C4FB154AEC673E
:102EE800A562154C1323C4E9002320460023802241
:102EF800C4E90233C4E90423C4E90633236201F0B8
:102F08001BFE08B1FFF7AEFB2520C5F88040002264
:102F18000221A56201F07EFD252001F0ADFD16B06D
:102F280070BD00BF0044004004000C00C003002036
:102F3800800002406C0002406003002002680E4BD3
:102F48009A4210B5044616D14FF0B0420C21936D49
:102F580023F4003393654FF0904002F061F9E06F7D
:102F680001F05EFED4F8800001F05AFEBDE8104082
:102F7800252001F08FBD10BD0044004008B50A4669
:102F88000146024803F0AAFD002008BD20040020E5
:102F980013B5114B114C18604FF40013009302AB9A
:102FA80013E90600204604F016FD2368DA69D10308
:102FB800FCD4DA695202FCD59A68084842F48002C7
:102FC8009A6004F04EFD06490448012204F0BCFC56
:102FD800002002B010BD00BFB4040020200400206F
:102FE800BC04002008B5074B1860FFF70CF8FFF782
:102FF800F1FE054AD2F8803043F00063C2F8803011
:10300800002008BDB80400200008005808B54FF09B
:10301800B04308489A6B42F400329A639A6B22F4E0
:1030280000329A63FFF78AFF0F2001F033FD00207A
:1030380008BD00BF2004002008B5074804F0CBFBFA
:1030480008B1FFF70FFB054801F076FD18B1BDE8A0
:103058000840FFF707BB08BD20040020C00300207C
:103068000268044B9A4203D1034B00201B6818479F
:10307800704700BF00440040B804002002680B4BB2
:103088009A4210B504460FD1094B1B682BB1D0F8F2
:10309800902012B907480121984720460549BDE804
:1030A8001040012204F050BC10BD00BF0044004095
:1030B800B4040020BC04002010B50A4C23780BB9D6
:1030C800E37C6BB1FFF7E6FB0038074B18BF012024
:1030D800400018701B78022B02BF00232370E37492
:1030E80010BD00BFDE060020D004002038B5114C0A
:1030F8002378F3B9E37CE3B90F4D2B68012B07D98B
:103108002B68042B04D80D4A0421012000F034FA5E
:103118002B68042B0DD9FFF7BDFB0038084B18BFEF
:103128000120400018701B78022B02BF0023237077
:10313800E37438BDDE060020CC0400200810010826
:10314800D004002038B50C4D0C4C0122082128462B
:1031580002F0E0F84FF47A70FFF7C0FC4FF480619A
:103168004FF0904002F0D0F8002220700821284645
:1031780002F0D0F8237838BD00040048D1040020BC
:1031880070477047022808B50ED801221021074859
:1031980002F0C0F83220FFF7A1FCBDE80840034860
:1031A8000022102102F0B6B808BD00BF0004004894
:1031B800054B1B78B3FA83F35B0903710023437152
:1031C800024B01221A707047D1040020DD0600204E
:1031D800034A002313715371024A1370704700BFEA
:1031E800BE040020DD060020704708B5FFF7C4FBC9
:1031F800BDE8084000F05EBB4FF0FF300DF0B4B9F9
:1032080070477047014BD870704700BF5C000020C2
:10321800014B1874704700BF5C00002020B1037890
:1032280013B102480DF0D0BB704700BF1406002050
:1032380008B5022000210DF05FF9BDE808400148FB
:103248000DF0C2BB2C060020002101200DF054B95E
:1032580010B5094C60B1206008480DF067FB216883
:1032680006480DF0EBFBBDE8104004480DF0ACBB80
:1032780042F210732360EFE7740000202C06002050
:1032880010B5094C206023680BB9084B2360084827
:103298000DF04CFB216806480DF0D0FBBDE810404E
:1032A80003480DF091BB00BF0C000020A086010070
:1032B8004406002038B504460D4607484FF400611F
:1032C800FFF750F830B92A4621460348BDE8384090
:1032D800FEF74ABF38BD00BF00F003080A4601499F
:1032E800FFF720B800F0030838B50C480DF01EFBB6
:1032F80005F072F860B90A4C0A480125257004F0F7
:10330800FDFE2078294604F04FFC04480DF05CFBD4
:10331800BDE8384004480DF057BB00BF2C0600201C
:10332800000000205C000020FC05002005F0F0B83B
:1033380030B585B0FFF750FB0446FFF703FF68463A
:10334800FFF736FF3B4B07221A703B4A11780029DA
:103358003FD00021117008221A70384A5968127833
:1033680062F07F020A705A6824B204EB440404EB4A
:103378004414FE21B4FBF1F4547002223049314C5C
:103388000978012988BF00225A70637A33B104F0A2
:10339800EDFC012802D120460DF0C8FA2A4B254839
:1033A800D978002204F00CFD063041D104F0D8FC95
:1033B800044626480DF0BAFA254B24481968A1425C
:1033C80038BF21460DF03AFB20480DF0FDFA05B054
:1033D80030BD204920480A7822B9057805F0FF0257
:1033E800002DCBD00022027014480A70596800786A
:1033F800087059684A705A68562191705A680121B4
:10340800D1705A6824B204EB4404FE2104EB44143E
:10341800B4FBF1F414715A68022151715A689DF88D
:10342800051091715A689DF80410D1710822A5E71A
:103438000024BEE7040000205C060020C40500202C
:10344800D0040020C80500205C0000202C060020C5
:1034580074000020F3060020DD06002008B5104B9C
:103468000122002102201A700DF046F80D480DF0D7
:10347800ABFA0D4B1B788BB10C4B1A7872B9DB7C0D
:1034880063B90B4B1A68042A9EBF1A6801321A6086
:103498000021BDE8084010200DF02EB808BD00BF7F
:1034A8005C06002044060020F8050020DE06002007
:1034B800CC040020044B1B78022B03D100210820E8
:1034C8000DF01AB8704700BF0000002008B504F0DE
:1034D8008CFF80B904F04AFC01280CD1BFF34F8F50
:1034E8000549064BCA6802F4E0621343CB60BFF398
:1034F8004F8F00BFFDE708BD00ED00E00400FA05AE
:1035080010B5044690B190F906307BB908480DF023
:103518000DFA084BE2791A70074B1868FFF7B0FEEE
:10352800064BBDE810401868FFF792BE10BD00BFFB
:10353800C8050020F80500200C00002074000020B9
:1035480070477047704770477047012808B50146B3
:1035580002D002280CD008BD4FF0904001F0D4FEF4
:103568000128F8D100210220BDE808400CF0C4BFB2
:1035780000210820F8E7000070B505460C461646FD
:1035880004F008FC0346002834D000241A480DF043
:10359800CDF91A4B18481968A14238BF21460DF0D9
:1035A8004DFABDE8704014480DF00EBA4A68F05C58
:1035B800D0540133DAB29442F8D8114B0D701B780D
:1035C800012B88BF00244C700E4C637A33B104F091
:1035D800CDFB012802D120460DF0A8F90A4B0B4873
:1035E800D978002204F0ECFB0630CED104F0B8FB09
:1035F8000446CBE70549DDE72C06002074000020CF
:10360800D0040020C80500205C0000200400002031
:10361800044B1B7823B9044A05210120FFF7ACBFEE
:10362800704700BFD00400200D10010810B5002419
:1036380090B03C22214601A800940DF089FB2F4B45
:103648002022DA7219788DF8001059788DF8011057
:1036580099788DF80210D9788DF8031019798DF8BA
:10366800041059798DF8051099798DF80610D979D3
:103678008DF80710197A8DF80810597A8DF8091005
:10368800997A8DF80A108DF80B2021460DF10B025E
:1036980058180131007B02F8010F1C29F8D193F862
:1036A80028208DF8282093F829208DF8292093F8D0
:1036B8002A208DF82A2093F82B208DF82B2093F8B8
:1036C8002C206AB193F83F2052B10DF12B01002252
:1036D8009818013290F82C0001F8010F142AF7D13C
:1036E80007484FF40061FEF73DFE20B90448402228
:1036F8006946FEF739FD10B010BD00BF7800002004
:1037080000F80308014940220CF0EABE00F803085B
:1037180070B52A4D28796B794D2BC0B233D1C0EBE7
:10372800001080000A2838BF0A204FF47A735843E3
:10373800234BAC791860EB794D2BE4B22BD1C4EB59
:103748000414A40095F82C301E4E63BB95F83F3046
:103758004BBB42F21070FFF77BFD3068FFF790FD1E
:103768002B7A194A1949DBB213706B7A184ADBB203
:1037780013700023EA1892F82C20D2B2CA540133ED
:10378800142BF7D170BD6B79482B0ABF4FF46163D6
:103798006B795843C6E7EB79482B0ABF4FF461634E
:1037A800EB795C43CEE7FFF753FD012C38BF0124CA
:1037B8004FF47A735C433460CFE700BF7800002091
:1037C800740000200C000020F2060020DE06002015
:1037D800D004002010B590B000213C2201A800912F
:1037E8000DF0B6FA4022314968460CF079FE9DF892
:1037F80000203AB99DF80100562803D19DF802101F
:10380800012909D0FFF712FF4FF47A70FFF766F924
:10381800FFF77EFF10B010BD254B1A7058709970D5
:103828009DF80310D9709DF8041019719DF80510C2
:1038380059719DF8061099719DF80710D9719DF876
:10384800081019729DF8091059729DF80A1099729A
:103858009DF80B1001F03F01D972D87AD1B2884295
:103868001BD89DF8282083F828209DF8292083F864
:1038780029209DF82A2083F82A209DF82B2083F8F8
:103888002B200DF12B0100229818013211F8014F5D
:1038980080F82C40142AF7D1BAE701F140006844B7
:1038A800194410F8340C08730132D6E700F80308FD
:1038B800780000201FB5002403A92046039404F0D3
:1038C80077FD03A9012004F073FD384B38480094B4
:1038D80022464FF4FA710CF0CBFF364B3648009471
:1038E80022464FF4FA710CF0C3FF344B344800946D
:1038F80001224FF4FA710CF0BBFF2046FEF72EFCB4
:1039080008B1FEF7AFFE2F4B009400224FF4FA6186
:103918002D480CF0ADFF2D4A002101200CF0A8FE27
:103928002B4A002102200CF0A3FE2A4A0021042081
:103938000CF09EFE284A002108200CF099FE00F0A9
:1039480039FB2649264804F0E9FC264804F0D6FB52
:103958001B480DF039F8244B0021187804F024F99D
:1039680022490094224B0968224800220CF080FF6B
:1039780020480DF029F8FFF72DFF1F4A00211020DD
:103988000CF076FE1D4A00214FF480600CF070FEAA
:103998001B4B1C4819681C4B009400220CF068FF54
:1039A80018480DF011F804B010BD00BF4D350008DF
:1039B800140600204F350008E005002049350008AE
:1039C800C8050020BD340008FC050020FD7E000865
:1039D8003933000835330008F132000800000301CC
:1039E800100000205C00002000000020740000206F
:1039F800393200082C060020F53000084D31000847
:103A08000C000020440600206534000830B500246E
:103A1800A3B07C22214603A802940DF099F9532300
:103A28008DF808304FF4AB73ADF80A3001238DF8E8
:103A38000C30ADF80440FEF7CFFF00B200EB4000B9
:103A480000EB4010FE23B0FBF3F08DF80D0001A849
:103A580000F055FBC0B143000133DBB20B4C8DF8CD
:103A68000E302C228021201D1D460DF071F9029880
:103A7800BDF80C302060A380A571224607210120E3
:103A8800FFF77AFD23B030BD5823E7E75D06002035
:103A980070B50378592B90B0044640F0C0810529D1
:103AA80059D84378443B162B55D8DFE813F010015A
:103AB80054000001540008015400540054005400FC
:103AC80073005400EB005400540054007701540074
:103AD80054008F0054005400540017008578482D76
:103AE80011D1A64A14210120FFF746FD41F2883082
:103AF800FEF7F4FF40F6B830FEF7F0FF10B0BDE86F
:103B08007040FFF7E3BC532D0ED1302280219C4832
:103B18000DF01EF9FFF77AFF41F28830FEF7DEFF5D
:103B2800974A1521012065E0432D16D100246846E7
:103B38008DF8004004F05AFA914A4C23137056232A
:103B480093709DF80030547001204133D070137188
:103B58000521FFF711FD10B070BD442DFBD1884C35
:103B68002C228021201D0DF0F3F8002325706370AE
:103B780001255623A370E5702571FEF72DFFFE235E
:103B8800B0FBF3F000EB400000EB40106071224600
:103B98000621C7E78378303BDBB2092BDBD87949AC
:103BA800794A0B700B78DBB25372754A592313703C
:103BB8004D2353700B783033937003210120FFF7A6
:103BC800DBFC10B0BDE87040FFF730BD8578482DAC
:103BD80015D16B4A5623137093700323137117235F
:103BE80053710B2300210120937112235170D0705F
:103BF800D371082110B0BDE87040FFF7BDBC432D5C
:103C0800A9D15F4C00213C2201A800910DF0A0F839
:103C18006846FFF777FD2422802104F10C000DF09F
:103C280097F89DF8003063709DF80130A3709DF8F7
:103C38000230E3709DF8033023719DF804306371FE
:103C48009DF80530A3719DF80630E3719DF80730A3
:103C580023729DF80830257063729DF80B509DF80B
:103C68000930A3729DF80A30E3722A4603A9257326
:103C780004F10D000DF09DF805F10D012246C9B2C1
:103C8800012066E7807839280CD83038C0B2FFF7B1
:103C980077FA3B4A2378137063785370A37893704C
:103CA80003213FE710B0BDE87040FFF7B1BC807852
:103CB8003928F7D83038C0B2FFF763FAE9E78078D7
:103CC8003928EFD83038C0B2FFF75CFAE1E78378DB
:103CD800303BDAB2092AE5D8C0783038C2B2092AAE
:103CE800E0D82179A1F14802D2B20B2ADAD8274DBF
:103CF80045FA02F2D207D5D40A224D2902FB030065
:103D080036D13C2358434FF47A735843204B1860FC
:103D1800204B1860FFF79CFA194A237813706378D0
:103D28005370A3789370E378D370237913710521C6
:103D38000120FFF721FC144B00221A7056225A70FA
:103D480001229A70DA70A278303A02EB8201E278A6
:103D5800303A02EB4102D2B21A7122795A710E4AF4
:103D68001278D2B21A72074A1278D2B25A7228E777
:103D78004829C8D14FF46163C4E700BF1310010894
:103D88005D060020D004002078000020DEF7FFFF49
:103D9800740000200C000020F20600208678A6F1AE
:103DA8003003092B3FF67EAFC078A0F13003092B12
:103DB8003FF678AF2179A1F14802D2B20B2A3FF63B
:103DC80071AF5A4B134113F001057FF46BAF584A9A
:103DD8005923137053235370D070117196700521B5
:103DE8000120FFF7C9FB534956230D704B7001237F
:103DF8008B70CB70A378303B03EB8302E378303BC6
:103E080003EB4203DBB28B712379CB714A4B1B78EE
:103E1800DBB20B72494B1B78DBB24B72D1E6502BED
:103E280048D102297FF697AE4378303B012B3FF605
:103E380092AE8378312B7FF48EAE0B2904D8FFF72E
:103E4800E7FB00213A4A6DE63A4D0234002214F8A5
:103E5800013FA918303B0132DBB20C2A0B73F6D1B3
:103E6800FFF7C2F9324B502256211A70997000227E
:103E780001215A70D97003F8041FA9180132097B6F
:103E88000C2A01F1300103F8011FF6D100232B7031
:103E980056236B700123AB70EB70274B1B78DBB29A
:103EA8002B72264B1B78DBB26B72EA72FFF7BEFBF4
:103EB8001121C7E7412B7FF44EAE4378432B7FF4A3
:103EC8004AAE16297FF447AE1D4D421C002312F856
:103ED800011FE9540133142BF9D1FFF7EDF8194B01
:103EE8005B7D012B19D113490023EA5CC818013303
:103EF800D2B2142B80F82C20F7D1104B00221A7064
:103F08001B78DBB24B72FFF791FB094A631E15342D
:103F1800A34206D1064A162104E6084B02221A706B
:103F2800F3E713F8011F02F8011BF1E7DEF7FFFFC3
:103F38005D06002078000020F2060020D004002052
:103F4800DE0600203403002038B504460D4661B370
:103F580016480CF039FD2B783BB334B360682378EE
:103F680018B3032B0CD0072B17D0022B1DD1617867
:103F780001291AD00B0618D4BDE83840FFF788BDD0
:103F88006378012B11D10078012802D0022800D0D3
:103F980058B9BDE8384003F0DFBF6378012B04D17E
:103FA8000378034A03F00103137038BDE0050020CD
:103FB800C4050020034B0022C3E902220122C3E901
:103FC80000227047F406002000487047F4060020DD
:103FD8004FF0B04382B0DA6C0243DA64DB6C034022
:103FE8000193019B02B070472DE9F04186B000248F
:103FF8000220154D0594FFF7EBFF0420FFF7E8FFBB
:10400800124F03944FF4807601230DEB0001CDE9A4
:1040180001632846032304934FF4005801F054F831
:1040280001A93846CDF8048001F04EF822464146F1
:10403800384601F06FF928462246314601F06AF900
:10404800204606B0BDE8F08100040048000800489A
:10405800032810B50ED8012810D868B902460B48B5
:104068004FF4807101F056F9002209484FF40051CD
:1040780001F050F9002010BD0122F0E700220348AA
:104088004FF4807101F046F90122EEE70004004880
:104098000008004802207047002070470120704740
:1040A80000280CBF0F201620704700000D488546D9
:1040B80000F027F80C480D490D4A002302E0D458B7
:1040C800C4500433C4188C42F9D30A4A0A4C00235A
:1040D80001E013600432A242FBD30CF041FEFEF76C
:1040E800AFFAFEE700000120000000204C0100208C
:1040F8000C1B01084C01002090240020FEE7002042
:104108007047704710B5032000F072FC01F018FBEF
:10411800064B18600F20FEF7D7FC044618B9FEF7C7
:1041280044FB204610BD0124FBE700BFB800002077
:104138004FF0E022136923F00203136170474FF038
:10414800E022136943F0020313617047014BD3F86F
:10415800900570470070FF1F014BD3F89405704716
:104168000070FF1F014BD3F8980570470070FF1FC0
:10417800024A536823F0010353607047002004E0AB
:10418800024A536823F0020353607047002004E09A
:10419800024A536823F0040353607047002004E088
:1041A8008068C0F380007047F7B500230193044688
:1041B800002800F0E980856D25B9FDF74FFEE5651B
:1041C80084F8545023689A68D00040F1A1809A6816
:1041D800D10000F1B480A26D42F01002A265E26D38
:1041E80042F00102E26501251846FFF7D9FFA26DEA
:1041F80002F01002024340F0C980A26D206922F447
:10420800817242F00202A2659A68D2075DD4226BDD
:10421800A67E94F82CC0003A18BF01221703D4E9EF
:1042280002120A43217E42EA8132617E42EAC132A9
:1042380042EA4632002842EA4C02B4BF20F000416C
:104248004FF400113A430A4394F82010012903D18E
:10425800002E76D142F48032616A21B1A66A01F457
:10426800E07131430A43D968E66C21F4FE3121F448
:10427800FF711143D96094F83C206168012A01F06C
:10428800404C4CEA060609D1D4E910273A43324398
:10429800A66C324342EA0C0242F001061F693E4A0C
:1042A8003A4032431A6121F00042B2F1804F0CD0FB
:1042B800B1F1004F09D0394ED6F8082701F4701132
:1042C80022F470120A43C6F808275A69666BA16B74
:1042D80022F0070232435A615A6922F0700242EA18
:1042E80001125A61002835D19A6A62F00F029A6267
:1042F8005B6903F007039E423CD10023E365A36D8D
:1043080023F0030343F00103A365284603B0F0BD7F
:104318009A68234922F0104222F0170242F0805294
:104328009A60204A1268B2FBF1F2013252000192FF
:10433800019A002A3FF44BAF019A013AF7E70025AA
:1043480052E7A16D41F02001A165E16D41F0010145
:10435800E16581E7B0F5001FCAD19A6AE269013ABE
:1043680092006FF00F0102F01C0201FA02F2216EB6
:104378000A43BCE7A36D23F0120343F01003A365BF
:10438800E36D43F00103E3650125BEE7A36D43F048
:104398001003A365F8E700BF02FCFF1F00200140DF
:1043A800400D0300B8000020F8B54569082D044603
:1043B8000E460AD00368DB68D80705D5A36D43F01D
:1043C8002003A3650120F8BD0425FEF77FFB0746FF
:1043D80023681A682A4221D0A26D42F40072A265AD
:1043E800DA6812F4406F14D1A27E92B91A681207E3
:1043F8000FD51846FFF7D4FE28BB5A6822F00C02E6
:104408005A60A26D22F4807222F0010242F0010289
:10441800A265207E00BB0C221A60D4E7711CD8D09C
:10442800FEF754FBC01BB04201D8002ED0D1236840
:104438001B682B40CCD1A26D84F8543042F00402A2
:10444800A2650320BFE7A26D42F02002A265E26DDB
:1044580042F00102E265DCE70020B4E70368186C6B
:1044680070470000F7B50023019390F85430012BF2
:10447800044600F0C58005680669012380F85430B9
:104488002846FFF78DFE002840F0B480D1E90020CF
:10449800022826F0040300F08280B3F1004FC2F333
:1044A800110E13D1AB6A43EA0E03AB628B686869DD
:1044B80003EA022323F07C4323F0FF0320EA0221CE
:1044C8000B43002A6B6126DB002055E0236E00F0C9
:1044D8001F074FF00F0C0CFA07FC6FEA0C0623EAD3
:1044E8000C0CBEF1000F11D1C2F38463BB4043EA48
:1044F8000C0323668008E36901309842D6D8A86A7D
:10450800C2F38363BB4006403343CEE792FAA2F37B
:10451800B3FA83F3EAE73B493B48D1F808378242CC
:1045280003F0E07519D11B02CED4D1F8083723F077
:10453800E0732B4343F40003C1F80837334B1A6880
:10454800334BB2FBF3F20C2302FB03330193019BC1
:10455800002BB9D0019B013BF8E72E48824210D1CD
:1045680013F08070B0D1D1F8083723F0E0732B43F3
:1045780043F08073C1F80837002384F8543003B03F
:10458800F0BD254882429FD113F480009CD1D1F818
:10459800083723F0E0732B4343F48003EAE7B3F1D1
:1045A800004F01BFAB6AC2F311018B43AB62002A13
:1045B8008ADA154813498242D1F8083709D1D1F867
:1045C800082703F0A07322F0E0721343C1F80837FC
:1045D8007AE71048824204D1D1F8082703F440034F
:1045E800F1E70D4882427FF46FAFD1F8082703F056
:1045F800C073E8E7A26D42F02002A2651846BBE747
:104608000220BCE700200140001000B0B8000020E4
:10461800400D0300004000B8002000B4026838B51F
:1046280004461046FFF7BCFD08B9002038BD936862
:10463800990707D4936823F0004323F0170343F046
:1046480010039360FEF742FA054623689B685B07F0
:10465800EBD5FEF73BFA401B0228F6D923689B6886
:104668005A07F2D5A36D43F01003A365E36D43F039
:104678000103E3650120D9E773B5002302680193BC
:104688009368DD07044602D5002002B070BD91682A
:10469800214B194209D0A36D43F01003A365E36DC4
:1046A80043F00103E3650120EFE7936823F000433B
:1046B80023F0170343F001039360184BD3F808372E
:1046C80018021CD4637E012BDED0FEF7FFF9144ECE
:1046D800054622681368DB07D6D49368D9075FBFFD
:1046E8009368334043F001039360FEF7EFF9401BF2
:1046F8000228EED923681B68DA07EAD4CBE7094B0E
:10470800094A1B68B3FBF2F301330193019B002BA9
:10471800D8D0019B013BF8E717000080002001403A
:10472800E8FFFF7FB8000020400D030038B50446BD
:104738000068FFF735FD054620BB94F85430012B7F
:1047480020D0012384F854302046FFF795FFB0B9F4
:10475800A36D226823F4706323F0010343F480738C
:10476800A3651C23E065136084F85400936823F064
:10477800004323F0170343F00403936038BD84F823
:104788005450FBE70220F9E7026838B5936891684E
:104798000446C80701D4002038BD9907FBD49368A4
:1047A80003F00503012B19D1936823F0004323F08C
:1047B800170343F00203936003231360FEF786F99F
:1047C800054623689B68DB07E5D5FEF77FF9401BA4
:1047D8000228F6D923689B68DA07F2D5A36D43F05F
:1047E8001003A365E36D43F00103E3650120D3E7FC
:1047F80070B5044600284BD0836D43F002038365EF
:10480800FFF70CFF054668B92046FFF7BDFF0546D0
:1048180008B90123A3652268936823F0104323F0A5
:104828001703936023685A6822F4677222F0030220
:104838005A6040F29F321A60D968164A0A40DA6014
:104848001A6922F040421A615A6922F007025A6135
:104858001A6A02F0F0221A625A6A02F0F0225A62C8
:10486800DA6A02F0F022DA629A6A0B4A00269E623D
:10487800D2F8083723F0FE73C2F808372046FDF750
:1048880001FBE6652666A66584F85460284670BD77
:104898000125FBE700023E830020014010B590F897
:1048A8005430012B044615D0012380F85430FFF70B
:1048B800B5FE58B92046FFF767FF38B9A36D23F452
:1048C800807323F0010343F00103A365002384F8F8
:1048D800543010BD0220FCE7F7B50023019390F88F
:1048E8005430012B04467FD0012380F85430FFF761
:1048F8004BFF23689A6812F00102054607D0A36DA2
:1049080043F01003A365002384F854302DE0A16D13
:10491800364F21F4817141F00201A165DE68D96842
:1049280026F4FF4626F07C0621F40041360421F0E7
:104938000301360CD96008209968394041F00041DC
:1049480099609968002913DA019901310191019957
:10495800B1F52E3FF5D3A36D23F0120343F01003F6
:10496800A365002384F854300125284603B0F0BD20
:10497800D3F8B410013801F07F010A44DCD19968FA
:104988001A48014041F001019960D3F8B41021F0B0
:104998007F0141EAD202C3F8B4209A68024042F08B
:1049A80002029A60FEF792F8074623689A68D207CF
:1049B80008D4DA683243DA60A36D23F0030343F0C6
:1049C80001039FE7FEF782F8C01B0228EDD9236890
:1049D8009B68D907E9D5A36D43F01003A365E36D80
:1049E80043F00103E365BFE70225BEE7E8FFFF7F69
:1049F8000749CA6822F4E0620302120403F4E06380
:104A0800120C134343F0BF6343F40033CB60704789
:104A180000ED00E0164B30B5DC68C4F30224C4F1A5
:104A28000703251D042B28BF0423062D4FF0FF354F
:104A38008CBF033C002405FA03F321EA0303A540D5
:104A480022EA0502A340002843EA0203ACBF00F1B2
:104A58006040084A4FEA0313B8BF00F00F00DBB20A
:104A6800AABF00F56140135480F8003330BD00BF81
:104A780000ED00E014ED00E0002807DB044A4109DE
:104A8800012300F01F00834042F82130704700BF27
:104A980000E100E000280CDB4309064900F01F0094
:104AA80020330122824041F82320BFF34F8FBFF308
:104AB8006F8F704700E100E070B5D0E9134565607D
:104AC800446D14B1D0E916456560D0E9105404F07E
:104AD8001C060124B4406C60046863608368102B72
:104AE8000BBFA260A160E160E26070BD0268416C2A
:104AF800D3B210B5083B1424B3FBF4F30B4CA24219
:104B080088BF0B4A21F0030199BF01F1804202F5E9
:104B18000232521807338264064AC26403F01F0344
:104B2800012202FA03F3036510BD00BF0704024027
:104B38001C0802408008024038B500285ED0026890
:104B48002F4B9A424FF014014CD82E4B1344B3FB11
:104B5800F1F32D499B00C0E91013022380F825309A
:104B68001368056923F4FF4323F070031360D0E949
:104B7800024323432B43456911682B4385692B4323
:104B8800C5692B43056A2B430B431360FFF7AEFF40
:104B9800B4F5804F04BF002343604268816C02F083
:104BA8007F030B60D0E91314013A032A4C6020D824
:104BB800164A174981651A44013B9200012103F006
:104BC800030301FA03F300214265C3651160114A2A
:104BD800536400230122C36380F8243080F8252021
:104BE800184638BD0C4B1344B3FBF1F30B499B003B
:104BF800B1E70023C0E91533C365EAE70120F0E710
:104C080007040240F8FFFDBF000002403F82001089
:104C18004009024000090240F8FBFDBF00040240C1
:104C280038B5002841D00268136823F001031360E7
:104C38001F4B9A424FF0140130D81E4B1344B3FB5C
:104C4800F1F31D499B00C0E91013012403F01C0374
:104C580004FA03F3002515604B60FFF747FF836CE8
:104C680041681D60D0E913325A604A1E032A06D8EB
:104C7800124B0B449B0094401D60114B5C64002355
:104C8800C363C0E91533C0E90B33C0E90D33C3650D
:104C980080F8253080F82430184638BD094B134475
:104CA800B3FBF1F308499B00CDE70120F5E700BF0E
:104CB80007040240F8FFFDBF000002403F820010D9
:104CC80000090240F8FBFDBF0004024070B590F8EF
:104CD8002450012D04463BD090F825600125AE42B2
:104CE80080F824504FF000062CD1022580F825507A
:104CF8000568C6632E6826F001062E60FFF7DCFE05
:104D0800036BBBB12B6843F00E032B60A36C1A68CE
:104D1800D20342BF1A6842F480721A60636D1BB1F5
:104D28001A6842F480721A602B6843F001032B6002
:104D3800002070BD2B6823F004032B602B6843F020
:104D48000A03E2E78023C36380F824602846F0E77B
:104D58000220EEE7034640B190F82520022A06D04B
:104D68000422C263002280F82420012070470268D0
:104D7800806C116821F00E011160016821F48071C6
:104D88000160116821F001011160D3E9100202F0FD
:104D98001C0101228A404260D3E9132151605A6DF7
:104DA80032B1116821F480711160D3E91621516084
:104DB8000122002083F8252083F82400704710B5CD
:104DC80090F82530022B03D00423C363012010BDC3
:104DD80003681A6822F00E021A601A6822F00102AB
:104DE8001A60826C136823F480731360D0E910137F
:104DF80003F01C02012393404B60D0E913325A6040
:104E0800436D33B11A6822F480721A60D0E9163201
:104E18005A60012380F82530836B002480F82440F1
:104E280013B198472046D2E71846D0E770B4426CD1
:104E3800046C036826681D6802F01C020421914076
:104E480031420FD015F0040F0CD01A6892065EBFDD
:104E58001A6822F004021A60036B6160002B33D0D9
:104E680070BC184702219140314217D015F0020F4B
:104E780014D01A68940606D41A6822F00A021A6036
:104E8800012280F82520114A93428CBF104B114B08
:104E98005960002380F82430C36ADFE70821914075
:104EA800314211D029070FD5196821F00E01196078
:104EB800012303FA02F26260C36380F825300023FD
:104EC80080F82430436BC9E770BC7047800002400B
:104ED80000040240000002400A4A536943F4802358
:104EE80030B55361EFF3108472B60023CD58C55026
:104EF8000433B3F5807FF9D11369DB03FCD484F361
:104F0800108830BD00400058064B5A69002ABFBFC0
:104F1800054A9A6002F188329A60BABF5869C00F90
:104F2800002070470040005823016745044B5A6928
:104F380042F000425A615869C043C00F704700BF31
:104F48000040005870B50546FDF7C0FD124E0446F6
:104F58003369D90313D43369DA0744BF01223261B4
:104F68004CF2FA32134011D10B4E306910F4802004
:104F78000BD0FDF7ABFD001BA842F6D304E0FDF70C
:104F8800A5FD001BA842E3D3032070BD024A1361AC
:104F9800024A01205360F8E7004000580407002047
:104FA8002DE9F041184D98462B78012B06460C4602
:104FB800174626D001232B704FF47A7000236B60BC
:104FC800FFF7C0FFA0B9012E16D1104A536943F06C
:104FD800010353612760BFF36F8FC4F804804FF457
:104FE8007A70FFF7AFFF094A536923EA0603536152
:104FF80000232B70BDE8F08139462046FFF76CFF8F
:10500800EDE70220F6E700BF040700200040005843
:10501800054A536923F47E7343EAC00040F48030A4
:1050280040F0020050617047004000582DE9F041FF
:10503800234F3B78012B054688463FD001233B7020
:105048004FF47A7000237B60FFF77CFF044688B931
:105058002B68042B13D11B4A536943F4803343F064
:10506800040353614FF47A70FFF76CFF0446154B45
:105078001A681B6800233B702046BDE8F0814FF09A
:10508800FF33C8F800306E68D5E901321344B342E3
:105098000AD93046FFF7BCFF4FF47A70FFF752FF8A
:1050A80050B1C8F800600446064A536923F47E7379
:1050B80023F002035361DAE70136E5E70224DBE770
:1050C80004070020004000582DE9F04F524C0023FF
:1050D8004FF00F090A6832FA03F501D1BDE8F08FE5
:1050E800012505FA03F818EA020200F08E804E68DE
:1050F800032706F003054FEA430E07FA0EFC6F1E5E
:10510800012F6FEA0C0C32D8876807EA0C0ACF68BF
:1051180007FA0EF747EA0A078760476827EA080888
:10512800C6F300179F4047EA08074760C76807EAC1
:105138000C088F6807FA0EF747EA0807022DC760C0
:1051480017D14FEAD30800EB880803F0070AD8F80C
:1051580020704FEA8A0A09FA0AFB27EA0B0B0F6943
:1051680007FA0AF747EA0B07C8F8207001E0032D91
:10517800DCD1076805FA0EF507EA0C073D4316F47B
:10518800403F056041D023F0030707F1804707F54A
:10519800803703F0030CBD684FEA8C0C4FF0070E04
:1051A8000EFA0CFEB0F1904F25EA0E0E2FD01B4DD3
:1051B800A8422ED005F58065A8420CBF0225072518
:1051C80005FA0CF545EA0E05BD602568D74316F4C7
:1051D800801F0CBF3D4015432560656816F4001F0D
:1051E8000CBF3D4015436560D4F8805016F4803FED
:1051F8000CBF3D401543C4F88050D4F88450B60322
:1052080054BF3D401543C4F88450013362E700257C
:10521800D6E70125D4E700BF00080058000400487D
:10522800374A2DE9F04F00234FF0010A4FF0070BE2
:105238004FF00F0931FA03F401D1BDE8F08F0AFAF3
:1052480003FC1CEA010654D023F0030404F1804453
:1052580004F5803403F00307A568BF000BFA07F8CC
:10526800B0F1904F08EA050E45D0264DA84244D02B
:1052780005F58065A8420CBF02250725BD40754588
:1052880017D1D2F8805025EA0605C2F88050D2F826
:10529800845025EA0605C2F88450156825EA0605F3
:1052A8001560556825EA06055560A56825EA0805CC
:1052B800A560056803265C0006FA04F423FA06F6DE
:1052C800254300EB8606056003F00705376AAD0045
:1052D80009FA05F527EA05073762856825EA04050E
:1052E8008560456825EA0C054560C56825EA04041B
:1052F800C46001339EE70025C0E70125BEE700BF73
:1053080000080058000400480369194214BF01202E
:10531800002070470AB181617047816270470000C0
:10532800044AD168014208B502D0D060FEF70DF9F1
:1053380008BD00BF0008005810B5044600284AD030
:1053480090F8413003F0FF021BB980F84020FDF7C8
:10535800B7F8242384F8413023681A6822F0010240
:105368001A60626822F070621A619A6822F4004238
:105378009A60D4E90221012924D142F400429A60BA
:105388005A6842F0007242F400425A60DA6822F425
:105398000042DA60D4E904210A43A16942EA012201
:1053A800DA60D4E907210A431A601A6842F0010258
:1053B8001A6000202023606484F84130206384F858
:1053C800420010BD42F4044202299A6004BF4FF41F
:1053D80000625A60D4E70120F3E710B590F8412045
:1053E800202A0346D4B21CD190F84020012A18D0B4
:1053F800242280F841200268106820F00100106023
:10540800106820F480501060106801431160116822
:10541800002041F00101116083F8414083F8400009
:1054280010BD0220FCE710B590F84120202A034661
:10543800D4B21BD190F84020012A17D0242280F83A
:1054480041200268106820F001001060106820F404
:10545800706040EA012111601168002041F00101EB
:10546800116083F8414083F8400010BD0220FCE73A
:10547800024A136843F480731360704700040058AD
:105488000D4B10B55B690C4628B99A0507D500F095
:1054980027F820B110BD9B0501D400F019F8074A80
:1054A8001369012C23F00403136101D130BFF1E724
:1054B80040BF20BF20BFEDE70004005800ED00E02A
:1054C800024B186800F4C060704700BF0004005821
:1054D800024A136843F4804313607047000400587D
:1054E8000C4A136823F4804313600B4B1B6832216A
:1054F8004B430A49B3FBF1F35169890500D533B928
:10550800536913F4007F14BF032000207047013B48
:10551800F2E700BF00040058B800002040420F0026
:105528000B4A136823F0070343F002031360094B87
:105538001A69012842F004021A6105D130BF1A69BC
:1055480022F004021A61704740BF20BF20BFF6E76F
:105558000004005800ED00E04FF0B0431868C0F3B5
:10556800404070474FF0B0431868C0F340007047A0
:105578004FF0B042536823F47F4343EA002353605B
:1055880070474FF0B0431868C0F3406070470000A0
:105598007FB54FF0B0432C4AD3F80831C0F303105D
:1055A80003F00F0352F82040284A52F82330B4FB86
:1055B800F3F4FFF785FF264B054693E80700B5F59A
:1055C800007F04AB03E9070010D0224B9C4218D39C
:1055D80003F5B70303F67F539C4229D903F57413E7
:1055E80003F510639C4225D802230BE01A4B9C421A
:1055F80007D91A4B9C421BD903F5370303F5D85337
:10560800F0E7002304AA02EB830353F80C4C144D73
:105618002B6823F0070323432B60FDF757FA064650
:105628002B6803F007039C4206D1002004B070BD2C
:105638000123E7E70024EAE7FDF748FA801B022880
:10564800EED90320F2E700BF8810010828100108EE
:10565800F80E0108C0CF6A00BFEA21013F93340267
:10566800004000584FF0B04310B59A68D96812F05E
:105678000C0205D00C2A4AD101F00303012B50D1AA
:105688004FF0B0412B480B6813F0080306D00B68A5
:1056980013F0080337D1D1F8941007E00C682407F9
:1056A80056BFD1F894300968C3F3032350F8233068
:1056B800002A0CBF184600204FF0B0418A6802F05B
:1056C8000C020C2A1ED1CA6802F00302022A2ED04C
:1056D800032A06D10B68184A13F4801F174B18BF0A
:1056E80013464FF0B042D068D168D268C0F30620A4
:1056F8005843C1F302130133B0FBF3F0530F0133E6
:10570800B0FBF3F010BD0B68C3F30313CEE7042A14
:105718000AD0082A05D11B6813F4801304D107485E
:10572800CAE700231846C7E703480023C4E7024B2B
:10573800D7E700BF881001080024F4000048E801FA
:1057480008B5FFF78FFF4FF0B043044A9B68C3F3D7
:10575800031352F82330B0FBF3F008BD28100108FA
:105768002DE9F0410446002853D04FF0B0439D681E
:10577800DE6803689B0605F00C0506F0030668D58D
:10578800026A1DB10C2D46D1012E44D1002A40D009
:105798004FF0B043A16A1A68170756BFD3F8943080
:1057A8001B681B0903F0F00399421FD90846FFF74D
:1057B800EFFE00282DD14FF0B042136843F00803E4
:1057C80013601368A16A23F0F0030B431360606A47
:1057D800FFF7CEFEFFF7B4FFAB4B1860AB4B186872
:1057E800FDF772F9002834D0BDE8F0814FF0B042DF
:1057F800136843F008031360136823F0F0030B43A6
:105808001360606AFFF7B4FE0846FFF7C1FE002880
:10581800E0D00120E8E74FF0B043002A54D01A68DE
:1058280042F001021A60FDF751F90746FFF79AFEA8
:10583800002842D04FF0B042136843F008031360C9
:105848001368A16A23F0F0030B431360606AFFF743
:105858008FFE2368D80748D42368990700F18C8005
:1058680023681E0740F1FA80A3694FF0B046002B69
:1058780000F0E180D6F89430E16903F0100291421B
:1058880000F0C48003F00302022AC2D0D80740F116
:10589800B380D6F8943023F00103C6F89430FDF7AE
:1058A80015F90746D6F89430990740F1A580FDF719
:1058B8000DF9C31B112BF5D904E0FDF707F9C01B3F
:1058C8000228B3D903208FE71A6822F001021A6070
:1058D800FDF7FCF80746FFF745FE0028B9D0FDF7AD
:1058E800F5F8C01B0228F6D9ECE7082D03D00C2DDB
:1058F80005D1032E03D16368002BADD189E74FF0A2
:10590800B043A1681A6822F480120A431A606268D8
:10591800B2F5803F10D11A6842F480321A60FDF760
:10592800D5F80746FFF718FE002895D1FDF7CEF801
:10593800C01B6428F6D9C5E7B2F5041F04D11A685C
:1059480042F400121A60E6E7196821F48031196000
:10595800196821F400111960002AE0D1FDF7B6F8A2
:105968000746FFF7F9FD00283FF476AFFDF7AEF8DC
:10597800C01B6428F5D9A5E7042D236903D00C2D95
:105988000ED1022E0CD1002B3FF443AF4FF0B042A2
:105998006169536823F0FE4343EA016353605FE79C
:1059A8004FF0B046BBB1336843F480733360FDF702
:1059B8008DF8074633685A0507D57368626923F07E
:1059C800FE4343EA026373604AE7FDF77FF8C31BAF
:1059D800022BEFD976E7336823F480733360FDF741
:1059E80075F8074633685B057FF53AAFFDF76EF843
:1059F800C31B022BF6D965E74FF0B042E169D2F834
:105A0800943023F010030B43C2F894304FF0B047A2
:105A1800D7F8943043F00103C7F89430FDF756F8EF
:105A28000646D7F894309A0718D4FDF74FF8831B29
:105A3800112BF6D946E7D6F8943023F00103C6F8BF
:105A48009430FDF743F80746D6F894309B0705D500
:105A5800FDF73CF8C31B112BF6D933E72368580729
:105A680054D50B4F3B68D90514D4FFF701FDFDF75A
:105A78002DF806463B68DA050CD4FDF727F8831B9A
:105A8800022BF7D91EE700BFB8000020BC00002099
:105A980000040058E3684FF0B046002B58D023F0BC
:105AA8008003052B02BFD6F8903043F00403C6F8F4
:105AB80090304FF0B046FDF709F8D6F8903043F033
:105AC80001030746C6F8903041F28838D6F890307E
:105AD8009B0705D4FCF7FAFFC31B4345F6D9F1E64B
:105AE800E36823F00403812B1BD1FCF7EFFFD6F802
:105AF800903043F08003C6F8903007464FF0B04628
:105B080041F28838D6F89030180504D5E06A0028A4
:105B18004AD1002068E6FCF7D9FFC01B4045F1D9FF
:105B2800D0E6FCF7D3FFD6F8903023F08003C6F810
:105B3800903007464FF0B04641F28838D6F890309A
:105B48001905E3D5FCF7C2FFC01B4045F6D9B9E6F5
:105B5800FCF7BCFFD6F8903023F080030746C6F860
:105B6800903041F28838D6F890301A0516D4FCF7F0
:105B7800ADFFD6F8903023F00103C6F89030074601
:105B88004FF0B04841F28836D8F890309B07BDD521
:105B9800FCF79CFFC31BB342F6D993E6FCF796FFCC
:105BA800C01B4045DFD98DE60C2D4ED04FF0B043D9
:105BB80002281A6822F080721A6033D1FCF786FF37
:105BC8000546FFF7DEFC38BBD4E90C314FF0B04294
:105BD8000B43D0682D4901400B43E16B0B43216C0B
:105BE8000B43616C0B43A16B43EA0123D360136839
:105BF80043F080731360D36843F08053D360FCF79D
:105C080065FF0446FFF7BDFC002882D1FCF75EFF64
:105C1800001B0A28F6D955E6FCF758FF401B0A284E
:105C2800CFD94FE6FCF752FF0446FFF7AAFC30B97C
:105C38004FF0B042164BD1680B40D360D4E5FCF767
:105C480045FF001B0A28F0D93CE601283FF4CCADFB
:105C58004FF0B043226BDB6803F0030191427FF4FD
:105C6800D8AD616B03F070028A427FF4D2ADA16BAC
:105C780003F4FE42B2EB012F7FF4CBAD626C03F06C
:105C8800604393423FF445AFC3E500BF8C80C11128
:105C9800FCFFFEEE2DE9F0410D46044610B9012047
:105CA800BDE8F081684E336803F007038B4216D3D2
:105CB80023689A0727D54FF0B047A268BB6823F03E
:105CC800F0031343BB60FCF701FF0646BB68DB0328
:105CD80019D4FCF7FBFE831B022BF7D911E03368BC
:105CE80023F007030B433360FCF7F0FE07463368E5
:105CF80003F00703AB42DBD0FCF7E8FEC01B022829
:105D0800F5D90320CCE72368580617D54FF0B047DC
:105D18006269D7F8083123F00F0343EA1213C7F872
:105D28000831FCF7D3FE0646D7F80831D90305D465
:105D3800FCF7CCFE831B022BF6D9E2E723685A074F
:105D480013D54FF0B047E268BB6823F4E063134310
:105D5800BB60FCF7BBFE0646BB689B0305D4FCF79B
:105D6800B5FE831B022BF7D9CBE72368180714D598
:105D78004FF0B0472269BB6823F4605343EAC2037B
:105D8800BB60FCF7A3FE0646BB68590305D4FCF7C5
:105D98009DFE831B022BF7D9B3E72368DA070FD4DC
:105DA800294C236803F00703AB4239D8FFF7C8FC36
:105DB800264B1860264BBDE8F0411868FCF784BEF6
:105DC8006268022A1DD1FFF7C7FB00283FF467AFBE
:105DD8004FF0B04641F28838B36823F00303134309
:105DE800B360FCF773FE0746B368626803F00C0300
:105DF800B3EB820FD4D0FCF769FEC01B4045F3D942
:105E08007FE7032A02D1FFF7BCFBDEE712B9FFF7F1
:105E1800A9FBDAE74FF0B0431B685B05D8D43EE72F
:105E2800236823F007032B432360FCF74FFE064645
:105E3800236803F00703AB42B8D0FCF747FE801B8A
:105E48000228F5D95DE700BF00400058B8000020DF
:105E5800BC00002008B5FFF773FC4FF0B043044ABC
:105E68009B68C3F3022352F82330D84008BD00BF13
:105E78006810010808B5FFF763FC4FF0B043044A07
:105E88009B68C3F3C22352F82330D84008BD00BF33
:105E9800681001084FF0B043D3F89000C0F34000F9
:105EA80070474FF0B0410209D1F8883002F47F22E0
:105EB800000123EA020300F47F200343C1F888307D
:105EC80070474FF0B041020CD1F88830120423EA31
:105ED800020343EA0040C1F88800704770B50668BD
:105EE80016F48036044638D0FFF7C2FAFCF7EEFD08
:105EF800614E05463368DB0529D54FF0B043616B29
:105F0800D3F8902002F44072914214D0D3F8901044
:105F1800D3F8902042F48032C3F89020D3F8902030
:105F280021F4407022F480328D07C3F89020C3F822
:105F3800900000F190804FF0B042616BD2F8903041
:105F480023F440730B43C2F89030002605E0FCF7B9
:105F5800BDFD401B0228CDD903262568E8070AD5D0
:105F68004FF0B0416268D1F8883023EA124392B208
:105F78001343C1F88830A9070AD54FF0B041A26889
:105F8800D1F8883023EA124392B21343C1F888301B
:105F9800AA0609D54FF0B0422169D2F8883023F417
:105FA80040630B43C2F88830AB0502D5206AFFF77F
:105FB80088FF680502D5606AFFF783FF290502D5C7
:105FC800A06AFFF77EFF6A0602D56069FFF769FFDE
:105FD8002B0602D5A069FFF764FFE80502D5E06942
:105FE800FFF75FFFE90610D54FF0B042E168D2F83D
:105FF800883023F440730B43C2F88830B1F5807FB2
:1060080002BFD36843F08073D3602A040ED54FF0E3
:10601800B042216BD2F8883023F040430B43C2F8DA
:10602800883019B9D36843F08073D3606B0410D5F6
:106038004FF0B042E16AD2F8883023F040530B4366
:10604800B1F1005FC2F8883003D1D36843F48033DC
:10605800D360304670BDFCF739FD41F288360546FD
:10606800FFF718FF01283FF466AFFCF72FFD401B30
:10607800B042F5D970E700BF0004005830B590F879
:106088002C30012B02464FF0020022D0174B82F829
:106098002D00CA24012582F82C505C6253245C62CE
:1060A800B1F5807F146B996914D121F488519961F5
:1060B800596C24F0010421F0004159641463DD6532
:1060C8000A4BFF2159620020012382F82D3082F803
:1060D8002C0030BD21F408519961D96C24F00204D8
:1060E80021F00041D9641463D865E9E7002800402D
:1060F80070B50B4E036B756D1D40EA07044603D55A
:106108000123F365FCF753FEAB0704D50223F365BF
:10611800204600F0CBF9012384F82D3070BD00BF74
:106128000028004038B50A4CE36823F02003E360F8
:10613800FCF7CCFC0546E3689B0601D5002038BD7A
:10614800FCF7C4FC401BB0F57A7FF4D90320F6E7CE
:10615800002800402DE9F041114DEC6814F040048E
:1061680007461AD1EB6843F08003EB60FCF7AEFCFE
:106178004FF003080646EB685B0601D4032C02D1F6
:106188002046BDE8F081FCF7A1FC801BB0F57A7FC2
:1061980084BF87F82D800324EDE70024F0E700BFD3
:1061A8000028004038B50F4CE36823F08003E36013
:1061B800A3699B06054606D4FFF7B4FF10B1032078
:1061C80085F82D0038BDA36923F02003A361FFF7EC
:1061D800A9FF10B1032085F82D00A36943F020031F
:1061E800A361EFE70028004038B5044600284BD0EB
:1061F80090F82D3003F0FF021BB980F82C20FCF733
:106208006DFA0223214D84F82D30EB68DB0632D479
:10621800CA236B6253236B622046FFF79BFF78BB50
:10622800AB6923F08E6323F04003AB612169636897
:10623800AA690B431343A2691343AB61D4E9022350
:1062480043EA02432B61D4E90931EA680B4322F49B
:10625800F8521343EB602046FFF7A4FF80B9D4E956
:106268000713AA690B4322F0604213436269134380
:10627800AB61FF236B62012384F82D30002002E01C
:10628800024BFF225A6238BD0120FCE7002800407B
:106298000023092803D840EA0310C0B270470A381F
:1062A8000133C0B2F5E700002DE9F04790F82C3033
:1062B800012B05464FF0020069D0012385F82C30E8
:1062C8004E4B85F82D00DE6806F44076B6F5807FE3
:1062D80078D04C69087891F8019091F802A091F86B
:1062E8002470002A55D19B6913F0400308BFCB7076
:1062F800FFF7CEFF80464846FFF7CAFF02465046E2
:10630800FFF7C6FF81463846FFF7C2FF0B6ACF7812
:10631800234343EA875343EA090343EA084343EA2A
:10632800022343EA0063354ACA2050625320506270
:106338008C6A8869B4F5807F946945D124F48854BF
:1063480094610124D465B6F5807F09BFCB691364D5
:106358000343536418BF5064284B4A681A672A6B72
:1063680042F001022A639A6942F488529A61244AE7
:10637800D2F8803043F40033C2F880301F4BFF223C
:106388005A620020012385F82D3085F82C00BDE8DD
:10639800F087B4F1803F07D0B4F5000F04D09B69B3
:1063A80013F0400308BFCB700B6ACA781C4344EA59
:1063B8000A0444EA004343EA092343EA825343EACE
:1063C8000763B0E70023AEE724F40854946102247D
:1063D800D465B6F5807F09BFCB6993640343D36462
:1063E80018BFD064054B4A685A672A6B42F002020C
:1063F8002A639A6942F40852B8E700BF00280040AF
:106408000008005890F82C20012A03464FF002009B
:1064180012D00A4A83F82D00CA21516253215162D1
:10642800916941F020019161FF2151620020012210
:1064380083F82D2083F82C00704700BF0028004007
:1064480090F82C20012A03464FF0020019D00D4A7B
:1064580083F82D00CA2151625321516291690A487B
:1064680041F080019161D0F8801041F48021C0F89A
:106478008010FF2151620020012283F82D2083F82B
:106488002C0070470028004000080058064B5A6D41
:10649800520610B5044603D54022DA65FCF78AFC9B
:1064A800012384F82D3010BD002800407047890072
:1064B80001F1804101F531410A607047890001F11D
:1064C800804101F53141086870470000034AD2F85D
:1064D800903043F40043C2F89030704700040058ED
:1064E800034AD2F8903023F40043C2F89030704742
:1064F80000040058074B1A6822F040021A6040F462
:1065080041704FF4B85218605A601A6842F040025D
:106518001A6070470000015837B5054600284ED06C
:10652800837903F0FF046BB1032C0BD0254B4FF498
:1065380000629A612868FFF7DDFF002401232B71B0
:10654800AC602FE000236B712846FCF7D5F91E4A92
:10655800D2F8903043F48053C2F89030002CE5D143
:1065680002234FF0B042AB71D2F8943023F40043C9
:10657800C2F89430154B1B681C214B43DB0C64217B
:106588004B430193019B93B90124AC60FFF79EFF35
:106598000C4B9A6842F400629A604FF400629A6168
:1065A800002CC7D00123AB71204603B030BD019B3E
:1065B800013B0193D2F894305B04E3D4E6E701246D
:1065C800F2E700BF0004005800080058B800002097
:1065D80037B5174D2B6802461C204343DB0C64205B
:1065E800434314480193019B93B901209060114CD7
:1065F80021732B681C214B43DB0C64214B43019313
:10660800019B6BB9012090600A4BDB6803B030BD79
:10661800019B013B019383689C07E4D50020E6E7D2
:10662800019B013B0193A368DB07E9D5ECE700BFB9
:10663800B80000200000015837B5184D2B680246F5
:106648001C204343DB0C6420434315480193019B02
:10665800A3B901209060124CFF2323732B681C25DB
:106668006B43DB0C64256B430193019B73B90120D9
:1066780090600B4BDB680B7003B030BD019B013B96
:10668800019383689C07E2D50020E4E7019B013B66
:106698000193A368DB07E8D5EBE700BFB80000204B
:1066A800000001580F4B13B51B680F4C18225343B9
:1066B8001B0D64225343014601936269019B02F05A
:1066C800040223B902238B60012002B010BD019B94
:1066D800013B0193606910F00200F6D0002AECD16A
:1066E8001046F2E7B80000200004005807B5037907
:1066F800012B0FD10A4B1B68182253431B0C019323
:10670800FFF7EEFE019B013B0193019B002BF9D1A2
:10671800FFF7DCFE03B05DF804EBFFF7C3BF00BF73
:10672800B8000020F8B51E468379012B15460446AB
:106738000F46DAB22DD14379012B2AD002234271B8
:106748008371FFF7D3FF0D212046FFF7C9FEFFF73E
:106758003FFF390A2046FFF73BFFF9B22046FFF713
:1067680037FF2E44B5420ED12046FFF7AFFEFFF7A4
:1067780099FFA06801230038A3714FF0000318BFE8
:1067880001206371F8BD15F8011B2046FFF720FFB3
:10679800E8E70220F6E7F8B51E468379012B15468F
:1067A80004460F46DAB22FD14379012B2CD042711F
:1067B800FFF79CFF1D212046FFF792FEFFF708FF19
:1067C800390A2046FFF704FFF9B22046FFF700FF19
:1067D80000212046FFF7FCFE2E44B5420ED120468C
:1067E800FFF774FEFFF75EFFA06801230038A3716E
:1067F8004FF0000318BF01206371F8BD29462046F9
:10680800FFF71AFF0135E8E70220F6E7F8B51F465B
:106818008379012B154604460E46DAB22CD143790A
:10682800012B29D04271FFF761FF06F0EF03A3F1B6
:10683800840253425341237131462046FFF750FEEC
:10684800FFF7C6FE2F44AF4210D1FFF73FFE842E5C
:1068580002D02046FFF726FFA06801230038A37165
:106868004FF0000318BF01206371F8BD15F8011B34
:106878002046FFF7ADFEE6E70220F6E7F8B51E462C
:106888008379012B154604460F46DAB227D143799E
:10689800012B24D04271FFF729FF39462046FFF724
:1068A8001FFEFFF795FE00212046FFF791FE2E44BC
:1068B800B5420ED12046FFF709FEFFF7F3FEA068A8
:1068C80001230038A3714FF0000318BF0120637142
:1068D800F8BD29462046FFF7AFFE0135E8E702205C
:1068E800F6E737B50023ADF8043001AA02231221D8
:1068F8000546FFF7C3FFBDF80440022364BA01AAA6
:10690800A4B219462846FFF781FFE20702D52846B8
:1069180009F076FBA30702D5284609F077FB600744
:1069280002D5284609F09CFB210702D5284609F024
:106938009DFBE20602D5284609F09EFBA30602D578
:10694800284609F087FB600602D5284609F064FB53
:10695800210606D514F4807118BF0121284609F0D4
:1069680061FBA20502D5284609F06CFB630402D539
:10697800284609F087FB03B030BDF8B51E46837979
:10698800012B154604460F46DAB227D14379012B6D
:1069980024D04271FFF7AAFE0E212046FFF7A0FD82
:1069A800FFF716FE39462046FFF712FE2E44B54281
:1069B8000ED12046FFF78AFDFFF774FEA068012379
:1069C8000038A3714FF0000318BF01206371F8BDB0
:1069D80015F8011B2046FFF7FBFDE8E70220F6E764
:1069E800F8B51E468379012B154604460F46DAB2E0
:1069F8002BD14379012B28D04271FFF777FE1E2156
:106A08002046FFF76DFDFFF7E3FD39462046FFF707
:106A1800DFFD00212046FFF7DBFD2E44B5420ED1F5
:106A28002046FFF753FDFFF73DFEA068012300381D
:106A3800A3714FF0000318BF01206371F8BD294608
:106A48002046FFF7F9FD0135E8E70220F6E702687E
:106A580052E8003F23F0C00342E8003102680029F1
:106A6800F5D102F1080353E8003F23F4000302F1D3
:106A7800080C4CE800310029F3D12023C0F88830F5
:106A88007047000010B5026852E8003F23F4907385
:106A980042E8003102680029F5D10F4C02F10803E1
:106AA80053E8003F234002F1080C4CE8003100296C
:106AB800F4D1C36E012B07D152E8003F23F0100335
:106AC80042E800310029F7D12023C0F88C30002398
:106AD800C366436710BD00BFFEFFFFEFF8B504466D
:106AE8001346D4F88850202D32D1F1B1EAB1E06FC5
:106AF800A4F85620A4F8542000262122C4F8906057
:106B08002165C4F88820226888B1124FC762124FE5
:106B18000763124F2832C0E90D76FEF7D7F830B177
:106B28001023C4F89030C4F8885001200FE023687F
:106B380040221A62226802F1080353E8003F43F03A
:106B4800800302F1080141E800300028F3D1F8BDC4
:106B58000220FCE7696B0008B16B0008BD6B0008F8
:106B680008B50346806A1B681B6813F0200317D119
:106B7800A0F85630026802F1080353E8003F23F0FA
:106B88008003083242E8003102680029F2D152E855
:106B9800003F43F0400342E800310029F7D108BD27
:106BA800FCF75EFAFBE7704708B5806AFFF7FBFF62
:106BB80008BD7047806A38B50468D0F88830D0F8C6
:106BC8008C50A268120606D5212B04D10023A0F808
:106BD8005630FFF73CFFA3685B0606D5222D04D18B
:106BE8000023A0F85E30FFF74DFFD0F8903043F057
:106BF8001003C0F89030FFF7DCFF38BD08B5806A95
:106C08000023A0F85E30A0F85630FFF7D2FF08BD89
:106C1800704700000368D9691A682DE9F04140F609
:106C28000F0631429D68044610D18E0640F19780C8
:106C380002F0200605F080573E4300F09080436F35
:106C4800002B00F08580BDE8F0411847AB4EAC48FA
:106C58002E401040304300F08280CF0709D5D00580
:106C680007D501201862D4F8900040F00100C4F85C
:106C780090008F0709D5E80707D502201862D4F8D5
:106C8800900040F00400C4F890004F0709D5E807C9
:106C980007D504201862D4F8900040F00200C4F828
:106CA80090000F070BD502F02000304307D00820D2
:106CB8001862D4F8900040F00800C4F890000E055F
:106CC8000AD5500108D54FF400601862D4F8903006
:106CD80043F02003C4F89030D4F89030002B37D01C
:106CE8008B0609D502F0200205F080552A4303D00F
:106CF800636F0BB1204698472668D4F89020B36894
:106D080002F0280203F0400353EA0205204621D08E
:106D1800FFF7B8FEB3685F0617D5226802F10803CB
:106D280053E8003F23F04003083242E800310029CD
:106D3800F3D1D4F8800040B1724B8363FEF73FF87B
:106D480030B1D4F88000836B7DE72046FFF731FF30
:106D5800BDE8F081FFF72DFFC4F89050F8E7E06E2A
:106D6800012840F08980CE0640F18680D00640F1A7
:106D7800838010221A629A6851064BD5D4F8802075
:106D880011684A6892B2002AE2D0B4F85C009042D6
:106D9800DED9A4F85E200A6892062FD453E8002FA3
:106DA80022F4807243E800210029F7D103F1080298
:106DB80052E8002F22F0010203F1080040E8002108
:106DC8000029F3D103F1080252E8002F22F0400213
:106DD80003F1080040E800210029F3D12022C4F87B
:106DE8008C20E16653E8002F22F0100243E80021CE
:106DF8000029F7D1D4F88000FDF7ACFF0223236700
:106E0800B4F85E30B4F85C10C91A89B22046FFF7AE
:106E1800FFFE9DE7B4F85E20B4F85E00B4F85C109D
:106E280080B292B2002893D0891A89B200298FD0F3
:106E380053E8002F22F4907243E800200028F7D18D
:106E4800314D03F1080252E8002F2A4003F10806E9
:106E580046E800200028F4D12022C4F88C2060677E
:106E6800E06653E8002F22F0100243E800200028D3
:106E7800F7D102232367C9E7CF0209D56E0207D5E8
:106E88004FF4801220461A62BDE8F04100F0A0BD20
:106E980008060BD502F0800005F40005284305D04C
:106EA800A36F002B3FF454AF2046CCE64F0611D514
:106EB80056060FD553E8002F22F0400243E8002180
:106EC8000029F7D12023C4F88830A1672046FCF7B1
:106ED800C7F83DE70D0206D5500004D52046BDE8A9
:106EE800F04100F077BDCB017FF532AF002ABFF645
:106EF8002FAF2046BDE8F04100F06BBD0100001047
:106F080020010004056C0008FEFFFFEFD0F88C207C
:106F1800B0F86010222A08B5036855D15B6A826D03
:106F28000B401370836D01338365B0F85E30013B0D
:106F38009BB2A0F85E30B0F85E309BB2002B42D115
:106F4800026852E8003F23F4907342E80031036876
:106F58000029F5D103F1080252E8002F22F00102BE
:106F680003F1080C4CE800210029F3D12022C0F8D5
:106F78008C20184A41679342016705D1C26E012AE5
:106F88000ED0FCF77BF81EE05A681102F6D553E8DC
:106F9800002F22F0806243E800210029F7D1EDE7B5
:106FA8000022C26653E8002F22F0100243E80021B5
:106FB8000029F7D1DA69B0F85C10D20644BF102274
:106FC8001A62FFF725FE08BD9A6942F008029A6125
:106FD800F9E700BF00800040D0F88C20B0F86010BE
:106FE800222A08B5036852D15A6A1140826D22F8E4
:106FF800021B8265B0F85E20013A92B2A0F85E20CA
:10700800B0F85E2092B2002A40D153E8002F22F453
:10701800907243E800210029F7D103F1080252E8F1
:10702800002F22F0010203F1080C4CE8002100298E
:10703800F3D12022C0F88C20174A41679342016798
:1070480005D1C26E012A0ED0FCF718F81EE05A6866
:107058001102F6D553E8002F22F0806243E80021A0
:107068000029F7D1EDE70022C26653E8002F22F08D
:10707800100243E800210029F7D1DA69B0F85C1062
:10708800D20644BF10221A62FFF7C2FD08BD9A69F2
:1070980042F008029A61F9E7008000402DE9F74FB5
:1070A8000368B0F86080DF691A689D68D0F88C10B2
:1070B80001922229044640F0B480B0F86890DFF8C5
:1070C8006CA1DFF86CB10026B9F1000F01D0BB0646
:1070D80021D4B4F85E309BB2D3B1B4F868209A4298
:1070E80016D9226802F1080353E8003F23F08053C1
:1070F800083242E8003122680029F2D14D4B63671B
:1071080052E8003F43F0200342E800310029F7D15C
:1071180003B0BDE8F08F2368A26D5B6A03EA080339
:107128001370A36D0133A365B4F85E30013B9BB2C5
:10713800A4F85E302368DF6978072CD0F9070AD5F0
:10714800019AD20507D501211962D4F8901041F0AF
:107158000101C4F89010B80709D5E90707D502213D
:107168001962D4F8901041F00401C4F890107A071D
:1071780009D5E80707D504211962D4F8903043F0FF
:107188000203C4F89030D4F8903023B12046FFF7BA
:1071980010FDC4F89060B4F85E309BB2002B93D118
:1071A800216851E8003F23F4807341E800302368E8
:1071B8000028F5D103F1080252E8001F01EA0A018C
:1071C80042E800100028F5D120215B45C4F88C1056
:1071D800606720670AD05968090207D553E8001F7D
:1071E80021F0806143E800100028F7D1E16E012901
:1071F80013D1E66653E8001F21F0100143E80010A0
:107208000028F7D1D969CA0644BF1021196220465F
:10721800B4F85C10FFF7FCFC56E72046FBF72EFF9E
:1072280052E79A6942F008029A6171E7FEFFFFEFA0
:1072380000800040156F00082DE9F74F0368B0F88B
:107248006080DF691A689D68D0F88C100192222945
:10725800044640F0B280B0F86890DFF868A1DFF823
:1072680068B10026B9F1000F01D0BB0621D4B4F8EB
:107278005E309BB2D3B1B4F868209A4216D922681E
:1072880002F1080353E8003F23F08053083242E834
:10729800003122680029F2D14C4B636752E8003F65
:1072A80043F0200342E800310029F7D103B0BDE8DC
:1072B800F08F2368A26D596A08EA010122F8021BBF
:1072C800A265B4F85E20013A92B2A4F85E20DF69A4
:1072D80078072CD0F9070AD5019AD20507D50121DC
:1072E8001962D4F8901041F00101C4F89010B80761
:1072F80009D5E90707D502211962D4F8901041F0A1
:107308000401C4F890107A0709D5E80707D50421C5
:107318001962D4F8903043F00203C4F89030D4F8DE
:10732800903023B12046FFF744FCC4F89060B4F8CD
:107338005E309BB2002B95D1216851E8003F23F4C1
:10734800807341E8003023680028F5D103F1080272
:1073580052E8001F01EA0A0142E800100028F5D1AE
:1073680020215B45C4F88C10606720670AD05968F3
:10737800090207D553E8001F21F0806143E8001097
:107388000028F7D1E16E012913D1E66653E8001F02
:1073980021F0100143E800100028F7D1D969CA0686
:1073A80044BF102119622046B4F85C10FFF730FC86
:1073B80058E72046FBF762FE54E79A6942F0080254
:1073C8009A6173E7FEFFFFEF00800040E16F00085D
:1073D80038B5044603682169A2681D68C0690A4374
:1073E80061690A437D49024329400A431A605A6881
:1073F800E16822F440520A435A60794AA1699342EB
:107408001CBF226A11439A6822F06E4222F430624D
:107418000A439A60DA6A616A22F00F020A43DA6262
:10742800704A93421CD14FF0B043D3F8883003F030
:10743800030343F44033A3F54033013B022B00F22E
:10744800C780694A9B5CB0F5004F40F08980082BE3
:1074580024D8DFE803F061C0832380232323650059
:10746800624A934209D14FF0B043614AD3F8883059
:1074780003F00C0343F44023E4E7594A93420DD147
:107488004FF0B043D3F8883003F44063B3F5006F8E
:107498001AD005D853B1B3F5806F12D0012009E096
:1074A800B3F5406FFAD14FF400400EE0FEF7D2FC7E
:1074B80058B900204FF00113A3660023C4E91D3317
:1074C80038BDFEF7CFF8F3E74A4865684A4B626A69
:1074D80005EB450133F81220B0FBF2F39942DDD8F1
:1074E800B3EB053FDAD800231946FAF70DFB09027A
:1074F80041EA10616B080002C0182A464FF00003E9
:1075080041F10001FAF700FB3C4BA0F540729A42AA
:10751800C4D82368D860CCE7FEF79CFC0028C8D004
:107528006168354B626A33F81220B0FBF2F24B08FF
:1075380003EB42034FF6EF72B3FBF1F3A3F1100133
:107548009142ABD823F00F02216892B2C3F34203F1
:107558001343CB60ADE7FEF785F8DFE72548DFE7A3
:10756800082B9BD801A252F823F000BFBD75000874
:10757800C9750008D5750008A5740008CF750008FE
:10758800A5740008A5740008A5740008997500087A
:107598004FF400406368616A174A32F81120B0FB63
:1075A800F2F000EB5300B0FBF3F04FF6EF73A0F1ED
:1075B8001002ACE7FEF74EFC00283FF47AAFE9E78B
:1075C800FEF758FCF8E7FEF74DF8F5E70948E1E75C
:1075D800B0F5004FF4D1FEF74DFC9FE7F369FFCFFC
:1075E8000080004000380140C810010800440040F5
:1075F800CB10F5070024F400D8100108FFFC0F0099
:10760800836ADA0710B506D50168C46A4A6822F4A5
:10761800003222434A609C0706D50168046B4A6819
:1076280022F4803222434A60590706D50168446B28
:107638004A6822F4802222434A601A0706D5016864
:10764800846B4A6822F4004222434A60DC0606D56D
:107658000168C46B8A6822F4805222438A609906C2
:1076680006D50168046C8A6822F4005222438A60B5
:107678005A060FD50168446C4A6822F480122243E6
:10768800B4F5801F4A6005D14A68846C22F4C002B0
:1076980022434A601B0606D50268C16C536823F46E
:1076A80000230B43536010BD2DE9F041DDF818802D
:1076B80004460E4615461F462268D36936EA030378
:1076C8000CBF01230023AB4201D0002027E0B8F112
:1076D800FF3FF2D0FBF7FAF9C01B4045206802D8FB
:1076E800B8F1000F1DD150E8003F23F4D07340E8F3
:1076F8000032002AF7D100F1080353E8003F23F0D5
:10770800010300F1080141E80032002AF3D12023E7
:10771800C4F88830C4F88C3084F884200320BDE88D
:10772800F08103685A07C7D5C3691B05C4D54FF450
:107738000063036250E8003F23F4D07340E800324E
:10774800002AF7D100F1080353E8003F23F00103B2
:1077580000F1080141E80032002AF3D12023C4F8DF
:107768008830C4F88C30C4F89030D5E773B5044637
:107778000026C0F89060FBF7A9F923681B681A0770
:10778800054619D423681B685B070AD56FF07E434A
:10779800009300222B464FF480012046FFF784FF18
:1077A800B0B900202023C4F8883084F88400C4F8D5
:1077B8008C30E06620670CE06FF07E430093324621
:1077C80003464FF400112046FFF76EFF0028D9D07A
:1077D800032002B070BD10B5044650B3D0F888300D
:1077E8001BB980F88430FBF727FB22682423C4F8F0
:1077F8008830136823F0010313602046FFF7E8FD83
:10780800012816D0A36A13B12046FFF7F9FE2368B2
:107818005A6822F490425A609A6822F02A029A60C2
:107828001A6842F0010220461A60BDE81040FFF7CE
:107838009DBF012010BD000030B581658168A0F8AA
:107848005C200023B1F5805FA0F85E20436735D146
:107858000369002B40F2FF1318BFFF23A0F8603024
:107868000023C0F890302223C0F88C30016801F161
:10787800080353E8003F43F00103083141E80034AE
:107888000368002CF2D1456E84680169B5F1005F88
:1078980034D1B0F86850954230D8B4F5805F1DD126
:1078A800254A264C002918BF22464267C1B153E831
:1078B800002F42F4807243E80021F7E729B90369F1
:1078C800002B14BF7F23FF23C8E7B1F1805FC5D128
:1078D8000369002B0CBF7F233F23BFE7174AE4E768
:1078E80003F1080252E8002F42F0805203F1080029
:1078F80040E800210029F3D1002030BDB4F5805FB5
:107908000FD10F4A0F4C002918BF2246426751B1C8
:1079180053E8002F42F4907243E800210029F7D180
:10792800EAE7084AF2E753E8002F42F0200243E86A
:1079380000210029F7D1DFE741720008A57000088F
:10794800E16F0008156F0008D0F88C30202B30B498
:1079580015D1B9B1B2B100230468C3660A4B9C4281
:107968000AD063681B0207D554E8003F43F08063E0
:1079780044E80035002DF7D130BCFFF75DBF022089
:1079880030BC70470120FBE700800040436E30B5F3
:107998002BB90123A0F86A30A0F8683030BD03681D
:1079A800094D9A689968094C490FC2F342626B5CA9
:1079B800615CDB00B3FBF1F3A0F86A30AB5CA25C5E
:1079C800DB00B3FBF2F3E7E7F8100108F010010859
:1079D8007047704770471FB504AB03E9060090F87D
:1079E8008430012B04463AD0012380F884302423C4
:1079F800C0F8883003681A6822F001021A609A6891
:107A080022F440120A439A6071B95A68BDF80C0012
:107A18009DF80E1022F0100202435A605A6822F0B4
:107A28007F4242EA01625A601A6842F001021A6013
:107A3800FBF74CF86FF07E42034600924FF480014A
:107A480000222046FFF730FE38B92023C4F88830DA
:107A5800002384F8843004B010BD0320F8E7022026
:107A6800F9E790F88430012B0FD0012380F8843097
:107A7800016851E8002F42F0020241E80023002B80
:107A8800F6D180F88430184670470220704710B548
:107A980090F88430012B044617D02423C0F888308E
:107AA80003681A68196821F00101196042F0005250
:107AB8004FF0005141661A60FFF768FF2023C0F8B5
:107AC8008830002084F8840010BD0220FCE770B5DF
:107AD80090F88430012B044617D005682423C0F899
:107AE80088302E682B6823F001032B60AB6823F0E5
:107AF80060431943A960FFF749FF20232E60C0F8AF
:107B08008830002084F8840070BD0220FCE770B53E
:107B180090F88430012B044617D005682423C0F858
:107B280088302E682B6823F001032B60AB6823F0A4
:107B380060631943A960FFF729FF20232E60C0F86E
:107B48008830002084F8840070BD0220FCE7000023
:107B580038B5084D052455F8043B2BB9013C14F001
:107B6800FF04F8D1204638BDDB6898470028F5D0D7
:107B7800F9E700BF38080020034BD870034B1B6897
:107B88001B6C03B1184770474C08002034080020CC
:107B9800034B1874034B1B685B6C03B118477047A1
:107BA8004C08002034080020F0B5314D314B95F9D0
:107BB8000420314E91B00C46012795F905108DF837
:107BC800047002288DF809208DF80A1010D18DF85C
:107BD8000800D8711C7202F09FFD337803B114B10C
:107BE80001A803F003FA254B059A1A6011B0F0BDFD
:107BF80059714FF480711A71D9801C7233788DF8DD
:107C0800087053BB1F2306A88DF81C208DF8183068
:107C180002F064FF20238DF8183006A82B798DF820
:107C28001C3002F05BFF22238DF8183006A86B7910
:107C38008DF81C3002F052FF21238DF8183006A869
:107C48006B798DF81C3002F049FF29238DF8183024
:107C580006A80B4B079302F041FF02F05DFD0123DC
:107C680006A88DF818308DF81C3002F037FFB4E7FD
:107C78004C080020C0000020280800202C08002004
:107C8800000400017FB5092301A88DF8043003F032
:107C9800ADF90038044B059A1A6018BF012040421C
:107CA80007B05DF804FB00BF2C08002070B504463F
:107CB8000B46134962784A700020A2780A7208704D
:107CC8001A884A729A788A72DB780B746368CB6078
:107CD8000C4B1B68DA6A2AB1237803F0FB030A2BE2
:107CE80000D09047084E052556F8043B1BB15B6A47
:107CF8000BB120469847013D15F0FF05F4D170BD42
:107D0800CC000020340800203808002070B5044654
:107D180010480123037063784370A3788372E36883
:107D2800C360E378037623694376237943720A4B69
:107D38001B689B6A03B19847084E052556F8043B13
:107D48001BB19B690BB120469847013D15F0FF0513
:107D5800F4D170BDE000002034080020380800206D
:107D6800014B1868704700BF2C08002000B58BB085
:107D7800012368468DF8003002F088FD38B99DF877
:107D88000400003818BF01200BB05DF804FB002088
:107D9800FAE7000008B501F073FE48B9FFF7E6FFFF
:107DA800012806D0054BD879197AFFF7FDFE012086
:107DB80008BDBDE80840FFF7CBBE00BFC0000020EB
:107DC8002DE9F04186B005460E46174601F058FEEB
:107DD80000287FD101F06CFE044640B9FFF7C6FFCA
:107DE800012807D03D4B197AD879FFF7DDFE6FF0EF
:107DF800020462E0DFF8E88088F80860003E18BFF7
:107E080001268DF80460374E687833798DF8123082
:107E1800694602F0D9FC00283ED08DF8044003944E
:107E2800ADF810406FF0060495E803002E4B83E888
:107E38000300337988F80A30394601A803F0DAF9E3
:107E48002A4B059A1A60112841D801A353F820F04B
:107E5800B77E0008DD7E0008D77E0008D77E0008C0
:107E6800D77E0008D77E0008D77E0008F77D000877
:107E7800D77E0008D77E0008D77E0008D17E00088C
:107E8800D77E0008D77E0008DD7E0008DD7E00086A
:107E9800DD7E0008CB7E00082B788DF808306B78E3
:107EA800ADF810306B6803934FF0FF34BCE7104B0C
:107EB80000221A70E31D18BF1446204606B0BDE81C
:107EC800F0816FF00404F8E76FF00504F5E74FF070
:107ED800FF34F2E76FF00104EFE700BFC0000020B5
:107EE800E00000204C080020F00000202C080020B2
:107EF8003008002037B501F0E5FD144D052455F88C
:107F0800043B5BB11B694BB155F8043C9B682BB132
:107F1800984718B155F8043C1B699847013C14F080
:107F2800FF04ECD1FFF714FE68B9094D2B7853B163
:107F3800084BADF80040D978019422466846FFF70F
:107F48003FFF00B92C7003B030BD00BF38080020D7
:107F5800300800204C08002030B58BB0054601F0F1
:107F68008FFD0446002839D1FFF700FF012838D1DA
:107F780068468DF8004002F089FC10B14FF0FF30E0
:107F880004E09DF80430AB4202D100200BB030BDB4
:107F9800012DF3D0022D11D0002DF7D1002BF4D0F4
:107FA80068468DF8045002F099FD0028E6D10E4B82
:107FB8001B681B6B002BE8D09847E6E7002BDDD148
:107FC80068468DF8045002F089FD0028D6D1064B8A
:107FD8001B681B6B002BD8D02846EDE76FF001001B
:107FE800D4E76FF00200D1E73408002010B504464A
:107FF8008AB018B94FF0FF300AB010BD00236846A8
:108008008DF8003002F042FC0028F3D19DF80430CE
:108018002370F1E77FB500220B4620498DF8072031
:1080280001220A7042784A700446002A33D1027944
:108038000A721A884A729A788A72DB780B74036912
:10804800CB60C378164D8DF80830037B8DF8093066
:10805800836803932B68DB6A0BB102A898472B68E7
:108068009B6B13B1227E02B198470E4E052556F838
:10807800043B1BB1DB690BB120469847013D15F065
:10808800FF05F4D10DF10700FFF7B0FF637913B1D5
:10809800054B01221A7004B070BD00BFCC0000204F
:1080A80034080020380800203008002010B50446A5
:1080B8008AB018B94FF0FF300AB010BD20236846C7
:1080C8008DF8003002F0E2FB0028F3D1024A9DF956
:1080D800043023701371EFE74C08002000B58BB013
:1080E8002323019068468DF8003002F0F7FC003831
:1080F80018BF012040420BB05DF804FB70B5654C19
:1081080001468EB01822204606F0ECF8624B002299
:108118001A70FBF759FF23784068012202FA03F12D
:10812800014004D15D4B084608F0D2F8FEE75C49EF
:108138005C481A4602F032F918B14FF0FF300EB021
:1081480070BD272304A88DF8103002F0C7FC564EE6
:10815800564D002870D1012333702B68DB690BB1B1
:1081680000209847272304A88DF8103002F08EFBD2
:10817800059B93F84820227093F8182193F81A3138
:108188006270A370464BD3E9020105F09DFF0546D6
:108198000028D2D1464E062304A88DF8103002F0EC
:1081A80075FB059B736104A802F098FC022304A8E0
:1081B8008DF81030059602F069FB0836032304A8F1
:1081C8008DF81030059602F061FB0F2606F040F896
:1081D800012304A88DF814308DF8106002F07EFC9D
:1081E80010230DEB03008DF810308DF8145002F0B9
:1081F80075FC04238DF8103004A8A3788DF814308A
:1082080002F06CFC3A238DF8103004A863690593DA
:1082180002F064FC02A920788DF8086004F0E4F804
:10822800003818BF0120E0711420FFF757FFE079EC
:1082380003F0A4F9284682E728238DF810302B682C
:108248001B6943B104A802F021FB2B6805981B6940
:1082580040F2C4519847272304A88DF8103002F043
:108268003DFC50B9012304A88DF8103002F00EFB34
:108278009DF81430002B7FF46EAF3378002B7FF419
:108288006CAF052204A88DF81020059302F026FC97
:1082980078E700BF4C0800203008002000110108D2
:1082A800740800208C0800202808002034080020CA
:1082B8001008002037B500230D4601930446D0B9B5
:1082C80000F0A8FB0190019BD3B10F4A42F824307B
:1082D8000E4A9A620E4A1268916B1963916C59633F
:1082E80092690C49D9625A6128465B680A49F222A8
:1082F8009847002006E001A900F092FB0028E2D090
:108308004FF0FF3003B030BD38080020B17B0008C3
:10831800340800208D7C00081C070020194B07B585
:108328001860194B194A1A60194A5A60194A9A6012
:10833800194ADA60194B02681A6042685A60826802
:108348009A60C268DA60164A1A6182695A61154BE6
:10835800C26B5A60144A019119609A601946134A0F
:10836800DA600020FFF7A6FF48B901A800F056FB25
:10837800003818BF0120404203B05DF804FB4FF0FD
:10838800FF30F9E7340800208C080020157D00082C
:108398001D80000835840008B57C0008740800209A
:1083A800A1C3000864080020817B0008997B0008AD
:1083B80051B118B1012804D000207047044B0B605C
:1083C8007047044B0B60F7E74FF0FF30704700BF72
:1083D800000400010100010208B503F0EBF80028D1
:1083E80014BF6FF00100002008BD08B502F0BCF909
:1083F800002814BF6FF00100002008BD10B5044626
:108408008AB018B94FF0FF300AB010BD2123684672
:108418008DF8003002F03AFA0028F3D1024A9DF9AB
:10842800043023705371EFE74C0800202DE9F04128
:108438002E4D2F4F00232B7043786B703B689B6A3F
:108448008AB004460BB128469847DFF8A88005266D
:1084580058F8043B1BB11B6A0BB120469847013EF4
:1084680016F0FF06F4D12378052B2FD00B2B35D02F
:10847800012B25D1204C062368468DF8003002F0E8
:1084880005FA0199E07905F065FE10B91B4B019AD0
:108498005A611B48FFF70AFE1A48FFF7AFFF6B78CF
:1084A8008BB9A371184B5878FFF756FD3B685B6A88
:1084B8000BB1114898476B7813B9E07905F0DAFEEB
:1084C8000AB0BDE8F081FF23A371EFE70F4B01224B
:1084D8005A74227A9A74627ADA74F1E76378002B14
:1084E800EED00AB0BDE8F041FFF7CCBBE0000020B9
:1084F8003408002038080020C000002010080020A0
:10850800C4000020C50000204C080020CC0000203A
:1085180030B58BB0FFF769FF0446F0B903F044FFAC
:10852800831C1DD0F8B9134D2B685B69DBB1272379
:1085380068468DF8003002F0A9F92B6801985B694C
:108548004FF4B961984703F041FF78B92CB9094B4A
:108558001B68DB690BB10120984720460BB030BD82
:108568006FF00704EFE74FF0FF34ECE74FF0FF340C
:10857800F3E700BF34080020014B1878704700BFAC
:10858800A0080020014B5878704700BFA0080020C1
:1085980070470000044B9A7A0AB101225A70034BC3
:1085A8005B6903B118477047A0080020FC00002051
:1085B80073B5224C6378002B33D008F073F96668E2
:1085C8000546FFF7CDFB0644AE4214D2A37A93B119
:1085D800E0228DF800208DF80130217AE3680193BC
:1085E80001226846FFF7ECFB08B1073010D10023E1
:1085F8006370A372656094F83430EBB1002384F89B
:1086080034300F4B5B6BBBB102B0BDE8704018470C
:1086180040F2DC510B4808F011FA0A4808F0D4F986
:10862800E8E794F83520002AE5D094F8360084F875
:108638003530FFF791FCDEE702B070BDA0080020DE
:10864800FC000020D808002037B5104D104CC8B1E8
:10865800C1B10123627200222860E16023700D48D5
:108668000D4B00924FF0FF3108F002F900250B483E
:1086780025822022294605F049FE6570A574A58645
:1086880003B030BD00232B602370EFE79C08002067
:10869800A0080020D80800209D850008B408002004
:1086A8002DE9F0478E4C23788CB0002B56D0C27839
:1086B8000AB9837B13B1238A01332382437B002BBE
:1086C8004CD0E02A4AD10023A372876897F800802B
:1086D800B8F1220F27D8B8F1220F30D8DFE818F008
:1086E8004100FB0052005A0061006E0075008E00C8
:1086F8009D00B400C7002F002F002F002F002F006F
:108708002F002F002F002F002F002F002F002F00E9
:108718002F002F002F002F002F002F002F002F00D9
:10872800C900D000D400B8F17E0F00F0CC80B8F1B9
:108738007F0F00F0DF80B8F17D0F00F0AB80A57AE5
:10874800002D00F05B81674C637A3BB94FF47A7176
:10875800204608F073F9204608F036F90CB0BDE859
:10876800F087E36801220021A2721970A37AE168F8
:108778009818A0720620C854A37AE1689818A072C5
:10878800CA54DCE7584B9B6A002BD8D00121022041
:108798009847D4E77B7884F83630012384F835305D
:1087A800CDE704238DF804307B78003B18BF012304
:1087B80001A88DF8083002F091F9C0E77878003800
:1087C80018BF012002F0DAFEB9E7484E0FCE01AD1E
:1087D8000FC50FCE0FC596E8070085E807007B7820
:1087E8000A2BACD8424A12685268002AA7D00CA9B2
:1087F80001EB830353F82C0C9047A0E77878431ECD
:10880800012B9CD83A4B01381B6818BF01202072F5
:108818009B68002B93D0984791E7E26801230821D1
:10882800A3721170627A057BA17AAA4228BF2A46F0
:10883800934284D285685A1CEB5CE56801334E1C70
:10884800A6726B54D3B2EDE7E3680122A272092243
:108858001A70A37AE268218A581CA072D154A27AAD
:10886800238AE1681B0A501CA0728B5467E7238295
:1088780065E705238DF8043001A802F0B7FB5EE731
:10888800194BDB6A98475AE7194B78781B6860756B
:10889800DB68BEE7037B072B7FF451AF06238DF817
:1088A8000430B7F80130ADF808307B793A791B0409
:1088B80043EA0223FA781343642253430393BB79B0
:1088C8008DF81030D8E73B2201A88DF804208DF8E8
:1088D800083002F003F9012384F834302FE700BF91
:1088E800A0080020D8080020FC000020040F010880
:1088F8009C0800202A2301A88DF8043001F0C6FF47
:1089080094F80A90E6689DF808009DF809509DF8CB
:108918000A709DF80BC09DF80D309DF80E209DF84B
:108928000F109DF80CE009F1010A84F80AA006F876
:108938000980354E94F80A903668D4F80C8009F10D
:10894800010A84F80AA096F803A008F809A094F888
:108958000A90D4F80C8009F1010A84F80AA096F864
:1089680002A008F809A094F80A90D4F80C8009F13C
:10897800010A84F80AA096F801A008F809A094F85A
:108988000A9009F1010A84F80AA096F80080E668BE
:1089980006F8098094F80A80E66808F1010984F865
:1089A8000A9006F808C094F80AC0E6680CF10108B5
:1089B80084F80A8006F80C70A77AE66807F1010CBB
:1089C80084F80AC0F555A57AE6686F1CA772705539
:1089D800A07AE568461CA6722954A17AE0684D1C65
:1089E800A5724254A27AE168501CA0728B54A37AF3
:1089F800E268591CA17202F803E0A0E6034807F0F8
:108A080095FF6570AAE600BF9C080020D8080020E2
:108A18007047000000487047FC00002000207047A5
:108A28004FF0FF3070470000044B054A93F81831A7
:108A3800022B18BF062382F890347047B40E00202A
:108A48007C140020034BD3F8483313B15B6903B19E
:108A5800184770477C140020034A137843F0040336
:108A68001370FFF7EFBF00BF781400201FB50A4B43
:108A78008DF8090093F87C208DF80A2093F88C2053
:108A880093F848000D3202A98DF8082003F0ACFCD9
:108A9800C0B205B05DF804FBB40E002010B5074C59
:108AA80004F5806007F042FF94F81A3413B10123EB
:108AB80084F81934BDE81040FFF7C4BF7C140020C7
:108AC80010B50C4CD4F8403343F08003C4F840335D
:108AD80094F81A3413B10020FFF7E0FF94F89134AA
:108AE80023F0120343F0120384F89134BDE81040D8
:108AF800FFF79ABF7C1400202DE9F041DFF8AC8025
:108B080098F81831022B06460D4602D0284BDB6A2E
:108B1800984702F0E9FD044628B1022002F0DAFD88
:108B2800002002F0DCFD98F81831012B17D102F073
:108B3800DDFD074630B1002002F0CDFD002002F037
:108B4800CFFD3C4602F0D4FD48B1002002F0C4FD40
:108B5800002002F0C6FDBDE8F041FFF765BF002C1C
:108B6800F9D1144C94F8902494F81A34BAB90BB18A
:108B780084F84164304602F065FFD8F82C0007F00D
:108B88009BFED4F8B4339842E5D30B4807F0CEFEE9
:108B980094F8913443F0100384F89134DBE70BB177
:108BA80084F84154284602F04DFFF1E7B40E002046
:108BB800841801087C1400201418002073B5164C82
:108BC800164D04F57A76EB6C95F8502095F97810E7
:108BD80095F84800009603F02DFC95F8303184F89C
:108BE800FC3395F8480040F2012304F22442314650
:108BF800A4F8FA3303F02AFC58B194F8243484F822
:108C08006A34074B00205B6B984794F8FB3384F871
:108C1800903402B070BD00BF7C140020B40E002058
:108C280084180108074A10B5137843F0020313703B
:108C3800FFF708FFBDE81040034B01220021022086
:108C480007F046BB7814002049110108074A10B5FF
:108C5800137843F008031370FFF7F4FEBDE81040E3
:108C6800034B01220021022007F032BB78140020B8
:108C7800591101082DE9F0410F4616461D46804658
:108C880007F010FE0B4A0C4C1378278123F01103D0
:108C980043F011031370C4E9000866812573FFF7D8
:108CA800D1FEBDE8F041054B01220021022007F06A
:108CB8000FBB00BF78140020281A00206911010892
:108CC80013B507F0EFFD0D4B6C461860204607F012
:108CD8003DFD94E803000A4A0A4B83E80300137831
:108CE80043F020031370FFF7ADFE074B012200216C
:108CF800022002B0BDE8104007F0EABA381A002096
:108D080078140020B417002076110108F8B5334D07
:108D180095F81841012C06464BD0022C51D064B965
:108D280038B9D5E91B0105F1740383E8030020462F
:108D3800F8BD01283DD0022801D00324F7E7284FC9
:108D480085F8180107F5747EBEE80F0007F57A7CF0
:108D5800ACE80F009EE8030095F8E9308CE80300C2
:108D680087F8FB63E3B195F80031022B18D1D5F8E9
:108D780004316B67C7F8EC3395F87D3095F8082116
:108D880087F8F83395F88C3085F8782087F8F93328
:108D980097F81B2487F8E82340F20133A7F8FA3341
:108DA800002387F81A340F4BDB6A9847FFF706FF52
:108DB800BDE702F0A4FC04460028B8D185F8186184
:108DC800B5E70028B9D1064B85F81801062283F8C3
:108DD8009024044BDB6A98473446A8E7B40E002079
:108DE8007C140020841801082DE9F04192B0064651
:108DF80002F07AFC002840F05981AD4D95F8183101
:108E0800012B09D02B6BAB4C93B194F80431BBB157
:108E1800042B6FD0032003E002F068FC18B10F2088
:108E280012B0BDE8F08102F063FC0028EAD0F6E752
:108E3800B5F82031D4F81C24013B53432B63E4E7F5
:108E48009D4803F008FA002840F02C8194F80C3172
:108E580023802B6B0C930DF1180895F839308DF899
:108E68003830404695F81C318DF83A3007F094FCBC
:108E7800D5F82831009302AF98E80600D5F82431D8
:108E8800384607F020FC97E803000FAB83E803009F
:108E9800EB6A0D9300238DF844302388ADF84630F3
:108EA80095F8303101228DF839201BB98DF844200E
:108EB8008DF83930814B0093814B95F84800A3F128
:108EC80079020CA903F005FBC0B10B28A8D1D4F88E
:108ED800941499B1002EA3D0D4F84033794843F0C4
:108EE8002003C4F8403307F0A9FD764807F06CFD6D
:108EF800002095E7704803F0E2F9A4E795F8487078
:108F080095F9693095F9392095F87D106E4E3846F7
:108F180003F0ECFA009641B2EB6C95F85020384615
:108F2800183603F087FA0096EB6C95F8502095F9FF
:108F3800701095F8480003F07DFAD4F8C413AB6DAF
:108F4800D4F8DC230B44C4F8B033EB6D1344C4F8F5
:108F5800B43394F80431042B07D02B6E0B44C4F8B7
:108F6800B0336B6E1344C4F8B4330023089395F8F8
:108F7800303183B108A802F095FC00284ED195F94C
:108F8800390094F837629DF82070FFF76FFD3E4472
:108F980080B2B04240D300238DF8133095F83930B1
:108FA8008DF8213095F838308DF82230D5F880309A
:108FB8000993D5F884300A932388ADF82C3095F8B6
:108FC800303194F81B648DF82E3095F848003F4BEB
:108FD8008DF820600DF1130208A903F03FFA012370
:108FE80084F8413495F8393084F842349DF81330C8
:108FF80084F84334D4F81C34C4F85064C4F84834B2
:10900800C4F8583402F076FB50B1D4F81C0402F0CE
:1090180083FB28B1102003E7082001E71320FFE6AF
:1090280095F81831012B01D102F078FB02F065FBAD
:109038000023059394F8043195F9395094F81B648A
:109048009BB1042B7FF4E6AE05A802F067FE58BB7F
:1090580094F8183413B1059B013B0593164B0598FA
:109068003246E9B202F0BCFE02E0134802F090FE7C
:10907800C0B9D4F8403394F80C11218043F00203AE
:10908800C4F8403394F8183411480133DBB284F83B
:10909800183484F845340F4B00259B6AC4F898545B
:1090A800984725E71120BBE61220B9E60E20B7E65F
:1090B800B40E00207C14002084150020E40E00204B
:1090C80010190020E41700203418002098180020F8
:1090D8007E14002084180108F0B5504C504EB4F8A6
:1090E800DC202287D4E92D0194F8B12084F8692086
:1090F80004F16C0282E80300D4E92F0104F1740240
:1091080082E80300B4F8C420A4F87C2091B0D4F815
:10911800CC20D4F8C810C4F884200025D4F8D02076
:10912800C4F888200123A4F82031C4F8801084F8FA
:109138003051A56284F81B5184F83A5084F81D51C7
:1091480084F81E51C4F83451C6F89854A6F8185437
:1091580086F81A54A4F838518DF8183004F50973B4
:10916800039304F50A7394F84800A4F8465104934D
:1091780003A92C4B84F84551C4E94F55059303F0D6
:1091880041F9E36EC6F8D43394F87D3086F8E033BD
:1091980094F88C3086F8E1334FF48073A6F8E23304
:1091A80086F8D05394F8303186F8E43306F57477AE
:1091B8000FCF06F57A740FC497E8030040F2012335
:1091C80084E80300A6F8FA33D6F8483386F81B5427
:1091D800CDE901551BB15A685B6901920293124BA4
:1091E8000793A3F148020892A3F1140209920F4AC7
:1091F8000B9229330A93A2F19C030C93A2F19803D2
:109208000D93131D0E9301A902F14C0307A802F553
:1092180099620F9302F05DFA11B0F0BDB40E002010
:109228007C14002098190020E4180020980F0020D2
:10923800F8B50D4F0D4C0E4E0D4607F077FB3B6B06
:10924800984796F8480004F22442294603F0FEF8AD
:1092580048B194F8243484F86A34706D7B6B98476D
:10926800EB7C84F89034F8BD841801087C14002045
:10927800B40E00200F4890F81B3480F8B8330E4B1A
:1092880093F8692080F8BB2393F87D2080F8C823E1
:1092980093F88C2080F8C92393F8303180F8CC33C8
:1092A8000022A0F8CA2300F56E7100F56070FFF780
:1092B800BFBF00BF7C140020B40E0020114890F8F6
:1092C8009034EBB190F81B3480F8D0330E4BDA6E43
:1092D800C0F8D42393F87D2080F8E02393F88C20FD
:1092E80080F8E12393F8303180F8E4334FF480724A
:1092F800A0F8E22300F5747100F56670FFF798BFD7
:10930800704700BF7C140020B40E002070B5344CA8
:109318002421204604F0FCFF636A984218BF60626B
:109328004FF01C012F4814BF0125002504F0F0FF61
:10933800636C984218BF60644FF480712A4818BF64
:1093480045F0020504F0E4FFD4F84831984218BF0C
:10935800C4F848014FF0D401244818BF45F004056B
:1093680004F0D6FFD4F82032984218BFC4F820027F
:109378004FF000011E4818BF45F0080504F0C8FF6B
:10938800D4F82432984218BFC4F824024FF460710C
:10939800184818BF45F0100504F0BAFFD4F8A835EE
:1093A800984218BFC4F8A8054FF01401124818BF16
:1093B80045F0200504F0ACFFD4F8C03598420F4BB7
:1093C80018BFC4F8C005D3F8483318BF45F04005A6
:1093D8002BB11B691BB12846BDE87040184770BD0A
:1093E800B40E0020DC0E0020FC0E0020001000202F
:1093F800D8100020DC100020601400207C1400200D
:109408002DE9F04F91B04FF00008012B05460F46AB
:1094180002928DF81580ADF8188003D8C84EC14661
:10942800B94502D311B0BDE8F08F15F8090002F074
:1094380077FA4844B842F5DC15F8093009F1010417
:10944800023BE4B2112BEDD801A252F823F000BF81
:10945800A1940008D3940008D3950008FD9500084E
:1094680085960008AD9600081F97000851970008D8
:10947800CD9700082D9400082D9400082B9800081B
:109488002D9400082D940008E99800081199000807
:109498005599000893990008052002F0EDFA90B15B
:1094A8000521002002F0ACFA2A5DA64B09F103045D
:1094B80009F102095FFA89F983F85C2415F8092093
:1094C80083F85D24E4B2A146AAE700238DF816309C
:1094D8008DF817308DF81C308DF82030B8F1000F5A
:1094E8006CD14FF0050896F87C208DF83920631E62
:1094F80096F839208DF83B202B4496F838200D93A8
:109508008DF83C2096F81A3196F868208DF83D20A1
:10951800D6F82C218DF83A300C9273B37B1C1B1BA8
:10952800DBB28DF8383008AB019307AB009396F89F
:1095380048000DF117030DF116020CA902F09AFF6D
:109548008DF8150000F00700072813D196F9392087
:109558009DF9163086F839309A429DF8173086F80A
:109568003830B8BF01229DF81C30B8BF86F81D21DD
:1095780086F868304FF0000909E00523D1E7012299
:109588000DF11501032002F0DBF809F101095FFA7A
:1095980089F29DF82030B3FBF8F19142EFD82344CB
:1095A800DCB2631EDBB29F420DD9EA5C032A9AD073
:1095B800A74288BF1C464FF0010884E709F1050956
:1095C8005FFA89F4F7E71C46F5E72B5D012203F003
:1095D8000F0309F1020986F81B3102FA03F35FFA57
:1095E80089F9A6F82031002206A9042002F0A8F87B
:1095F8004C4668E707238DF815302B5D96F8480030
:10960800C3F3021203F00F038DF8303009F103039E
:10961800DBB28DF83120EA5C09F10403DBB209F111
:109628000504EB5C09F102095FFA89F91B0443EAB6
:10963800022315F809201343642253430CA90D9300
:1096480002F027FF00F00703072BE4B28DF815009E
:109658000CD19DF8303086F8703086F878300D9B44
:10966800F36673679DF8313086F869308DF8180015
:10967800012206A9052002F063F824E7314BD3F84C
:1096880048336BB11B685BB19847029B8DF8180093
:1096980003F03F038DF81930022206A90620EAE7F5
:1096A800FF20F2E703238DF815302B5D8DF8243069
:1096B8000CAB089309F10303DBB209F10604EA5C79
:1096C80096F8480009F10403DBB208A9EB5C1B0417
:1096D80043EA022309F10202D2B209F10509AA5CA0
:1096E8001343642253435FFA89F90C9300230D93C3
:1096F80015F809308DF8383002F0D1FEC3B20028D1
:10970800E4B28DF81530FFF6DEAE8DF81830012280
:1097180006A90720AFE72B5D03F00F03012B4FF4D9
:109728007A7238BF0123534309F10209B365134420
:109738005FFA89F9F365002206A9082056E700BFF9
:10974800B40E00207C1400202B5D96F84800C3F36B
:1097580040128DF81D2007A9C3F3001203F00F0370
:109768008DF81C208DF81E3002F09FFE09F10209C9
:1097780001305FFA89F93FF43BAFBDF81C30914ADC
:10978800A6F87C309DF81E309DF81C40D05CF8F798
:109798003DF90223C6F880000CA996F848008DF818
:1097A80030308DF8324002F01FFE96F939300890BB
:1097B80040B29842B8BF184686F83900002206A978
:1097C800092013E703238DF815302B5D8DF8303011
:1097D80009F10303DBB209F10504EA5C96F84800D5
:1097E80009F10403DBB209F10209EB5C5FFA89F9BC
:1097F8001B0443EA022315F8092013436422534348
:109808000CA90D9302F057FEC3B20028E4B28DF8FC
:109818001530FFF658AE8DF81830012206A90A2037
:1098280029E7092002F028F9DFF89CA1002854D084
:109838000921002002F0E4F80023ADF8263009F1F0
:109848000203DBB24FF47A71EA5C09F10303DBB27D
:109858000DF1300BEB5C1B0443EA02232A5D134332
:1098680009F10402D2B209F1060409F10509AA5C5A
:109878005FFA89F943EA026315F8092003934A431A
:1098880012125846ADF8242006F060FF039B03F13E
:10989800965303F5A91303F5EC530893DAF83C3310
:1098A80000930DF1200999E80600DAF838330AA880
:1098B80006F009FF0B9B00939BE806000A9B4846AD
:1098C80006F0E6FE99E8030006F018FF01F021FF14
:1098D8000123E4B28AF83834F5E58AF83804F2E569
:1098E8000C2002F0C9F800283FF4EDAD0C2100204F
:1098F80002F086F8344B93F89034043B012B7FF642
:10990800E2AD01F002FFDEE509F10203DBB22A5DF8
:10991800E95C09F10303DBB209F10504EB5C09F129
:1099280004095FFA89F91B0415F8090043EA0123C1
:1099380013436421594300F00F0001F0E7FEE4B23D
:109948008DF81800012206A9112094E60D2002F0D6
:1099580093F800283FF4B7AD0D21002002F050F82D
:1099680009F10203DBB2194AE85C2B5D126809F1C0
:10997800040409F103095FFA89F943EA002015F89C
:109988000910E4B201F0C4FE9DE52A5D09F1020365
:1099980009F1040409F10309DBB25FFA89F9E95C0A
:1099A80015F809301B0443EA012313436420584384
:1099B80001F0B0FEE4B28DF81800012206A91320C8
:1099C80059E600BF831101087C140020281A0020E2
:1099D8000E4B93F89124920703D593F88F24012A0C
:1099E80008D90B4991F81A2122B18A6A501C18BF6C
:1099F80001328A620022A3F8182483F81A24D3F8C3
:109A0800402322F00202C3F8402370477C14002050
:109A1800B40E002070B5184C184D04F55A7006F0B5
:109A280085FFD4F84033D4F89804D5F8906023F033
:109A38002003C4F8403338B106F03EFF864203D213
:109A4800002385F83A3070BD0120FFF7CDF90028D2
:109A5800F9D00B28F7D095F8393084F8423409202A
:109A680094F8183484F8453484F8410401F0EAFF86
:109A7800BDE87040FFF7ACBF7C140020B40E002096
:109A8800094BD3F84023012A0AD008490978C907A5
:109A980008D43AB993F89204013818BF01207047E6
:109AA80000207047012070477C14002078140020A3
:109AB800034BD3F84003431E58425841704700BF38
:109AC8007C1400202DE9F04FA9B0EFF3108272B694
:109AD800DFF8F4820021D8F80030C8F8001082F3CB
:109AE8001088BA4C002B00F0E480DAB29B0603928F
:109AF80064D5B74D95F81831022B02D0B54BDB6A07
:109B08009847EFF3108972B6B34F06F0CBFE3E6864
:109B1800D4F8B013361A3144B04806F08FFFAF4876
:109B280006F052FFD4F8B413AD48314406F086FF6E
:109B3800AB4806F049FF89F3108894F81A34002BD3
:109B480000F06D81152312A995F848008DF848306A
:109B580002F04AFCD4F8B4130F900144A14806F06F
:109B68006DFFA04806F030FF3B6894F81B24EB62B9
:109B78000DAF38468DF870201D9306F00DFED5F810
:109B88002831009306AE97E80600D5F82431304610
:109B980006F099FD96E803001FAB83E80300D4F8AC
:109BA8001C341E9395F8303195F84800003B18BFD7
:109BB80001231CA98DF8713002F01FFC039BDF06FE
:109BC8004BD5834DDFF820A2D5F8E420BAF90A3046
:109BD800059298F800200493002363F300020A9387
:109BE80088F8002084F84434049AA4F8223484F8CD
:109BF8002534C4F82834A4F82C3484F82E34C4F856
:109C0800303484F82034C4F8343484F83834C4F850
:109C18003C34704B9AF90C90A4F88C2494F8902456
:109C2800DB6A84F88E9484F88F24DAF80470BAF822
:109C38000860984794F88F3413B9694806F076FE9F
:109C48003146384601F04EFD8346002800F0EA8090
:109C5800049BA4F87E3484F88094039B19071AD5D2
:109C68005B4B93F81831022B02D05A4BDB6A9847AA
:109C78000220FEF7D9FE84F8410401F0E3FE94F8CF
:109C88001A3413B1012384F8193494F8913443F049
:109C9800100384F89134039B5A0703D50621052045
:109CA800FEF72AFF039B9B0703D504210320FEF739
:109CB80023FF01F035FD94F89124D7065FD50023E2
:109CC80084F89234D4F840331E0644BF23F082034C
:109CD800C4F8403312F0050F00F0FC820B2001F0AD
:109CE800CBFE002800F0F68294F89134DD0700F1ED
:109CF800F182580740F10883D4F8403323F0020377
:109D0800C4F84033D4F8402382BB94F8915415F03A
:109D180001011EBF2B4662F3000384F8913494F8C6
:109D280091345E0744BF6FF3820384F891340123B2
:109D380084F8923421B1D4F844332C481B689847EE
:109D48006D070BD52A4801F0A3FE01F0D1FE28B11A
:109D580094F8913443F0040384F8913401F0CEFC74
:109D680094F891346FF3041384F89134012384F840
:109D7800923494F8913443F0200384F8913494F8A1
:109D8800913418070AD56FF3C3031A4984F891343C
:109D9800D4F84433A1F12400DB68984794F891344F
:109DA80099070AD56FF34103124984F89134D4F81E
:109DB8004433A1F16C005B68984794F89034022B07
:109DC8001AD1FEF7FBFE17E0781400207C1400205F
:109DD800B40E002084180108381A0020FC1700204F
:109DE800141800207C180020281A0020BC18002015
:109DF800D01800200819002094F891349A0640F1F0
:109E0800C6826FF3451384F89134D4F84033002B9D
:109E180040F0BD8229B0BDE8F04FFFF777BA84F86B
:109E28004134A1E695F81821012A0CD101F05EFC15
:109E3800804668B1584601F04EFC584601F050FC87
:109E4800042384F88F347EB9012384F8213450E147
:109E580001F04EFC0028F6D0404601F03DFC40469B
:109E680001F03FFC0523ECE73B7804935B09013BD9
:109E7800062B00F21882DFE813F00700160295009F
:109E88001602920016020702102EDDD995F830311D
:109E98001297F6B28DF84C60002BD5D11CA804F0AF
:109EA8004BF912AA1CA9FF2002F0AEF89DF8583011
:109EB800C3F3030307468DF82C3095F8480095F84E
:109EC8007D308DF82D3007220BA902F0A0FA002F63
:109ED8005DD100285BD09DF853309DF8522015992C
:109EE800C5F8E4101B0443EA02239DF85120022020
:109EF8001343C5F8E03004F02DF99DF8583095F873
:109F0800480085F82E71C3F30212C3F3030385F8E2
:109F1800703085F878309DF8593085F86920012B24
:109F280038BF01234FF47A725343AB651344EB6592
:109F38000DF15A034FF001081093113E94F81B34A9
:109F48008DF83C300FA985F868808DF8446002F0E0
:109F580066FA0223404685F8303101F08DFD18B1CC
:109F68004146384601F04CFD94F88F34012B00F23D
:109F7800A88194F81A34002B40F09B8194F891340E
:109F880043F0100384F89134FEF74EFD65E6012096
:109F980001F072FD0028E7D001210720E2E7012344
:109FA80084F8203495F87D308DF82E3094F82434D8
:109FB8008DF82D3095F88C3095F848000D330BA9A5
:109FC8008DF82C3002F010FAA6F10D031BB209909F
:109FD80023EAE37300B283423FF736AF0B2E7FF6D6
:109FE80033AFBB4B25931CA8FF231C978DF87460D7
:109FF8008DF8983002F0D4F8074600287FF424AF93
:10A0080095F81831012B13D101F070FB002873D09B
:10A01800384601F060FB384601F062FB04239DF8E6
:10A028007C101E9884F88F34C1F3001101F077FB7F
:10A038009DF87C301E99C4F8341413F00F0203D035
:10A048009DF89000002863D19DF89800002862D000
:10A05800002A7FF4F9AE9DF89020002A0CBF4FF03B
:10A0680002084FF0030800220A92D5F8EC2091422A
:10A0780054D195F8E910002950D0D5F80C1195F86D
:10A08800EAB009680A9195F81811022902D103214A
:10A0980084F88F14B8F1030F7FF4D6AE13F0600F75
:10A0A8007FF4D2AE0592012795F82E31BBF1000F4F
:10A0B80037D0BBF1010F38D1012B34D16FF009062D
:10A0C80046FA08F606F00106C6F10206F6B2BDF831
:10A0D8007E100AAA304601F02DFE40B307280CBFB7
:10A0E8000823012384F821340A9BC4F83034C4F8C7
:10A0F8006C34FEF7E5FCB0E501F0FAFA002897D0D9
:10A10800384601F0E9FA384601F0EBFA052386E70C
:10A118004FF00008A7E74FF00108A4E74FF0010B44
:10A12800C2E70426D3E70326D1E70123DAE71CAB0D
:10A13800009305990A9B3246584601F0B7FE20B1B4
:10A1480002280CBF0A230B237FE60A9BC4F830348D
:10A15800C4F86C349DF87C3084F82104C3F34013B0
:10A1680084F82E3484F8443494F88F3484F82274B4
:10A17800012B9EBF0122A86285F81E21012FC4F879
:10A18800280484F82C0484F8410438D1022284F885
:10A19800202495F83A20002A4AD19DF87C20D6063A
:10A1A80046D4012B94F840149DF87C2005D8012949
:10A1B80001D1900601D501F05FFBB8F1020F94F8C8
:10A1C8008F3443D0B8F1030F0AD09DF87C10B8F152
:10A1D800010F4A4601F00F0120A83BD0FFF710F904
:10A1E8009DF8903084F82334259BC4F828349DF8D2
:10A1F800983084F82C34012384F82D3430E0049A04
:10A2080002F0E002A02A1BD195F82E11012285F850
:10A218003A2009B927996963012B84F8202407D9C2
:10A22800D5F89020C4F83C24DAF80020C4F8982423
:10A2380095F81821002AB4D1012284F82524B0E722
:10A24800002285F83A2084F82024A6E79DF8981083
:10A2580025984A46FFF7D4F89DF8903084F82334BF
:10A268009DF89020E02A08D195F81F312BB984F881
:10A278002324C4F82834A4F82C3494F8913443F0F7
:10A28800020384F891346FE6114D013EB2B2791C95
:10A29800284604F027F80323A4F82034C4F82854E7
:10A2A80084F82C64E9E7012384F82134FEF708FCDC
:10A2B8005AE694F84434002B3FF460AE0020FEF7D1
:10A2C800EDFB94F88F34022B3FF45EAE56E600BFE8
:10A2D800B416002094F89134590715D5012001F0DF
:10A2E800CBFB60B1012001F09DFB08B984F818048C
:10A2F800D4F8403323F00203C4F8403304E00620C6
:10A3080001F0BAFB0028F3D194F89134DA077FF50D
:10A31800F9AC94F840240AB1032A18D11D4A94F8DC
:10A32800181492F86820914205D29B0723D594F817
:10A338008F34012B1FD8184806F0F8FAD4F84033A8
:10A3480023F02003C4F84033FFF742FBDAE4012A84
:10A3580011D194F81924002A3FF4D4AC0D4A94F88A
:10A36800181492F868209142E5D29F0703D594F813
:10A378004434002BDFD194F8913400206FF3041398
:10A3880084F8913484F81904FFF744FBBAE429B03F
:10A39800BDE8F08FB40E0020E41700202DE9F04F3F
:10A3A80089468DB090460746002800F08F81002925
:10A3B80000F08C810368002B00F088814368002B33
:10A3C80000F084818368002B00F08081C368002B33
:10A3D80000F07C81104602F003F8002800F0788134
:10A3E800BD4CBE4D384601F0C1FA40F2C4520021BE
:10A3F800204603F08BFF40F21C520021284603F050
:10A4080085FFB74BC4F82C3104F50973089304F59C
:10A418000A7300264046099308A9B24B84F848807D
:10A428000A9384F8186184F88C608DF82C6001F028
:10A43800E9FF0F2306A994F848008DF8183001F0B9
:10A44800D3FF801B18BF01204FF00A0B84F81C01B2
:10A4580006A994F848008DF818B001F0C5FF4FF030
:10A46800060A84F8DC0006A994F848008DF818A0BC
:10A4780001F0BAFF102384F8DD0006A994F848001B
:10A488008DF8183001F0B0FF1123C4F89C0006A91C
:10A4980094F848008DF8183001F0A6FF1223C4F88C
:10A4A800A00006A994F848008DF8183001F09CFF28
:10A4B8001323C4F8A40006A994F848008DF81830AE
:10A4C80001F092FF1423C4F8A80006A994F84800E4
:10A4D8008DF8183001F088FF1623C4F8AC0006A9DF
:10A4E80094F848008DF8183001F07EFF172384F89F
:10A4F800B10006A994F848008DF8183001F074FFEF
:10A5080018230DEB0301C4F8B400C4F8BC0094F898
:10A5180048008DF8183001F067FFC0B21D2384F899
:10A52800B80084F8C00006A994F848008DF81830DF
:10A5380001F05AFF1E2384F8C40006A994F84800C5
:10A548008DF8183001F050FF1F2384F8C50006A9C4
:10A5580094F848008DF8183001F046FF2023C4F81D
:10A56800C80006A994F848008DF8183001F03CFF9F
:10A578000B23C4F8CC0006A994F848008DF81830CD
:10A5880001F032FF0C2306A9A4F8D00094F8480083
:10A598008DF8183001F028FFD4F89C306365D4F8A2
:10A5A800A030A365D4F8A430E365D4F8A8302366B6
:10A5B8004FF00108D4F8AC300590A4F8D2006366D7
:10A5C80084F8B080C4F894B084F898A0C4F84CB06B
:10A5D80084F850A084F8688084F81F81C5F84893EF
:10A5E800FEF77AFD404B009632464FF0FF3105F5F5
:10A5F8005A70C5F84473C4E90B6684F8198185F864
:10A608009164C5F8408306F033F9384B009632461A
:10A618004FF0FF3105F5607006F02AF9344B0096CB
:10A6280032464FF0FF3105F5667006F021F902AFAA
:10A63800304B009632464FF0FF3105F5806006F04A
:10A6480017F9384606F0A8F897E8030004F592735E
:10A6580083E80300284B294F1E60294BC5F84C336B
:10A66800284BC5F85433284BC5F85C33274BC5F83D
:10A678005033274BC5F8583305F553703B68984756
:10A6880004F5A67003F084FB20B1112630460DB006
:10A69800BDE8F08F204601F01DFB0028F5D101F040
:10A6A80041F8B8B91B4801F067FB06460028ECD111
:10A6B8007B69984703F0F4FDBB6D94F8190198473E
:10A6C800FB6A9847012385F89234DFE70326DDE724
:10A6D8000926DBE71326D9E7B40E00207C140020F6
:10A6E80000040001981900201D9A00087D920008B6
:10A6F800C5920008A58A000878140020841801086B
:10A70800C98C00087D8C0008618A0008558C0008F7
:10A718002D8C00089C0F002008B5034B0020C3F8BF
:10A728004003FEF781F908BD7C14002010B5FFF73F
:10A73800A7F90A4C60B90A4B93F81831022B02D1D9
:10A74800084BDB6A98470123C4F84033002010BD4A
:10A75800D4F84003013818BF0120F8E77C14002022
:10A76800B40E00208418010838B5134C04F55A704B
:10A7780006F0DCF804F5607006F0D8F804F56670A9
:10A7880006F0D4F804F5806006F0D0F800F0B5FFC4
:10A798000A4B0025DB6A9847C4F84053FEF7B6FD1C
:10A7A8000749084840F2C45203F09CFD0123C4F84D
:10A7B8004033284638BD00BF7C14002084180108A7
:10A7C800B40E0020F008002070B52E4B8AB0054664
:10A7D80093F8DD008DF8090093F8DC008DF80A0085
:10A7E80029489A6A90F81804039200268DF80B00FD
:10A7F80004960C46002940D00692D3F88820079288
:10A808001A8F93F81A118DF8151052BAADF8202046
:10A8180093F87C2093F848308DF8243003AB8DF8FA
:10A8280022008DF8232000930DF10A020DF10B038D
:10A838000DF1090105A88DF8146000F0DDFE9DF901
:10A848000900FEF713F9607004A801F02BF8B0B9FD
:10A85800049A0F2A0DD863789A420AD81544AB4255
:10A86800A3EB02012CBF002001202170C0000AB018
:10A8780070BD002323700820F9E70320F7E71320B1
:10A88800F5E700BFB40E00207C1400201FB5044675
:10A89800002800F012810078412800F20881DFE8E2
:10A8A80010F0420048004D00520056005A005F0068
:10A8B8000601060106010601060106010601060158
:10A8C80066006A006E0079008000830086008B00B5
:10A8D80089008D009100940097009A009D00A000C7
:10A8E800AF00B300BB00B700BF00C200C600CF0076
:10A8F800CB00CD000601D3000601060106010601C2
:10A908000601060106010601060106010601060107
:10A91800060106010601DB00DF00E300E800EC00A9
:10A92800F000F400FD00674B93F81831237104B070
:10A9380010BD644B93F83031237102E0606803F076
:10A94800B5FB0020F3E7606803F0F6FBF9E75D4B21
:10A9580093F81A31F0E75B4BD3F8E0306360F0E727
:10A96800584B211D93F8300103F0FEFBE9E7554BE6
:10A9780093F81931E0E7534B93F88C30DCE71C234C
:10A988008DF808304F4B02A993F8480001F02CFDD0
:10A998006060D6E74C4B043493E8030084E8030076
:10A9A800CFE74A4B0434F7E7494B0434F4E7494B03
:10A9B8000434F1E71A23E3E71923E1E7414B93F85D
:10A9C8006830B9E73F4B5B6DC8E73E4B9B6DC5E709
:10A9D8003C4BDB6DC2E73B4B1B6EBFE7394B5B6EF5
:10A9E800BCE702238DF80830364B02A993F87C2087
:10A9F80093F848008DF80A2001F0F6FC2071A0E7D2
:10AA0800304B93F8DD3097E72E4B93F8393093E7C6
:10AA18002C4B93F8DC308FE72A4B93F838308BE7D0
:10AA2800284BDB6C9AE7274B93F8503084E7254B8B
:10AA3800D3F88430636084E7224B8FE7264B8DE799
:10AA4800204BD3F8CC30F5E71E4BD3F82C3163609C
:10AA580001F058FDA06074E71A4BD3F890307DE7F9
:10AA6800184B93F81F3167E7164BB3F88830A3806B
:10AA780067E7144BB3F88A30F9E7124BB3F8D030D4
:10AA8800F5E7104BB3F8D230F1E70E4B93F84820B6
:10AA98000AB1062A13D1B3F8A035E8E7094B93F8B1
:10AAA80048200AB1062A0AD1D3F8A43556E7204629
:10AAB80004B0BDE8104000F024BE032037E718209A
:10AAC80035E700BFB40E0020200F0020680F0020DB
:10AAD800280F0020700F0020F00800207FB50446E2
:10AAE80010B9032004B070BDA44DD5F840339A07BF
:10AAF80000F171820278412A00F26A82DFE812F0DE
:10AB08004200480056005C00600065006A0077005B
:10AB1800820088008E0094009A00A000A600AC0075
:10AB2800B6006802BB00DD00F000170139012A01F8
:10AB380044014D015101550159015D01680261014E
:10AB480073019B018901AD01B301BA01BF01C401C1
:10AB580068022A02680268026802680268026802DB
:10AB6800680268026802680268026802680268028D
:10AB78006802680236023B02400245024A024F025E
:10AB880054025E020079FEF7C1F80028AAD105E058
:10AB98000379022BA5D07A4A82F8303195F891349E
:10ABA80043F0200385F8913400209BE7406803F0C8
:10ABB8006FFA0028F2D094E7406803F0ADFAF8E79E
:10ABC8006F4B027983F81A21E8E76D4B4268C3F8A6
:10ABD800E020E3E76A4E416896F8300103F0BAFADC
:10ABE80000287FF47EAF6368C6F8E430D6E7416892
:10ABF80000293FF476AF002001F0EAF90028CDD013
:10AC080011206FE7416800293FF46BAF0120F3E79B
:10AC1800416800293FF465AF0820EDE74168002945
:10AC28003FF45FAF0920E7E7416800293FF459AFD7
:10AC38000C20E1E7416800293FF453AF0D20DBE722
:10AC4800416800293FF44DAF0E20D5E7416800293F
:10AC58003FF447AF0F20CFE74A4C494B007983F8C0
:10AC68001901A36D9847E36A984797E7444B02791F
:10AC780083F88C2092E7424E037A8DF8043096F8D8
:10AC8800480096F87D308DF80530072201A901F0BB
:10AC9800BEFB00283FF425AF636896F8480001938F
:10ACA800002201A901F0B3FB00283FF41AAF6C366B
:10ACB800D4E9010186E8030070E7314E037A8DF884
:10ACC800043096F8480096F87D308DF80530072254
:10ACD80001A901F09CFB00283FF403AFB436E7E775
:10ACE800274E037A8DF8043096F8480096F87D30A0
:10ACF8008DF80530072201A901F089FB00283FF4EF
:10AD0800F0AED4E9010106F1740383E8030096F874
:10AD18001831022B7FF442AF96F83031002B3FF404
:10AD28003DAF184BDB6A9847FDF748FF36E7144EEE
:10AD3800037A8DF8043096F8480096F87D308DF83F
:10AD48000530072201A901F062FB00283FF4C9AED3
:10AD5800BC36ADE74368029301238DF80C30084BED
:10AD680002A993F8480001F05FFB00287FF416AFB2
:10AD7800B7E6436802930023EFE700BF7C14002086
:10AD8800B40E00208418010803795A1E0E2A3FF6D3
:10AD9800A8AE934A82F8683000E7914B42685A653A
:10ADA800FCE68F4B42689A65F8E68D4B4268DA6597
:10ADB800F4E68B4B42681A66F0E6894B42685A669D
:10ADC800ECE6874C037994F848008DF804300622A5
:10ADD80001A901F01CFB00283FF483AE9DF8043064
:10ADE80084F8DD30DAE67E4C03798DF8043094F887
:10ADF800480094F87C308DF80630052201A901F04E
:10AE080006FB00283FF46DAE9DF8043084F8393015
:10AE1800C4E6734C037994F848008DF804300A228C
:10AE280001A901F0F4FA00283FF45BAE9DF8043064
:10AE380084F8DC30B2E66A4C037994F848008DF85F
:10AE48000430092201A901F0E2FA00283FF449AED2
:10AE58009DF8043084F83830A0E6614B4268C3F8A6
:10AE68009420DA649AE65E4B027983F8982083F896
:10AE7800502093E65A4B4268C3F884208EE6584B1C
:10AE88004268C3F8CC2089E6012B40F0A480554CD9
:10AE98002421204603F03CFA636A984201D0172027
:10AEA80020E61C2104F1280003F032FA636C984272
:10AEB800F5D14FF4807104F1480003F029FAD4F871
:10AEC80048319842EBD1D42104F5A67003F020FA5A
:10AED800D4F820329842E2D1002104F5097003F039
:10AEE80017FAD4F824329842D9D14FF4607104F596
:10AEF8000A7003F00DFAD4F8A8359842CFD114217E
:10AF080004F2AC5003F004FAD4F8C0359842C6D124
:10AF1800334E2146304640F2C45203F0E3F920464E
:10AF280040F2C452002103F0F1F995F81B3485F87A
:10AF3800E833736FC5F8EC3396F87D3085F8F8334D
:10AF480040F20123A5F8FA33274B96F819019B6DB7
:10AF5800984723E68379012B3FF6C3AD204B42681F
:10AF68004068C3F82C2100F0D1FE47E61C4B42682C
:10AF7800C3F8902012E61A4B027983F81F210DE6D8
:10AF8800174B8288A3F8882008E6154B8288A3F817
:10AF98008A2003E6124B8288A3F8D020FEE5104BE6
:10AFA8008288A3F8D220F9E50D4B93F848200AB11E
:10AFB800062A12D1A288A3F8A025EFE5084B93F83A
:10AFC80048200AB1062A08D16268C3F8A425E5E535
:10AFD80000F099FBD9E5012084E5182082E500BF3F
:10AFE800B40E0020F0080020841801082DE9F04371
:10AFF80087B00023ADF800300646002800F0ED8049
:10B008000361FEF73DFD20B10124204607B0BDE8ED
:10B01800F08300F073FD0028F6D100F069FD0146C9
:10B0280018B96F48142203F071F96E4D95F89134F0
:10B03800012243F0040385F8552485F891343378C8
:10B048008DF804300021013B8DF80520ADF806107D
:10B058000C2B00F2BA80DFE803F007B8B8B87881A3
:10B06800B8B88FB8AC99A800D5F8407317F0200786
:10B07800CAD196F80480B8F1020F45D1DFF868818B
:10B088005A4CFEF729F896F9051098F848003A4600
:10B0980001F017FA88F83900B37988F8383038465B
:10B0A80007238DF80530FDF731FEFF2304F5867080
:10B0B800A5F80C31C5F8084185F8047103F03CF88F
:10B0C80004F58A7002F0F2FF3846FDF78DFE04465B
:10B0D80040B196F9051098F84800012201F0F1F9FD
:10B0E80088F83900D5F894343361002C71D000F019
:10B0F800FFFC002889D195F8913485F81A0460F38B
:10B10800820385F8913480E7B8F1010F4FF002040B
:10B11800E8D1DFF8D4908DF8144099F8480089F800
:10B128001D7102A901F06EF9337989F830318DF873
:10B1380005708DF80680FDF785FC95F8913443F08D
:10B14800100385F891340024CCE7002269460220D8
:10B1580000F0F6FA0028F6D01324C3E7244BB2888F
:10B16800DB6B96F90C10B0689847D5F8403343F07C
:10B178000203C5F84033E6E702A90D2000F060FBA2
:10B188000028E0D0002269460D20E1E7164B93F82D
:10B198001831D3B9347904F0070000F0ADFA8DF80E
:10B1A8000040012269461020D2E700226946122099
:10B1B800CEE78DF8072000F090FA044638B900F081
:10B1C80089FA204600F08BFA8CE702248AE70124EA
:10B1D80088E701A800F0DEFB17E7032415E700BFA6
:10B1E800D01800207C140020B40E00207E1400200B
:10B1F800841801082DE9F04F99B08046059118B9D7
:10B20800032019B0BDE8F08F00230361FEF738FC76
:10B218000646002840F0AB8045460FCD0EAC0FC463
:10B228005A4C98F800A0B8F80C7098F90EB014228F
:10B2380004F58860314603F069F8012284F8412456
:10B24800534C94F83021022A35460BD194F8182132
:10B25800022A07D194F81E2122B9BAF1010F38BF8A
:10B268004FF0010ABAF1010F2DD0BAF1030F2CD01B
:10B27800BAF1000F35D102229DF83C30DDF840903C
:10B28800029362F34715012694F87C108DF832106A
:10B2980002220CA994F848008DF8302001F0A4F897
:10B2A80094F81A3194F830C194F81D1140B2022272
:10B2B800002B6FD0BCF1010F65D1002963D1002E9E
:10B2C8006DD1104627E00422D6E70023DDF83C9034
:10B2D800BDF840709DF942B0029365F01F05012644
:10B2E800D2E74FF0000BD946CDF808B0CCE74FF0C5
:10B2F800010084F81A04DDE005F29A420BA900F077
:10B30800DDFA002800F020811320049B33871F4BAF
:10B31800002283F81A241D4BD3F89434C8F810304F
:10B328006FE705F29A452A460BA900F0C7FA0028EC
:10B33800EAD10B9B84F82801C4F82C5184F83031E9
:10B3480002E1B9F1000F00F0FF80002A00F0FC8054
:10B358004946E01C02F0C6FF94F8373201332380D7
:10B36800F2E01220D1E70220CFE70720CFE7012043
:10B3780047E7064B93F8912483F840A442F0010272
:10B3880083F89124C7E7EEB90220C4E77C140020B3
:10B39800B40E0020002E94D05845B8BF584694F8F3
:10B3A8007C308DF82000052294F848008DF8223072
:10B3B80008A901F02CF800283FF422AF9DF82030AE
:10B3C80084F83930694A6A4BD2F89804D3F8904027
:10B3D80038B105F071FA664B84423CBF002283F80D
:10B3E8003A20198F1A8F93F830010491996A0991BC
:10B3F80052BA0028B9D093F81B0100B9186393F822
:10B408001801ADF85820013893F87C2093F81A41B8
:10B418001491D0F1000BD3F888108DF85B204BEB1A
:10B42800000B93F8482093F83A0093F868308DF8A9
:10B438005A3009AB00934F4B03904FF001008DF841
:10B448004C0015918DF85C20A3F12F01A3F1300277
:10B4580013A88DF84D4000F0CFF8039B4FEA0B1B63
:10B468004BEA431B00264BEA801B4BEAC413B14549
:10B478003E4C039308BF37463A46494604F59C704C
:10B48800CDE90A669B46268084F81A6402F02AFFF2
:10B49800E9B2A570C5F34215FAB2042D344E039BE8
:10B4A80084F837223FF423AF072D3FF44AAF022D2B
:10B4B8007FF459AF304D84F80D110420029984F8B7
:10B4C8000401FF2084F80C0184F8281184F8143151
:10B4D800D6F8E410C4F8085105F59B730AA8C4F817
:10B4E800101184F83021C4F82C3100F017FC002822
:10B4F8007FF437AF0A9BA4F844040BA8A4F81631CC
:10B50800C4F84C3400F0CEF900287FF4FDAE0B9B54
:10B51800D3B196F93900FDF7A9FA94F83732002B20
:10B528003FF4FFAE0B9B0F2B3FF6E6AE05F58B7293
:10B538000BA90F2000F0C2F900287FF4E5AE0B9BA1
:10B5480063F3030B84F814B10598FDF74DFC00284C
:10B558007FF4DBAE099B86F83A00B36200F07EF90F
:10B5680000283FF406AF1320D1E600BF7C1400206A
:10B57800B40E00201C0F00207E14002037B50B4DA0
:10B588008DF8040004460F2295F8480001A900F040
:10B598003EFF40B1064A85F81C4192F8913443F0C9
:10B5A800200382F8913403B030BD00BFB40E0020F0
:10B5B8007C14002010B5FFF7B9F8044688B90A488A
:10B5C80005F0B4F9094805F0B1F9094805F0AEF9F4
:10B5D80000F093F8FDF780FD064BDB6A984720469C
:10B5E80010BD0124FBE700BFE4170020FC17002072
:10B5F80014180020841801082DE9F04F8BB0477803
:10B608000093149B90F90C8090F90D6090F80E90BF
:10B618008B464168196004469246002F57D0022392
:10B628008DF8103004A9C37B007C8DF8123000F02F
:10B63800DBFEB4F808C0618943B2606898454546A6
:10B648006144B8BF1D46604534BF002701278842C2
:10B6580009D30A218DF81010207C019304A900F069
:10B66800C3FE019B46B2B4F808C0608961680CEB60
:10B67800400E714520D3A1EB0C01B1FBF0FC00FB9F
:10B688001C11C9B998450ADC237833B10223207C00
:10B698008DF8243006A900F0B5FE4FF001092123EA
:10B6A8008DF81030207CE37B8DF8115004A98DF8BB
:10B6B800123000F099FE45B2009B8BF800503846D6
:10B6C8008AF8006083F800900BB0BDE8F08F45461B
:10B6D800F2E770477047704770470020704770471F
:10B6E800704770470020704700207047002070475F
:10B6F800002070470020704770477047704702204D
:10B70800704702207047022070477047002070473A
:10B718007047704700207047002070477047704797
:10B728007047000010B5054C4FF403722046002105
:10B7380002F0ECFD0020C4E9000010BD3C1A002016
:10B748002DE9F8438146174600293FD0244B0025B0
:10B7580003F1010C1A462801103312F8018FB8F1D1
:10B76800000F36D19A42F8D11E4E33680BB9C6F88D
:10B7780000C073680BB1C3F800C03318002401354A
:10B788009C6083F80C900D302B01BAB206EB0515BE
:10B798003044F750C6F804C002F0A4FDB9F1110F07
:10B7A8004FF0000398BF104C6B71D6F8083298BF61
:10B7B80024FA09F403F1010398BF04F001043B449F
:10B7C8002C71C6F808324046BDE8F8834FF00108EE
:10B7D800F9E70135202DBBD14FF00208F3E700BF90
:10B7E800431A00203C1A00202007020010B510B3AD
:10B7F800124A1368984204D103681360002304E0D6
:10B808000B4613B119688842FAD15168884208BFBB
:10B8180053600BB101681960D2F808328168013BA6
:10B8280000245B1A04602146C2F80832102202F094
:10B838006DFD204610BD0120FCE700BF3C1A00202A
:10B84800054B1B6813B11A798242FAD1002B0B60A1
:10B858000CBF0320002070473C1A002010B5054B90
:10B86800186800B910BD037B04680BB9FFF7BEFF69
:10B878002046F6E73C1A002038B5084B084C1868F3
:10B8880000B938BD03790568112B05D824FA03F3EC
:10B89800DB0701D5FFF7AAFF2846F1E73C1A00208D
:10B8A8002007020028B1044BD3F8083203600020B7
:10B8B80070470120704700BF3C1A00202DE9F04175
:10B8C80007460E4615463AB331B3144B1C6800239D
:10B8D8002CB93046FFF7E6FF0020BDE8F081A268EA
:10B8E800F91A0132914210D32279EA54581C22895C
:10B8F8005FFA80F8611D55FA80F002F0F3FCA36846
:10B90800246898445FFA88F3E2E720462468FFF742
:10B918006DFF002CF9D1DCE70120DEE73C1A00209E
:10B928000238C0B211289ABF014B185C002070473A
:10B938009311010830B50B4B93F8202004460846B4
:10B9480072B100211C330578A54208D00131984214
:10B95800CDB20CBF04480430AA42F4D8002030BD50
:10B968001046FCE7481C0020541C002010B5084C69
:10B9780000232060142204F10C00FF2184F82030F9
:10B98800C4E9010002F0C2FC012384F8213010BD93
:10B99800481C002010B50E4A92F82010042915D82A
:10B9A800936804781C7044785C70C47880789870C8
:10B9B8000131DC7082F8201002F11C018B4214BFA7
:10B9C800043302F10C039360012010BD0020FCE752
:10B9D800481C0020094B93F8200068B15A6803F10D
:10B9E8001C018A4200F1FF3014BF043203F10C023B
:10B9F80083F820005A600120704700BF481C0020CF
:10BA080010B5074B93F820200446084632B1596810
:10BA1800FFF790FF10B101234470837010BD00BF81
:10BA2800481C002008B5064B93F820202AB1596815
:10BA3800FFF780FF08B1407808BD0120FCE700BF90
:10BA4800481C002030B50A4A92F82010536882F842
:10BA5800210061B1916801241C32DD78587005B964
:10BA68009C7093420CBF034B04339942F5D130BD0F
:10BA7800481C0020541C002008B5044B5968FFF7E7
:10BA880059FF003818BF012008BD00BF481C00201E
:10BA98002DE9F3410422154E044600210DEB020066
:10BAA80096F8208002F032FC0025EBB2984502D8C7
:10BAB80002B0BDE8F0817368197821705A78627015
:10BAC8009F785FB1336820469B689847FFF782FFED
:10BAD80017B901A8FFF75EFF0135E6E7DB788DF8B7
:10BAE80004108DF805208DF80730EFE7481C00207A
:10BAF800014B93F820007047481C0020034B93F833
:10BB08002000042894BF002001207047481C002012
:10BB18001FB50024CDE90244C41F8DF800408DF8FC
:10BB280001100C0AADF80420090C120C8DF8031052
:10BB38008DF806208DF8073002461B0A0121684659
:10BB48008DF802408DF8083002F04BFA002818BF33
:10BB58000E2004B010BD2DE9F04188B017460D46FF
:10BB68000F9A064600284DD000240121CDE904444F
:10BB78008DF810109DF838108DF81510ADF81630A6
:10BB8800190CCDE900441B0ECDE902448DF819309B
:10BB9800ADF81A20130C120E07948DF818108DF8B2
:10BBA8001C308DF81D20E3B24FEA0318002D5FFA10
:10BBB80088F803DC002008B0BDE8F08101331021CB
:10BBC8008DF81F303A466B460DEB010002F09FF9E5
:10BBD8000346C8B9102DAC46A8BF4FF0100CDAB216
:10BBE800624503F1010303DB103D2DB20134DAE7AE
:10BBF80008EB020020326A44315C12F8202C4A40DB
:10BC08003254ECE70920D6E70E20D4E701380328A0
:10BC180015D8DFE800F002080C100A4B1B681B69F6
:10BC28000B6000207047074B1B685B69F8E7054B02
:10BC38001B689B69F4E7034B1B68DB69F0E7052089
:10BC4800704700BF6C1C00202DE9F041C4B00C46C1
:10BC58004A9E17461D468046B8B3B1F5807F36D850
:10BC68004FF488720021684602F050FB4923009384
:10BC78004FF48073ADF804302B0C8DF80830330C7A
:10BC8800ADF80650ADF80A608DF80C302246002356
:10BC9800414604A82D0E360E8DF80E308DF8095049
:10BCA8008DF80D608DF80F4002F01CFB04F11001B7
:10BCB8004B9A3B4689B2684602F013F910B1012845
:10BCC80018BF0E2044B0BDE8F0810920FAE70D2026
:10BCD800F8E7000010B590B10A4C28220021206036
:10BCE80002F014FB2368084A1A6000204FF0FF3264
:10BCF800C3E90302C3E90522C3E9072210BD0820EE
:10BD0800FCE700BF6C1C002000010101024B1B680E
:10BD180018600020704700BF6C1C002030B1044B35
:10BD28001B68DB68013303600020704709207047F7
:10BD38006C1C002013B500230C460193D2B101A955
:10BD4800FFF764FF18B9019B591C02D1146002B0B7
:10BD580010BD99B2611A002902DD0B441360F6E7A1
:10BD680002D113600720F2E71B0C1B0403F5803394
:10BD78002344F3E70920EAE728B1044B1B681C3386
:10BD88004362002070470920704700BF6C1C0020E8
:10BD980013B50446D8B1114B1A68938801339BB286
:10BDA8009380C38200F057FA98B904F118030093FE
:10BDB80021680123132202F08BF860B9204600F0B5
:10BDC8004AFA003818BF0120000102B010BD09204E
:10BDD800FBE71020F9E70E20F7E700BF6C1C0020F6
:10BDE800F0B5054687B01C463BB32F4E3368DB6879
:10BDF800834257D894F82020002A14BF0922082229
:10BE0800834205D3204600F05AFA70B110200AE0A8
:10BE1800002301900093A36894F82810606AFFF744
:10BE28009AFE0028EED007B0F0BD23792168B4F857
:10BE380008C0A768043B9AB209B90920F3E7B2F52C
:10BE4800807F2DD8ADF80EC08DF817304FEA174C0B
:10BE580004F12C033F0E8DF8117000932F0C08236A
:10BE68004FF0490EADF80C008DF814708DF81600DF
:10BE78002F0E0DEB0300CDF808E08DF810C0ADF8DB
:10BE880012508DF8157002F023F808B10E20CAE799
:10BE9800204600F014FA0028B8D13368DD60C2E704
:10BEA8000D20C0E70620BEE76C1C00202DE9FF41ED
:10BEB8000A9D80460F4616461C46002D5AD0002380
:10BEC80003A910460393FFF7A1FE18B1062004B09A
:10BED800BDE8F081039B9C4201D80133F6D1284686
:10BEE80000F05EF9002847D1264B1A78424503D066
:10BEF8001A79424542D10120AA68BA4240D103EBDF
:10BF08008002EB6A92F801802979CDE9004304396F
:10BF1800927828683B4689B2FFF796FE0028D6D16A
:10BF280095F820300194002B4FF00103009314BFC3
:10BF38004246082295F82810686A3B46FFF70BFE30
:10BF48000028C4D1013E032EC1D8DFE806F002075D
:10BF58000B0F0D4B1B681C611C62B8E70A4B1B6872
:10BF68005C61F9E7084B1B689C61F5E7064B1B68A9
:10BF7800DC61ACE70920AAE70F20A8E70B20A6E7B9
:10BF88000220A4E7340100206C1C00201FB50A46DB
:10BF98000B2A4FF00001CDE90011CDE9021107D0BD
:10BFA8000C2A13D00A2A0FD00A2005B05DF804FB2A
:10BFB800012802D120238DF80030684602F011F8DC
:10BFC800002818BF0E20F0E73023F4E70B21F4E730
:10BFD80038B5054602F000F8044678B97DB9094B32
:10BFE8001B680B219878FFF7D1FF38B90C21FFF7B0
:10BFF800CDFF18B90A21FFF7C9FF00B10E2420466A
:10C0080038BD00BF6C1C00202DE9F04380468FB07E
:10C018000C461746002A6BD0002969D0002529460E
:10C028001D2206A8059504F093FE8DF81350344D93
:10C038002B680DF114099E88CDF804900DF11303B7
:10C0480002933B7900933B6832462146404601F013
:10C05800E4FF00284ED138683A79494602F042F99F
:10C06800384600F04FF8002846D13C7AFA79BB7977
:10C07800240444EA02241C432B689A6894423DD95C
:10C088009C609DF813000B21FFF780FF034658BB07
:10C098000C21FFF77BFF034630BB0A21FFF776FF31
:10C0A800034608BB7B7ABA7AFF7A3F0447EA02273D
:10C0B8001F433A46334621460920FFF729FD034628
:10C0C80090B933463A4621460820FFF721FD03463A
:10C0D80050B92A689DF8131091700021D1604FF073
:10C0E800FF31C2E90411916118460FB0BDE8F08331
:10C0F8000923F9E70E23F7E70F23F5E70323F3E70F
:10C108006C1C002010B50446002845D001680029A1
:10C1180042D011F8013B43710322063002F0E2F8E5
:10C128002046032250F8091B043102F0DBF821688D
:10C13800CB79E3600A7A43EA0223E3604A7A43EA66
:10C148000243E3608A7A43EA0263E360CB7A2374AA
:10C158000B7B63742379212B1AD110220D3104F142
:10C16800120002F0BFF81D222168501C8B5C63622C
:10C17800085C43EA0023901C6362085C033243EACC
:10C18800004363628A5C43EA02636362002010BD75
:10C19800112B03DC0D22E7E70220F8E70120F6E780
:10C1A80010B50446002854D00168002951D00B78F6
:10C1B80043714B7883608A7843EA02238360CA78A4
:10C1C80043EA024383600A7943EA026383604B7956
:10C1D80003738B79C381CA7943EA0223027BC38143
:10C1E80002F00F020831103002F07CF8237B0022A5
:10C1F80003F00F0384F8202084F82820227903F123
:10C208000800111A04290DDD21680933043AD21AED
:10C21800085C84F82000D2B2606A84F828201944A7
:10C2280002F060F8237922681A44002012F8043CCE
:10C23800E36212F8031C43EA0123E36212F8021CCA
:10C2480043EA0143E36212F8012C43EA0263E36222
:10C2580010BD0220FCE710B5044660B3036853B371
:10C268000279162A29D942791A700146082251F80A
:10C27800060B013002F040F82146082251F80E0B57
:10C28800093002F039F82368E28A5A74E38A22688E
:10C298001B0A93742368A269DA74A36922681B0ACB
:10C2A80013752368628B5A752368E27E9A75172383
:10C2B8002371002010BD0120FCE70220FAE738B501
:10C2C8000446002863D00168002960D0037B90F8F9
:10C2D800282003F00F03002A57D1083320790432AD
:10C2E8001344984255D363790B702368A2685A7037
:10C2F800A36822681B0A937023686289DA7023682E
:10C30800E27A1A712368227B5A712368E2899A714A
:10C31800E38922681B0A2146D371227B51F8100B4E
:10C3280002F00F02083001F0DDFF237B94F828208B
:10C3380003F00F0303F108052AB1226894F82010CE
:10C34800515503F10905206894F82820616A2844AA
:10C3580001F0C8FF94F828302268E16A2B44D154D0
:10C368005A1CE16A206892B2090A81549A1C216811
:10C37800E08D92B28854DA1C216894F82F0092B2AA
:10C38800043388542371002038BD0933A6E70120FF
:10C39800FAE70220F8E70000024B1A8810431880D9
:10C3A800704700BF701C002008B5074B1B883BB1C5
:10C3B800FEF7BCF900280CBF00206FF0020008BD92
:10C3C8006FF00100FBE700BF701C002010B5034BA5
:10C3D80000241C80FEF7A0F9204610BD701C002028
:10C3E800B0FA80F04009704782B018B9084602B028
:10C3F80000F0CAB8002002B0704710B9084600F033
:10C4080077B9704710B9084600F08EB970470346EF
:10C41800084611460BB900F0E5B90020704710B97D
:10C42800084600F071BD704710B9084600F006BA1A
:10C438000020704710B40446084611461A46019B6E
:10C4480014B910BC00F018BA10BC7047034608466F
:10C4580011460BB900F042BA0020704710B40446E8
:10C46800084611461A4614B910BC00F0AFBA0020AD
:10C4780010BC704730B40546084611461A46DDE937
:10C4880002341DB9029430BC00F02EBB002030BC31
:10C49800704710B9084600F0DFBB0020704710B99C
:10C4A800084600F06FBD0020704710B9084600F03C
:10C4B800EEBB0020704710B9084600F0EBBB002027
:10C4C80070470346084611460BB900F005BC00202A
:10C4D800704710B40446084611461A46019B14B921
:10C4E80010BC00F0FBBB092010BC704710B4044618
:10C4F800084611461A4614B910BC00F063BDC8B20C
:10C5080010BC70470048704701000102064B10B587
:10C518001B6A0446984730B10448054B20449842AA
:10C528008CBF0020012010BD8418010840C220C91A
:10C5380080B92A00F0B5114B85B00C4610491F563A
:10C54800054601F049F80F4BE4B25E6A072D4FF03B
:10C558000103CDE9024301460AD105220023CDE9B2
:10C5680000234FF47A727A431846B04705B0F0BDFD
:10C5780008220020CDE900203A46F5E7CF1101084E
:10C58800A8110108841801081FB500230093037837
:10C59800013B372B21D8DFE803F01C242020201E84
:10C5A800202020204143454E2055585B5E61642081
:10C5B8006C1E6E73787A20207D8126202020202012
:10C5C800202020202020202083858A2020838A2064
:10C5D8008C90C3780BB102230093009805B05DF8E6
:10C5E80004FB8378F6E743788DF8043005238DF84B
:10C5F80005308378003B18BF01235B008DF80630B7
:10C6080010238DF80730304B1B6801A803F55872CA
:10C61800CDE9022300F0C0FF0090DEE74023DBE70E
:10C628002023D9E7827890F9013012B9274AD35CE0
:10C63800D2E7274AFBE7827890F90130002AF8D13F
:10C64800244AF4E740F6B833C6E74FF47A73C3E7F1
:10C658004FF4FA63C0E741F28833BDE741F27073E3
:10C66800BAE71D484FF47A7101F020FE00F5FA6030
:10C67800D2E71A4BB0E7144B1B6803F55873ABE7C6
:10C68800114B1B6803F55B73A6E71023A4E70E4B59
:10C698001B68A1E74FF0834300939EE7104BFBE72D
:10C6A800104B99E740F21113ADF8003095E70323DA
:10C6B80092E790F901300C4AB9E70C4990F901006A
:10C6C80000F08AFFA8E700BF781C00205712010875
:10C6D8005F1201086712010818FCFFFF00EA06371D
:10C6E8009A99094040F70937CF110108A8110108A4
:10C6F80037B50B4B02781B680C2101FB02335B7AC0
:10C7080003EB4304074B1D6803690093C368427831
:10C71800816805EBC40000F0DFFC03B030BD00BF4A
:10C72800781C0020741C002070B586B0027B64233E
:10C73800ADF80030012A4FF00003CDE90133CDE90F
:10C7480003338DF802308DF8143030D0022A39D0F6
:10C758005ABB03684BB343683BB31F4D80682B60DB
:10C768001E4B18226946186001F0BCFD1C4B2C6852
:10C7780093E807000C3384E8070093E8070004F106
:10C788000C06032386E80700A4F86C33012204F59D
:10C798005B7104F5587000F090FC2B684FF6B0728E
:10C7A800A3F878230522C3F87C2306B070BD0A4994
:10C7B80008684360036100F55B7100F5587000F08C
:10C7C8007CFCF2E7044B1B68B3F86023B3F86C13E6
:10C7D8000A43A3F86023E8E7781C0020741C0020B3
:10C7E800300F010808B503460A2924D8DFE801F00C
:10C7F80006232323230B161B23212100BDE8084011
:10C808000068FFF783BE90F900009978052271B996
:10C8180000F013FC003818BF012008BD052293F969
:10C8280000000021F4E790F900005978EEE70221B2
:10C83800EEE70722F3E70020EFE7000010B50479E0
:10C848001CB1012C0BD0002010BD0A4B01681B68DD
:10C85800012203F5587000F030FC0120F4E7054B85
:10C8680001681B68224603F55B7000F026FC204631
:10C87800EAE700BF781C0020F7B50528144D1C46D0
:10C88800A8BF052058700E462946174600F0A4FE9A
:10C8980094F90130A070072B13D1322000F09CFDD1
:10C8A8000C4BDB6D0546984704F10C02083403462F
:10C8B800019200943A463146284600F092FD03B0B2
:10C8C800F0BD054A55F82310D05C00F07DFDE7E780
:10C8D800A811010884180108CF1101082DE9F04FAB
:10C8E800344F90F901607B68D0F804908BB004460F
:10C8F800884698470546002859D1E37C73B92E4AE3
:10C908002378126803EB4303990002EB8303D3F8FF
:10C918000490B9F1000F01D152F80190274B484615
:10C9280013F906B0FB689847A37CD7F818A02289AA
:10C938000993072E28D100230121CDE90223204A9B
:10C948000693CDE90431CDE907330521CDE900216E
:10C958004FF47A7202FB0BF24CF250311846D04772
:10C96800637C13B3174B995D7B6D0D31C9B22846B3
:10C978009847E07C3246494600F040FE88F800605F
:10C9880001200BB0BDE8F08F002101250823CDE977
:10C998000013CDE90715CDE90511CDE90311029280
:10C9A800A1782B465A462846D9E7074BDBE70020F3
:10C9B800E7E700BF84180108781C0020CF110108A0
:10C9C8008545010067120108571201082DE9F04F4B
:10C9D8008DB090F90130DFF8FCA0DFF8FC90CDE9CC
:10C9E8000A123E4A12F903B00278DAF800300C2530
:10C9F80005FB02333A4A5B7A126803EB430302EB06
:10CA0800C303044693F9021090F9020000F0DFFD19
:10CA18003449064694F9010000F0DEFDA268616819
:10CA28008046304600F005FD2178DAF80020D9F874
:10CA38000C306943074650589847D9F81C309C4633
:10CA480094F901300025072B4FF47A63CDE9075399
:10CA5800CDE905552DD10123CDE903530523CDE9B2
:10CA680001534FF47A7303FB0BF3009339464346A3
:10CA780046F2A81228466746B8472378DAF8002015
:10CA88000C214B4394F90110D05800F0D9FDA1892D
:10CA980094F90100FFF74EFD0B9B217B1860D9F834
:10CAA8005430284698470A9B01201E700DB0BDE8F7
:10CAB800F08F01200823CDE90350CDE901032A4670
:10CAC800CDF800B0654643463946A84701200546DB
:10CAD800D3E700BF781C002084180108CF11010893
:10CAE800741C0020A81101082DE9F04F8FB0002414
:10CAF80005468A46914698460494ADF81440ADF828
:10CB0800024007264FF0010B2B7AA34206D968682A
:10CB180004A9204400F0F2FB00285ED102238DF81E
:10CB2800083002A86B7A8DF80A30FFF72DFDAB7A32
:10CB38008DF81D309DF811308DF81E309DF812309B
:10CB48008DF81F309DF810308DF82030EB7A8DF875
:10CB580021302B7B8DF822306B7B8DF8233010230E
:10CB68008DF81C608DF824303A4E8DF82C000DF1AC
:10CB780002030A9305238DF82D3033680C9307239D
:10CB8800ADF834302B6806930DF1120204AB0DF1A9
:10CB9800110106A800F0CCFB072805460BD1306828
:10CBA8000C22002100F5587001F0B0FB3368BDF885
:10CBB8000220A3F860239DF811308AF800309DF810
:10CBC800123089F800309DF8103088F80030189B32
:10CBD80028461C700FB0BDE8F08F9DF81330BDF8E3
:10CBE8001470ADF802702044C4B2F3B917B3194AEF
:10CBF80000201168072602464FF00C0C062B1BD1AB
:10CC08000CFB00FE51F80EE0BEF1000F04D00BFA49
:10CC180000F23A4397B2012201301028EED1002ADF
:10CC28003FF472AFADF802706EE75A1E042A01D9BC
:10CC3800062BDCD0062667E747FA00FE1EF0010F38
:10CC4800EAD00CFB00FE51F80EE0BEF1000F08BF61
:10CC58000626E1E7781C002038B505464068FFF74E
:10CC680055FC0522841D002195F90000E4B200F06E
:10CC7800E4F908B904F0FD0495F901000722002140
:10CC880000F0DBF908B904F0FB04204638BD0020A9
:10CC98007047000010B503780F2B044618D8406879
:10CCA800FFF734FC22780B4902EB42020968831C27
:10CCB80001EB820051F82220DBB21AB903F0FD0320
:10CCC80058B210BD032B06BF626842600223F7E723
:10CCD8000020F6E7781C0020022070472DE9F04F6D
:10CCE800DFF838810446D8F8000099B0894617461D
:10CCF80000211E460122032300F55870CDE90611D4
:10CD0800CDE908118DF814108DF81510ADF816300E
:10CD180000F0B5F938B9D8F80020B2F8603343F01C
:10CD28000303A2F86033D8F80020637A8DF828301E
:10CD380002F55871CDE90B12394A94F90830126896
:10CD48000D920DF116020F922268109262681192EC
:10CD5800D4E90301A27A8DF8482001228DF84920F0
:10CD680013AA82E803001025227DE18A8DF8293074
:10CD780018468DF85420ADF83850FFF7DBFB0AABA6
:10CD880017930DF11503169000933146019705ABE3
:10CD980006AA10A800F0BCFB064698BB9DF8141024
:10CDA800204F013901F082FA1F4B1B690393C4B26B
:10CDB8004FF00C0B04F160036B44D8F8000013F833
:10CDC80048AC9DF814300BFB0AFC01343946B4FB1F
:10CDD800F3F203FB1244D0F87C33B0F9782350F80F
:10CDE8000C00DDF80CC0E4B2E04728B189F800A0D7
:10CDF800304619B0BDE8F08F013D15F0FF05D9D1D7
:10CE08000D26F5E70C2801BFD8F80020B2F86033EA
:10CE180043F00303A2F86033EAE700BF781C002060
:10CE2800741C0020400D030084180108F8B5067929
:10CE3800012E054601D80620F8BD0F2E2BD8036811
:10CE4800187A40F303000522002140B200F0F5F8FB
:10CE58002B680446187A40F303100522002140B2DB
:10CE680000F0EBF8A8B1B4FA84F4640929680B7AE5
:10CE7800086843F3030243F3031352B25BB29A42C6
:10CE8800C8BF0124FFF742FB48B9002CD3D10420C6
:10CE9800D2E70124EAE70320CEE70520CCE7002CFF
:10CEA800FBD10C4F29683B6806EB460003EB80007A
:10CEB8000C2201F017FA3A680C2303FB06232046DC
:10CEC8005C72B2F860130123B3400B43A2F86033DD
:10CED800B2E700BF781C002010B4017801290ED9F0
:10CEE800084B18680C234B43C4180022C250C4E9ED
:10CEF800012200F5587010BC102200F0A7B80020DD
:10CF080010BC7047781C00202DE9F04186B05023F2
:10CF18008DF81430037A102B074630D14368DD7B37
:10CF28006DBB0224A8466426062C14D87A68535D83
:10CF380003932A44517843EA01230393927843EAFE
:10CF480002437343CDE9033863B968468DF800405E
:10CF5800FFF7C2FF0DE0CDF80C808DF81480CDF8F6
:10CF68001080F2E703AB01A801938DF80840FFF7A2
:10CF78005DFF0134E4B2102C05F10305D4D106B0ED
:10CF8800BDE8F0811FB502680379116851B901A89D
:10CF98008DF80430FFF7A0FF78B9002040B205B043
:10CFA8005DF804FB02A802928DF80C30FFF73EFFF3
:10CFB8000628F2D8024B185CF0E70320EEE700BF22
:10CFC800C8110108C90020B9034B0B449856C0B2D8
:10CFD8007047024BF9E700BFD71101081712010883
:10CFE800F0B59A42069D03DB9DF914309A4220DD84
:10CFF8000020F0BD03EB430331F814C005EB8303B5
:10D0080000264CFA06F7FF0707D51F7A07F00F0E20
:10D01800724502DBB2EB171F0DDD0136102E03F14E
:10D028000C03EED10134E4B22301DBB29842E1D81B
:10D03800DEE70024F8E70120DBE7884204DB9042C2
:10D04800CCBF0020012070470020704710B514099C
:10D05800B4EB111F03464FEA11100ED391420CD2C4
:10D0680002B201F00F0133F81240012000FA01F179
:10D0780024EA010123F8121010BD0020FCE7F0B5E6
:10D0880028B100EB410501270020914200D3F0BDF3
:10D09800002435F802CB234607FA04F636EA0C06D4
:10D0A80008BF013304F1010408BFDBB2102CF3D12F
:10D0B80018440131C0B2C9B2E7E710B500B149B9A7
:10D0C80010BD31F8134020F813400133DCB2A242FE
:10D0D800F7D8F5E70023F9E782B030B50488049360
:10D0E8006AB9B3F5616F18D349F6AF2542F21072E9
:10D0F800AB4298BF4FF47A72944238BF1446012C61
:10D1080038BF01246143BDE83040C3688B428CBFFF
:10D118005B1A0023C36002B070476422ECE700008A
:10D128002DE9F04F91B01546DDF86C8004939DF819
:10D13800683009930C46064603F0B4FB684ADFF8EA
:10D14800A4B10590A8F5F633303BB3FBF2F3534393
:10D1580003F5F63203F5A83303F5C07303931823D8
:10D1680013FB054330320692089300254FF0FF3A2F
:10D17800089BA34207D1002D14BF50464FF0FF3043
:10D1880011B0BDE8F08FBDF97030ADF82C300B99B7
:10D19800CDF86C804046CDF8288003F013FBB4F836
:10D1A80000906EB9B8F5616F5BD349F6AF2242F2D1
:10D1B8001073904598BF4FF47A73994538BF9946D4
:10D1C8004B46012B38BF01230793002E52D1B9F1EA
:10D1D800640F48D1A0605F46A1680EA803F014FB55
:10D1E8000F9B0093DDE90A120E9B0CA803F06BFA63
:10D1F800049B0C9A0BB9099B2BB12369BB4202D142
:10D20800394B9A420DD9394BE760984509D9002323
:10D21800ADF83430069B0D990C93184603F0D2FAFA
:10D22800A060606800B9E760276126B103F044FB9D
:10D23800E3680344E360D4E903329342059B1D99F4
:10D248006360079B88BFE2604B43E168994202D262
:10D258000498A8B9A6B101231D442375EDB218346A
:10D2680086E76423A9E7B9F57A7F0ABF204F214FE3
:10D27800A060B1E7049B0BB9C4F80CB05F46D0E7D7
:10D2880000209342207506D85B1A9A4505F10105DE
:10D2980028BF9A46EDB2002EE1D1B9F1640F164AC3
:10D2A800ADF8346019D049F6B023B9F57A7F18BFC4
:10D2B8001346904584BF039A9B180C931C9B0093BC
:10D2C8000CAF97E806001B9B384603F0FCF997E87B
:10D2D800030003F077FA8246C1E74FF46163E8E799
:10D2E8008051010040771B007F5101002FEC0100A5
:10D2F80080A81201002E930230EC01000378032B62
:10D3080014D1437803F00F021B098A704B7083789D
:10D318008B80C27843EA02238B800379C3F302121D
:10D3280003F00F03CA700B70052070470020704788
:10D338002DE9F34798464379057990F907609146B6
:10D34800044690F906208A4683B190F9087075B3AF
:10D358000F2A12D194F909200F2E1ED194F90A60D0
:10D36800072D24D1002F08BF012720E090F90B706A
:10D3780090F9092090F90A60E9E7A369019394F903
:10D3880015300093216994F91430207BFFF728FEAB
:10D398000028E1D105F0FD05DEE794F91D30B34220
:10D3A8000FDC94F91C30B342DADA05F0FB052846A5
:10D3B8008AF8002089F8006088F8007002B0BDE89B
:10D3C800F0871E46CCE70000024B03FA00F0B0FBE2
:10D3D800F1F0704740420F004FF4FA53B3FBF0F0FE
:10D3E800704730B54FF47A750C1F6A4300FB04226E
:10D3F80052001EBF00F1FF341219B2FBF0F2914245
:10D4080038BF1146039A1160820048431CBF01309F
:10D4180040084FF47A71121A01FB1323002BCABF7C
:10D4280003F2E73393FBF1F1B3FBF1F1049B1960CD
:10D4380030BD38B5400014460D46F4F7E7FA01460A
:10D448002846F4F731FA2146F4F72EFAF4F720F9D2
:10D4580003F0C2FCF4F7FCF940B238BD2DE9F74FF0
:10D46800019300231F469C461C01058A5FFA84FE2F
:10D4780004F0F004A54206D8019B82F800C01F7092
:10D4880003B0BDE8F08F0EEB4E054FEA4309AD003F
:10D498000024466836F809602641F60727D58668CD
:10D4A80006EB050A765916B3067836B9466926B1E9
:10D4B80036F809602641F60719D59AF8086090F9F8
:10D4C80001B046F303084FFA88F8D8450FDC46F355
:10D4D800031676B25E450ADB9AF8096006EB460841
:10D4E800C66806EBC806367D4EB90137FFB201346F
:10D4F800102C05F10C05CCD10133DBB2B4E70CF1EB
:10D5080001060EEB040801F80C805FFA86FCEEE7D2
:10D518002DE9FF4704464068DDE90C671D468A4649
:10D52800914603F0C9F923681B1A3B604FF00008C5
:10D538000123337085F80080636813B12368834240
:10D5480024D8CAF80080D4F81CC0A3699CF800E06D
:10D558000393D4E9030101AB83E80300237D00931F
:10D56800DCF80C10237A627A7046FFF7D9FD33464F
:10D5780038602A46E0694946FFF770FF2B782BB1DF
:10D58800C7F80080002004B0BDE8F0873378002B8E
:10D5980014BF0B200C20F6E737B590F9002090F95E
:10D5A8000250954204460FD0013A52B295420BD030
:10D5B800A368019394F9013000936168E0782B46E1
:10D5C800FFF70EFD0028EFD0104603B030BD8842AB
:10D5D800B8BF08467047000051F82000054B984234
:10D5E80005D0054BC31A58425841400070470120E6
:10D5F800704700BF90D0030020A1070005281FB581
:10D608000ED80C4B53F820300093CDE901120A4B89
:10D6180001220021022002F05BFE05B05DF804FB48
:10D62800CDE90012054B01220021022002F050FE34
:10D63800F3E700BFDC1201086F1201088E1201081F
:10D6480007B5054BCDE9000101220021022002F0B7
:10D658003FFE03B05DF804FBAA12010810B51022C2
:10D6680004460021F13000F051FE0021C4F81411E5
:10D678002046F022BDE8104000F048BE02460846A9
:10D68800102100F0A5B92DE9F0430446D0F81401A3
:10D6980085B00E46154604F2011988B3C0F110088A
:10D6A8009045474628BF1746BAB2484400F01AFECC
:10D6B800D4F814313B440F2BC4F814312DD9A845A4
:10D6C8002BD204F1F00304F5807113F8012F187CB4
:10D6D8008B4282EA00021A70F7D104F1F108102295
:10D6E8004146684600F0FEFD22466946684600F05D
:10D6F800E9F910226946404600F0F4FD3E44ED1B6E
:10D7080004F5807804F1F107102D09D8AAB2314642
:10D71800484600F0E7FDC4F8145105B0BDE8F083B1
:10D7280004F1F003711E13F8012F11F8010F43459E
:10D7380082EA00021A70F6D110223946684600F0D3
:10D74800D1FD22466946684600F0BCF910226946B8
:10D75800384600F0C7FD1036103DD5E7F0B589B062
:10D768000C46102200210546684600F0CFFD2246EF
:10D778006946684600F0A6F99DF90030002B6A4614
:10D788004FF0000143DA137812F8010F01315B0002
:10D7980043EAD0130F2902F8013CF4D19DF80F3069
:10D7A8005B0083F08703D4F81401DBB210288DF8EE
:10D7B8000F303BD104F58073694604F5887013F87F
:10D7C800016F11F8012B984282EA06021A70F6D10D
:10D7D80004F1F00304F5807113F8012F187C8B42D3
:10D7E80082EA00021A70F7D110220DEB020004F150
:10D7F800F10100F077FD2246294604A800F062F9FD
:10D8080010220021684600F081FD09B0F0BD1378B0
:10D8180012F8010F01315B0043EAD0130F2902F817
:10D82800013CF4D19DF80F305B00BCE79DF9003056
:10D83800002B6A464FF0000137DA137812F8016FAF
:10D8480001315B0043EAD6130F2902F8013CF4D1F9
:10D858009DF80F305B0083F08703471CDBB28DF81F
:10D868000F30102F04EB0003C0F10F064FF08002B9
:10D8780088BF002600F5817083F801210021324617
:10D8880020443E4403F064FAC4F8146104F580733C
:10D89800694604F5887013F8016F11F8012B984256
:10D8A80082EA06021A70F6D192E7137812F8016F2D
:10D8B80001315B0043EAD6130F2902F8013CF4D189
:10D8C8009DF80F305B00C8E70A780378534003706F
:10D8D8004A784378534043708A78837853408370FA
:10D8E800CA78C3785340C3700A79037953400371E7
:10D8F8004A794379534043718A79837953408371D4
:10D90800CA79C3795340C3710A7A037A53400372C0
:10D918004A7A437A534043728A7A837A53408372AD
:10D92800CA7AC37A5340C3720A7B037B534003739A
:10D938004A7B437B534043738A7B837B5340837387
:10D94800CA7BC37B5340C373704710B50B781478F8
:10D958006340037054784B786340437094788B78B5
:10D9680063408370D478CB786340C37014790B79A3
:10D978006340037154794B796340437194798B798F
:10D9880063408371D479CB796340C371147A0B7A7D
:10D9980063400372547A4B7A634043728B7A947A69
:10D9A80063408372D47ACB7A6340C372147B0B7B57
:10D9B80063400373547B4B7B63404373947B8B7B43
:10D9C80063408373CB7BD27B5340C37310BD00008D
:10D9D800A1F11003DBB2102B2DE9F04704D8374C26
:10D9E80024FA03F3DB0705D4002382F8F030FF2084
:10D9F800BDE8F087531E4418A0424ED101F11C0324
:10DA08009B005FFA83F9C3F30313013B2C4D82F8A3
:10DA1800F03001240B46D618B3FBF1F001FB1030AF
:10DA280010F0FF0016F804AC16F803EC16F802CC58
:10DA380016F8017C36D115F80E8015F80CE015F8AB
:10DA480007C015F80A70E00900EB400084EA0808EE
:10DA580000EBC0006400C0B2E4B24440C246581AA9
:10DA6800C0B212F800808AEA080A02F803A010443B
:10DA7800043390F801808EEA080E86F801E090F8E9
:10DA880002E08CEA0E0C86F802C0C078DBB2474090
:10DA98009945F770BFD80020AAE710F8015B03F892
:10DAA800015FA9E71829DAD9102801BF15F80AA0DB
:10DAB80015F80EE015F80CC0EF5DD0E70101010084
:10DAC800F41401082DE9F04FA3B092F8F0301D913D
:10DAD8001B920193002B00F0538101461EA8FFF70B
:10DAE80034FF1B9BA74CA84DA84E1033029300236C
:10DAF80003939DF87C0004909DF886000590205CB7
:10DB080006909DF87B000790205C089004989DF88B
:10DB180081C0205C099014F80C000A909DF88000E0
:10DB28000B909DF885009DF878809DF87DE09DF824
:10DB380082A09DF887900C909DF87A00029B1C9318
:10DB480014F80A2014F8093014F8081014F80E70A4
:10DB58000D90205C0E909DF87F000F90205C109037
:10DB68000B98205C11900C98205C12909DF8840012
:10DB780013909DF8790014909DF87E001590205C14
:10DB880016909DF883001790205C18901398205CDD
:10DB980019901498205C1A90039801300390029809
:10DBA800DDF804B0103002909DF80C00834536D89B
:10DBB8008DF878108DF87A2009990E9A8DF87C10D6
:10DBC8008DF882201199069A8DF880108DF87E20A4
:10DBD8001999169A8DF884108DF886200A99189A42
:10DBE8008DF87D108DF887201299109A8DF87B306A
:10DBF8001B9B8DF881108DF883201A99089A1D981F
:10DC08008DF885108DF87F201EA903EB0B128DF877
:10DC18007970FFF79AFE002023B0BDE8F08F15F861
:10DC280008B082EA03008BEA000016F80EB080EA1A
:10DC38000B008DF8780015F80E004B40434016F89D
:10DC48000A0043408DF8793081EA070315F80A1075
:10DC5800594016F80930594016F808308DF87A10EE
:10DC68007A40534015F8092053408DF87B30089AC4
:10DC7800069B5340049AAA5C534016F80C20534064
:10DC88008DF87C30DDE908325A4015F80C305340E5
:10DC9800059AB25C53408DF87D30DDE909325A406F
:10DCA800059BEB5C5340079AB25C53408DF87E307D
:10DCB800069B0A9A5340049AB25C5A40079BEB5C55
:10DCC8005A408DF87F200E9B109A53400B9AAA5CFD
:10DCD80053400C9AB25C53408DF88030DDE9103225
:10DCE8005A400C9BEB5C53400D9AB25C53408DF844
:10DCF8008130DDE911325A400D9BEB5C53400F9A9D
:10DD0800B25C53408DF88230129A0E9B53400B9AA6
:10DD1800B25C5A400F9BEB5C1C995A408DF88320EB
:10DD2800169B189A5340139AAA5C5340149AB25CF3
:10DD380053408DF88430DDE918325A40149BEB5C6F
:10DD48005340159AB25C53408DF88530DDE919329D
:10DD58005A40159BEB5C5340179AB25C53408DF8C0
:10DD680086301A9A169B5340139AB25C5340179AFE
:10DD7800AA5C1EA853408DF88730FFF7A5FDB8E6CA
:10DD8800FF2049E7F4140108F4120108F41301080C
:10DD980008B538B1044A05491060D82200F0A2FA43
:10DDA800002008BD0220FCE77C1C0020241A010882
:10DDB8000A4B1A6870B5002302F1180503EB031427
:10DDC8002E5D864204D1183422440A60002070BDBA
:10DDD80001330B2BF2D10320F9E700BF7C1C002094
:10DDE8002DE9F041CCB00646DDF8488117461C46BF
:10DDF8000D4631B3B8F1000F23D006A8FFF72EFC6B
:10DE0800204601A9FFF7D4FF0446B0B9019906A836
:10DE18000131FFF733FC26B11022314606A8FFF77F
:10DE280032FC3A46294606A8FFF72DFC06A902A8A7
:10DE3800FFF794FC029BC8F8003020464CB0BDE8C0
:10DE4800F0810224F9E7000030B595B013A9044623
:10DE5800FFF7AEFF002830D11B490C2303FB00F26B
:10DE6800555CA5422BD1139B187C1090D87B0F9042
:10DE7800987B0E90587B0D90187B0C90D87A0B905D
:10DE8800987A0A90587A0990187A0890D879079061
:10DE9800987906905879059018790490D878039065
:10DEA800987802900A445B78019393680093002263
:10DEB800064B1146022002F00BFA15B030BD0130B6
:10DEC8000B28CBD1F9E700BF6C170108F41501083E
:10DED8000B2B10B402D810BCFFF782BF032010BC74
:10DEE800704730B50D4685B01446014668B103AA9F
:10DEF800002000922A460390FFF772FF18B9039892
:10DF0800001B18BF012005B030BD0220FBE72DE93A
:10DF1800F0430D46BFB014469946804620B31BB364
:10DF280011F00F0122D1F02201A800F0EFF92046EC
:10DF38006946FFF73DFF044648B9009801AA102139
:10DF48000130FFF745FD2E46AF1BFFB21EB9204634
:10DF58003FB0BDE8F08301AA09EB070108EB070011
:10DF6800FFF7B0FD103EEFE70224F0E70524EEE7E7
:10DF7800F0B5184E3468024685B00846002304F10F
:10DF8800180103EB03154F5D97421ED10D2A05F1C9
:10DF9800190513D10023CDE90033CDE902330C2252
:10DFA80010216B46FFF7B3FF04463068102269461C
:10DFB800284400F097F9204605B0F0BD014610222C
:10DFC800601900F08FF90024F5E701330B2BD8D145
:10DFD8000324F0E77C1C002009B1FFF7C9BF022029
:10DFE80070471FB51446A0B10C2A01D10B2912D1D4
:10DFF8000023CDE90033CDE902330A466B461021F0
:10E00800FFF785FF18B969462046FFF7B1FF04B04E
:10E0180010BD0220FBE70320F9E7F8B51E46DDE94D
:10E0280007479DF818505BB354B34FB3212D29D837
:10E0380019462A46204600F055F90122631C691E3C
:10E04800B018FFF764FFF8B9E37ADB093B70EBB966
:10E058006319204613F8012C13F8021C120642EA31
:10E06800014213F8041C0A4313F8031C012342EA73
:10E078000122291FFFF735FF003818BF0120F8BD1E
:10E088000220FCE70520FAE70720F8E70420F6E776
:10E0980008B5014630B1044B0822186800F022F98F
:10E0A800002008BD0220FCE77C1C002008B530B128
:10E0B800044B0822196800F015F9002008BD022059
:10E0C800FCE700BF7C1C00207FB5124E00230446ED
:10E0D80002A801930D46FFF7E9FF33685B690193D6
:10E0E8006CB102AA082312F8011B41B9013B13F0D5
:10E0F800FF03F8D102A8A04702A8FFF7C9FF35B16E
:10E10800019B23B901A8A8473368019A5A610020E6
:10E1180004B070BD7C1C002008B5014638B1054B21
:10E1280018680822104400F0DDF8002008BD02201D
:10E13800FCE700BF7C1C002008B538B1044B196807
:10E148000822114400F0CEF8002008BD0220FCE7A8
:10E158007C1C0020034B1B6802280CBF1961596105
:10E16800002070477C1C002041B1054B1B68022829
:10E178000CBF1B695B690B60002070470220704769
:10E188007C1C002030B58FB0002405460CA80994EB
:10E19800FFF78CFF9DF8373007939DF836300693CC
:10E1A8009DF8353005939DF8343004939DF833304D
:10E1B80003939DF8323002939DF8313001939DF816
:10E1C80030300093224621461E4B022002F080F890
:10E1D8000AA8FFF7B1FF9DF82F3007939DF82E305E
:10E1E80006939DF82D3005939DF82C3004939DF8E7
:10E1F8002B3003939DF82A3002939DF82930019320
:10E208009DF82830009322460F4B2146022002F049
:10E218005FF809A92846FFF7A7FF9DF82430039364
:10E228009DF8253002939DF8263001939DF82730FC
:10E2380000932246054B2146022002F049F80FB010
:10E2480030BD00BF501601088E160108CC16010813
:10E2580008B50020FFF7F8FD0120FFF7F5FD0920BC
:10E26800FFF7F2FD0820FFF7EFFD0020FFF78AFF18
:10E27800002008BD10B504460B20FFF7E5FD0C2073
:10E28800FFF7E2FD0920FFF7DFFD0820FFF7DCFDBF
:10E298000A20FFF7D9FD2046FFF774FF002010BDC4
:10E2A800014B1860704700BF3C0100200B4A30B595
:10E2B80014680B4D43F2390305FB04331360091A44
:10E2C8006FF00042B3FBF2F2C2EBC27201319B1A4B
:10E2D80093FBF1F201FB1233184430BD3C010020DE
:10E2E8006D4EC64101380A44914200D1704711F879
:10E2F800013B00F8013FF7E710440A44914200D17E
:10E30800704711F8013B00F8013DF7E702F020BD26
:10E3180030B530B10A4D01444FF0FF33814201D18D
:10E32800D84330BD10F8012B5340082243F30004B2
:10E33800013A2C4092B284EA5303002AF6D1EDE761
:10E348002083B8ED01207047054B4FF400529A62C4
:10E35800044B1B6813B15B6803B11847704700BFD3
:10E3680000040048801D0020054B4FF480529A623B
:10E37800044B1B6813B1DB6803B11847704700BF33
:10E3880000040048801D00200120704701207047CC
:10E3980001F048B901F036B910B501F019FE0E21A7
:10E3A800044640F61F1001F02DF92046012101F026
:10E3B800F9FDBDE8104001F0D7BA000070B50C4E69
:10E3C80001EB40030D46B3654FF6FF710023044689
:10E3D8001A46084601F05EFB96F85600002101F047
:10E3E800E1FD29462046BDE8704001F095BA00BF1E
:10E3F8009C1D002010B5044601F0AAFE01281CD17E
:10E4080001F0AEFE34B11248214602F017FB104865
:10E4180002F0DAFA0F4C104B00214FF48052A1653C
:10E428009A6194F8560001F0BDFD63786BB16FF006
:10E438007F40BDE8104001F053BA002340F262214A
:10E448001A46084601F026FBDCE7A0688001F0E7E1
:10E45800841D00209C1D002000040048002001F0BD
:10E46800BFB9000008B501F0C7F80438C0B20328E6
:10E4780096BF024B0020185C08BD00BF8018010839
:10E4880008B501F0BAFD033008BD01F049B901F043
:10E4980009B908B501F000FD00B208BD38B50D4650
:10E4A800144601F05DFB284601F092FD0E21054659
:10E4B80040F61F1001F0A6F828460121074D01F08B
:10E4C80071FD01F051FA4FF47A716143284602F068
:10E4D800B5FA2846BDE8384002F076BAF81D0020A3
:10E4E80001F03EBB08B5084B002193F8560001F037
:10E4F80059FD00234FF4C0711A46084601F0CAFAC4
:10E50800BDE8084001F024BA9C1D002010B504465F
:10E5180001F01EFE01281CD101F022FE34B1124880
:10E52800214602F08BFA104802F04EFA0F4C104BBD
:10E5380000214FF48052A1659A6194F8560001F0C9
:10E5480031FD63786BB16FF07F40BDE8104001F09A
:10E558007DB9002340F262211A46084601F09AFA72
:10E56800DCE7A0688001F0E7841D00209C1D0020E6
:10E578000004004808B54FF0040001F017F9BDE8A1
:10E5880008400220F4F7AABA08B500231A4619462B
:10E59800184601F07FFABDE8084001F06DB90000A7
:10E5A8001D4B73B51D4D186000241D486C70C5E9DE
:10E5B8000144AC6501F098FAAC8101F003FA2146F8
:10E5C800204601F04BFC21460422012001F0FCFA10
:10E5D800144E154D4FF6FF7123462246084601F0AA
:10E5E80059FAFFF7C7FF2246104B00944FF0FF314E
:10E5F800304602F03DF90E4B009422464FF0FF31B1
:10E60800284602F035F9304602F090F9284602B063
:10E61800BDE8704002F08AB9801D00209C1D0020D2
:10E62800F1F50008F81D0020841D002051E30008C2
:10E6380071E300080128084805D1084BC177197013
:10E648000E3001F0A7BB437D012B03D1034B81752D
:10E658001970F5E7704700BF9C1D0020400100209D
:10E668000D4B10B5044618735873012000F016F8C6
:10E678005CB134214FF4E86000F0C4FF4421BDE8E8
:10E68800104040F2417000F0BDBF14214FF4E86023
:10E6980000F0B8FF2421F2E79C1D002038B5114C8A
:10E6A8000546207001F061FD052D04D8DFE805F06E
:10E6B800090B03171709032001F070FA002363738D
:10E6C80038BD0020F8E7012001F068FA207B637B61
:10E6D8008342F5D06073BDE83840FFF7C1BF022020
:10E6E800EAE700BF9C1D00202DE9F0431E4687B0D5
:10E6F80000230546CDE901330C46174601F027FDF6
:10E70800032D61D8DFE815F07B00C3000E0104007B
:10E71800A27C082A04D94FF0FF3007B0BDE8F08387
:10E72800A16801A801F0DCFE21680029F3D042F2BB
:10E7380010729142E37C864D51D80322AA7385F862
:10E748003820E96385F844304FF002086368A17DFA
:10E75800DB002B820423AB74A37CDB00EB7402295F
:10E768004FF000032B75637D02D0227D022A42D12F
:10E7780003F10F02D2B2012A01D9012BCBD1754B7B
:10E78800754A196803944FF0010903A88DF814908D
:10E7980001F0DAFC0028BED1287685F81790687554
:10E7A800FFF75CFE4046FFF779FF6C4801F086FAF8
:10E7B8006B4801F0EFFA01A800F084FF208A00F00E
:10E7C80055FFA08900F09AFF384601F001FC604C23
:10E7D80084F8560001F0C0FC666000209DE74FF009
:10E7E8000008E963890885F80E8085F8388085F87F
:10E7F80044302964AAE7EB7529766A75D0E723685F
:10E80800002B88D0A27C082A85D8514DA16801A880
:10E8180001F066FE002385F838302268EA63E27C5E
:10E8280085F84420A269AB732A646268A17DD2008E
:10E838002A820422AA74A27C2B75D2000229637D45
:10E84800EA7402D0227D022A1DD103F10F02D2B24E
:10E85800012A02D9012B7FF45EAF3E4B3E4A19686C
:10E8680003944FF0010803A88DF8148001F06CFCA4
:10E8780000287FF450AF287685F817806875FFF771
:10E88800EDFD00208FE7EB7529766A75F7E7304DC7
:10E89800012185F83810227885F85020637885F8AA
:10E8A8005130A37885F85230E3788B4202D0022B9E
:10E8B80003D03BB985F8533004E00B3A012A29D834
:10E8C80085F853104FF0010885F80E80A388AB83B4
:10E8D800A379AB77E37985F82030237A85F821305E
:10E8E800FFF7BCFD4046FFF7D9FE1C4801F0E6F9EA
:10E8F8001B4801F04FFA95F85130062B40F6890075
:10E908000AD100F08FFE00F0FB0140F6890000F00C
:10E9180079FE59E70023CDE700F084FE40F00401BA
:10E92800C9B2F2E72368013BB3F57A7FBFF4F3AECF
:10E938000320FFF7B3FE0648022380F83830236827
:10E948008364162380F84C30383001F0B7F93BE780
:10E958009C1D0020801D0020F81D0020D41D0020D3
:10E96800AA1D00202DE9F041002686B01F46144656
:10E97800CDE9016680460D4601F0E9FBB442764CCC
:10E9880016BF0123334637466370B8F1000F06D02F
:10E99800B8F1010F7CD0002006B0BDE8F081AB686B
:10E9A800002B00F0D680EB68002B00F0D280AA7F05
:10E9B800082A00F2CE80296901A801F091FD286893
:10E9C800003818BF012000F0D9FF84F83880AB6800
:10E9D800E36395F8203084F84430686801F05AFB06
:10E9E80084F80E8084F84500EB68DB002382EB7F17
:10E9F800A374AB7FDB00E37495F82130237595F899
:10EA08002230002B3ED12A7D95F82410A2750229C8
:10EA180095F8232001D0022B36D102F10F03DBB287
:10EA2800012B02D9012A40F0948000238DF814307C
:10EA38004A4B4B4A1968049503A801F085FB002846
:10EA480040F0878001232076E3756075FFF706FDA7
:10EA58000020FFF723FE434801F030F9424801F057
:10EA680099F901A800F02EFEA88B00F0FFFD288B75
:10EA780000F044FE4FF4FA53AA687B43B3FBF2F369
:10EA8800A36088E7FF22BFE7E27521766375DDE7BB
:10EA98002B8E002B5DD095F83230A86A012B0CBF65
:10EAA80095F814804FF0FF08003818BF012000F0D7
:10EAB80065FFF8B200F06EFF012184F8381095F870
:10EAC8002C2084F8502095F82D3084F8513095F892
:10EAD8002E3084F8523095F82F308B4202D0022B1A
:10EAE80003D03BB984F8533004E00B3A012A28D804
:10EAF80084F853102B8EA38395F83230A377AB8E0E
:10EB080023840126A67384F81F80FFF7A7FC3046EC
:10EB1800FFF7C4FD134801F0D1F8134801F03AF9A2
:10EB280094F82130B34240F236700CD100F07AFDEF
:10EB380000F0FB0140F2367000F064FD4FF6FF7301
:10EB48009EE70023CEE700F06DFD40F00401C9B256
:10EB5800F0E74FF0FF301FE79C1D0020801D0020CC
:10EB6800841D0020D41D0020AA1D00202DE9F04F8F
:10EB780085B082460E9DBDF840B09DF844709DF862
:10EB88004890019288461E4601F0E1FABAF1010F59
:10EB9800524C54D0BAF1040F00F09180BAF1000F32
:10EBA8003AD10B22304684F8442084F838A0E56333
:10EBB80001F070FA019B23644FEACB03B9F1000F0F
:10EBC800238241F60403638214BFF2230123E37511
:10EBD80087F001070123237684F8450084F80EA006
:10EBE80084F814A06775FFF739FC5046FFF756FD07
:10EBF80004F1380001F062F804F10E0001F0CAF8DF
:10EC0800374A1068516802AB03C302A800F05AFDE6
:10EC180040F2FF1000F02AFD404601F0D9F90E211C
:10EC280084F8560040F61F1000F0ECFC94F85600EB
:10EC380001F092FA169B636005B0BDE8F08F294990
:10EC480084F838A0EAB2895D84F8502076BB0B3D81
:10EC5800012D8CBF00250125053A012A04D8BBF1F6
:10EC68000C0F38BF4FF00C0B1F4B9DF83C201B7846
:10EC780084F85350E37701259DF8543084F85110F7
:10EC880084F8522084F82130A573A4F81CB0A77723
:10EC980084F82090FFF7E2FB2846FFF7FFFC1348B3
:10ECA80001F00CF8124801F075F8B5E7012E04D10F
:10ECB800A5F10C035D425D41CEE70025CCE7504647
:10ECC800FFF7ECFC022384F8383004F138001623EF
:10ECD800A56484F84C3000F0F1FF9DE79C1D0020EE
:10ECE800480F01084E18010840010020D41D0020DB
:10ECF800AA1D00202DE9F04F87B0DFF8B4B29DF8C7
:10ED080064A09DF84C90029314469DF854309DF8E9
:10ED18005020BDF84880039205468BF801A0BDF845
:10ED2800446001930F4601F012FABAF1000F18BFC0
:10ED38004FF00008DFF87CA2039AB9F1000F08BF72
:10ED4800FF22012D8AF8002000F0C880052D48D048
:10ED5800002D40F0C080284600F010FE0B223846F7
:10ED68008BF844208BF83850CBF83C4001F092F9EE
:10ED7800019B8BF8450041F60402002BABF81220EA
:10ED88009AF800208BF8162014BFF22201228BF883
:10ED98001720F600012289F001098BF818208BF85A
:10EDA8000E50ABF810608BF814508BF81590FFF7E5
:10EDB80055FB2846FFF772FC0BF1380000F07EFF88
:10EDC8000BF10E0000F0E6FF7B490868496804AAC9
:10EDD80003C204A800F076FC40F2FF1000F046FCE5
:10EDE80071E0012000F0CAFD09224FF000098BF8FC
:10EDF800442038464FF44872CBF840208BF83890BE
:10EE0800CBF83C4001F046F94FF48052ABF81220A1
:10EE18009AF800208BF845008BF816202846012226
:10EE2800F6008BF817208BF80E90ABF81060ABF853
:10EE380014908BF81890FFF731FC0BF1380000F0B4
:10EE48003DFF0BF10E0000F0A5FF5B498868C9681B
:10EE580004AA03C204A800F035FC40F2FF1000F039
:10EE680005FC40F6B80000F0DDFB00F0EF0140F6CD
:10EE7800B80000F0C7FB042140F6B90000F0C2FB5F
:10EE880040F69B0000F0CEFB00F0E30141F00801E2
:10EE980040F69B0000F0B6FB40F2D16000F0C2FBE8
:10EEA80040F01801C9B240F2D16000F0ABFB40F26B
:10EEB800AC6000F0B7FB00F08F0141F0500140F268
:10EEC800AC6000F09FFB4FF4FA5202FB08F2B2FB71
:10EED800F4F2CBF8082007B0BDE8F08F002000F06E
:10EEE8004DFD36498BF83850E2B2C95D8BF8502099
:10EEF800002F4DD10B3C012C8CBF00240124053A76
:10EF0800012A02D80C2E38BF0C26029B9AF8002042
:10EF18008BF852308BF85340019B8BF81F2001244B
:10EF28009DF860208BF821208BF851108BF8203049
:10EF38008BF80E40ABF81C608BF81E90FFF78EFA2A
:10EF48002046FFF7ABFB1E4800F0B8FE1D4800F056
:10EF580021FF5FFA88F000F01DFD40F6A30000F0E5
:10EF680061FB00EA040140F6A30000F04BFB9BF8AC
:10EF78002120A24240F2367013D100F053FB00F07A
:10EF8800FB0140F2367000F03DFB4FF6FF72A0E740
:10EF9800012F04D1A4F10C035C425C41AFE70024CB
:10EFA800ADE700F03FFB40F00401C9B2E9E700BF5C
:10EFB8009C1D002040010020480F01084E18010840
:10EFC800D41D0020AA1D0020F0B58BB00D460446C4
:10EFD80017461E46FFF742FA0020FFF75FFB204660
:10EFE80000F0BEFD00240123CDE9084303234FF4BC
:10EFF800167229462046CDE90644CDE90444CDE9F8
:10F008000244CDE900532346FFF774FE2046FFF77C
:10F018007DFAFFF735FAF3F761FD01F043FC04468A
:10F02800204601F049FCB04205D30124FFF716FA47
:10F0380020460BB0F0BD00F02FFF00B28742EFDA98
:10F048000024F3E7F7B500230C4640F201211A46E5
:10F058000646084600F01EFD644B654D4FF400520D
:10F068009A6195F85600012100F09CFF2B78012B3E
:10F0780040F6890013D195F85130062B0FD100F0D6
:10F08800D1FA00F0FB0140F6890000F0BBFA2B78BA
:10F09800042B6CD8DFE803F0524B527F090000F0D4
:10F0A800C1FA40F00401C9B2EDE7524A731E104696
:10F0B800C6F101074FF0000CF9188C426FDC0022F2
:10F0C800E7001346BA4271D19A0142EAC3125B01C2
:10F0D80083F020031343661C0355F6B20223464807
:10F0E800AB73AE7600F056FE0021F12000F08AFAEC
:10F0F8000021F02000F086FAAB6C642B70D17021EF
:10F10800F32000F07FFA1D21F22000F07BFAE100E5
:10F118008C1CF420090A00F075FA04F0FE01F520B1
:10F1280000F070FA33486FF07F4231461DE0EC770B
:10F13800314800F02FFE0022214615E001F008F8C2
:10F148000128074625D121460DF10702304601F076
:10F1580004F80446A0B99DF807302748AB7500F0BD
:10F1680019FE9DF807102246304600F065FB6968D5
:10F17800224801F063FC214801F026FC002006E04B
:10F188001F4B3A460021022001F0A2F8032003B0E9
:10F19800F0BDAC75CCE70223AB73AC76C8E713F8C7
:10F1A800011FC943197002F801CB85E7D1106FEA36
:10F1B800020C715C0CF0070C013241FA0CF101F001
:10F1C80001014FEAE20C4B40D14310F80CE001F08A
:10F1D800070103FA01F141EA0E0100F80C1071E78A
:10F1E800E121F32000F00EFA04218DE70004004825
:10F1F8009C1D0020801C0020AA1D0020F81D002056
:10F20800F0170108F0B5BDF814409DF818709DF886
:10F218001CE09DF8205040B1012814D001220023A1
:10F2280098180138B0FBF2F0F0BD87F00107E30051
:10F2380003EBC70318330EEB450503EBC5034FF487
:10F248007A714B43ECE7501F012803F1040302D8FD
:10F258000C2C38BF0C24D1B9A2F10B0CBCF1010F56
:10F268008CBF4FF0000C4FF0010C2801002F00EB71
:10F27800CE0014BF00251425A0EB8200062A4FEA11
:10F2880082062844A2F102070DD8354610E001296C
:10F2980006D1A2F10C00D0F1000C4CEB000CE4E715
:10F2A8004FF0000CE1E70830BCF1000FEDD0BD00D5
:10F2B8000028ACBF2E182E1C701E90FBF5F003FB27
:10F2C8000044094B062A5A5C8CBF0C340E340A2AB7
:10F2D80009D8A30001334FF47A71BB404B4303496B
:10F2E80051F822209CE7FFDE4E1801085418010847
:10F2F80008B5094B012193F8560000F053FE4FF46E
:10F30800D7602D2100F07EF900F033FBBDE80840FE
:10F31800024800F07BBA00BF9C1D0020FFFF0F00D1
:10F3280073B5A44CB4F854300025202B8DF8035045
:10F33800019500F01B8114D8082B0DD87BB1013B37
:10F34800072B0CD8DFE813F042005B000B00CD0060
:10F358000B000B000B00FD00102B00F0008102B029
:10F3680070BDB3F5807F00F0988011D8402B00F075
:10F378001081802BF3D1284600F032FA8E4B1B689F
:10F38800002BECD09B69002BE9D028469847E6E78C
:10F39800B3F5007FE3D1894B01222946022000F012
:10F3A80097FF00F029F9042840F08580844B8548B0
:10F3B8004FF400529A6201F0B9FA284600F010FAA8
:10F3C8007D4B1B68002BCAD05B6814E07C4B7D48E2
:10F3D8004FF400529A6201F0A9FA002000F000FAF6
:10F3E80000F0B8FE012801D100F0BDFE724B1B6889
:10F3F800002BB4D01B68002BB1D09847AFE7704BF7
:10F4080071484FF480529A6201F090FA657895B984
:10F41800284600F0E5F9294640F6021000F0F2F817
:10F4280040F6441000F0FEF840F00201C9B240F680
:10F43800441000F0E7F8FF220DF1030163485E4D28
:10F4480000F05AFD624800F071FD2B68002B86D051
:10F458009E68002E83D094F82430012B08D194F9AB
:10F46800313094F930209DF803105848B04776E7BA
:10F47800E06B01A900F022FE019B9DF803105348A0
:10F488004FF47A7203F5FA7393FBF2F32A685BB2CE
:10F49800956894F92920A84761E7284600F0A0F963
:10F4A800454B1B68002B3FF45AAF9B69002B3FF478
:10F4B80056AF01206AE700F09FF805287FF44FAFA8
:10F4C8003F4B41484FF480529A6201F02FFA284688
:10F4D80000F086F9384B1B68002B3FF440AFDB681F
:10F4E80089E700213B4B0122022000F0F1FEA16DCB
:10F4F80000293FF434AFC1F3074140F6031000F090
:10F5080081F894F8591040F6041000F07BF894F84C
:10F51800581040F6051000F075F840F6021000F09B
:10F5280081F840F00101C9B240F6021000F06AF813
:10F53800002340F262211A460846A36500F0AAFAA1
:10F548000DE7254B01220021022000F0C1FE00F04A
:10F55800FFFD01287FF403AF00F006FEFFE61F4B16
:10F5680001220021022000F0B3FEF8E6164801F05F
:10F57800DDF9607808B900F033F90F4B1B68002BF0
:10F588003FF4EDAEDB68002B3FF4E9AE9847144B2F
:10F59800E6E7144B01222946022000F099FE607824
:10F5A80008B900F01DF9044B1B68002B3FF4D7AED7
:10F5B8001B6920E79C1D0020801D002005180108FC
:10F5C80000040048F81D0020841D0020801C002035
:10F5D800C01D002019180108221801082C1801085C
:10F5E800351801083E180108024BA3F85400FFF72C
:10F5F80097BE00BF9C1D0020014B1878704700BFC4
:10F60800161E002007B501238DF807100DF107021B
:10F6180001460348F7F786F803B05DF804FB00BF1E
:10F628004C03002007B5012301460DF107020448E9
:10F63800F7F7B1F89DF8070003B05DF804FB00BFC9
:10F648004C03002010B50446F4F728FD01280CD11E
:10F6580040F62310FFF7E6FF00F0F901214340F6DA
:10F668002310BDE81040FFF7CDBF10BD10B50C4BFF
:10F678001B7804469BB94FF4D760FFF7D3FFC4F358
:10F68800002100F0FE0001434FF4D760FFF7BAFFF6
:10F69800E1B240F2B960BDE81040FFF7B3BF10BD5A
:10F6A800171E002010B51346EFF3108472B60A46F1
:10F6B80001460348F7F736F884F3108810BD00BFF9
:10F6C8004C03002008B5014608224FF4D860FFF724
:10F6D800E9FF002008BD000007B5074B1B7840BABA
:10F6E800ADF804002BB9022201A940F2BC60FFF773
:10F6F800D9FF03B05DF804FB171E002007B5074BC0
:10F708001B7840BAADF804002BB9022201A940F2D7
:10F71800BE60FFF7C7FF03B05DF804FB171E0020AB
:10F7280010B51346EFF3108472B60A460146034833
:10F73800F7F731F884F3108810BD00BF4C030020A0
:10F7480010B51346EFF3108472B60A460146034813
:10F75800F7F713F984F3108810BD00BF4C0300209D
:10F768000A4601460020FFF7EBBF000010B513461C
:10F77800EFF3108472B60A4601460348F7F730F9EA
:10F7880084F3108810BD00BF4C03002010B5134649
:10F79800EFF3108472B60A4601460348F7F736F8C5
:10F7A80084F3108810BD00BF4C03002013B5044635
:10F7B8000020F4F74DFC0220FFF744FF04F0070493
:10F7C80001220DF1070184208DF80740FFF7DEFFC5
:10F7D800024B00221A7002B010BD00BF161E002096
:10F7E80007B501228DF807000DF107018020FFF70A
:10F7F800CDFF9DF80730002B034B0CBF01220222DE
:10F808001A7003B05DF804FB161E002007B5094BFB
:10F818008DF8060004221A70030C8DF804300322B8
:10F82800030A01A983208DF80530FFF7AFFF03B065
:10F838005DF804FB161E002010B51446FFF790FF74
:10F848002046BDE81040FFF7E1BF000007B5094BAF
:10F858008DF8060005221A70030C8DF80430032277
:10F86800030A01A982208DF80530FFF78FFF03B046
:10F878005DF804FB161E002073B5002640F6E20072
:10F888000196FFF7CFFE00F0FE01054640F6E200C4
:10F89800FFF7B8FE40F6E500FFF7C4FE00F07F0171
:10F8A800044640F6E500FFF7ADFE6FF07F40FFF736
:10F8B800CDFF04220DEB020140F61900FFF730FFDF
:10F8C8003046FFF78DFF294640F6E200FFF79AFE23
:10F8D800214640F6E500FFF795FE019802B070BD9D
:10F8E80013B50C4B04460522972140F6AC001A705C
:10F8F800FFF788FE230C8DF804300322230A01A9A0
:10F9080082208DF805308DF80640FFF73FFF02B0E2
:10F9180010BD00BF161E002007B5030C8DF800307F
:10F92800030A8DF801300B0C49BA8DF80200ADF8C6
:10F9380004100622694694208DF80330FFF726FF4D
:10F94800024B06221A7003B05DF804FB161E002055
:10F95800002208B51146C520FFF718FF014B072202
:10F968001A7008BD161E002000221146D120FFF78C
:10F978000DBF00221146D220FFF708BF07B50122AC
:10F988008DF807000DF107019F20FFF7FFFE03B078
:10F998005DF804FB07B501228DF807000DF107019A
:10F9A800A020FFF7F3FE9DF807103F2907D901F0C3
:10F9B800F8010131C9B240F20670FFF723FE03B027
:10F9C8005DF804FB07B5F4F769FB431E584258413C
:10F9D8008DF8070001220DF107019620FFF7D6FEEA
:10F9E80003B05DF804FB07B500F07F008DF8070051
:10F9F80001220DF107018920FFF7C8FE03B05DF869
:10FA080004FB0000154B984207B51BD8144B9842CD
:10FA18001BD8144B98421BD8134B98421BD8134B36
:10FA2800984295BF29226B222B236F238DF804203F
:10FA380001A9022298208DF80530FFF7A7FE03B030
:10FA48005DF804FBE122E923F0E7D722DB23EDE7A9
:10FA5800C122C523EAE775228123E7E700E9A43537
:10FA680080F8A9328044E52D000B6B1B40FC54192B
:10FA780007B58DF8062004228DF804008DF80510CE
:10FA880095200DEB02018DF80730FFF77FFE03B0DC
:10FA98005DF804FB07B552BAADF8042040BA082255
:10FAA80049BAADF80000ADF802105BBA69461046D5
:10FAB800ADF80630FFF76AFE03B05DF804FB07B542
:10FAC8000B0C042200F0070049BA8DF80400ADF8C9
:10FAD800061097200DEB02018DF80530FFF756FE52
:10FAE80003B05DF804FB000010B508B1194B1860AD
:10FAF800F2F7F4FE0220FFF7A5FD0024164B20467E
:10FB08001C70FFF76DFEF4F7C7FA012817D14FF400
:10FB18002071FFF7D4FF40F611102146FFF772FD60
:10FB28004FF07F00FFF75FFF0E2140F61F10FFF731
:10FB380069FDF4F759FA094B01221A7010BD10211A
:10FB480040F61110FFF75EFD102140F61210FFF786
:10FB580059FDE9E7181E0020141E0020161E00207B
:10FB680037B50C4D2B7804461BB9FFF74BFF012323
:10FB78002B700023084A6006E109F1F7C5FF04224B
:10FB880000BA01900DEB02018620FFF7FFFD03B0DC
:10FB980030BD00BF141E00200048E80107B5094B1E
:10FBA8008DF807000146187018B940F2AC60FFF7ED
:10FBB80029FD01220DF107018A20FFF7E7FD03B0B7
:10FBC8005DF804FB171E0020012873B50C46164685
:10FBD80037D10020F4F764FAA042B8BF44B20E2827
:10FBE80005461AD101231A4600210420FFF740FFD9
:10FBF8006FF010039C42B8BF1C46182140F6E7007E
:10FC0800FFF700FD022201A98E208DF804408DF82F
:10FC18000560FFF7BBFD02B070BD01230A28E4B2FE
:10FC28001A464FF0000105D11846FFF721FF0334AB
:10FC380064B2DDE70720C5F10E05FFF719FF2C4474
:10FC4800F6E740F6D800FFF7EDFC40F01E01C9B218
:10FC580040F6D800FFF7D6FC0120F4F721FAA042BD
:10FC6800B8BF44B2142805464FF001034FF0000214
:10FC78000CD105210320FFF7FBFE023464B26FF0BC
:10FC880008039C42B8BF1C463821B7E7112805D1A4
:10FC980003210220FFF7ECFE0534EFE70E2804D11C
:10FCA80002210846FFF7E4FEE9E7C5F1160507213A
:10FCB80004202544FFF7DCFE6CB2E0E713B5314AB7
:10FCC8000446516810686B4603C32F4B20781B7895
:10FCD800834201D0FFF762FF2378032B27D8DFE8A0
:10FCE80003F00239283C6268284BB3FBF2F31A0C84
:10FCF800A1688DF800208DF802301A0A237B8DF850
:10FD08000330637B8DF801208DF80430204A0023EE
:10FD18004806C909F1F7F8FE030C40BA8DF805301A
:10FD2800ADF80600082269468B20FFF72FFD02B0C8
:10FD380010BD2269154BB3FBF2F31A0C8DF80020A5
:10FD48008DF802301A0A237D8DF801208DF80330D2
:10FD58000422E8E7A3690093FAE762680B4BB3FB58
:10FD6800F2F31A0C8DF800208DF802301A0A237B62
:10FD78008DF80330637B8DF801208DF8043005225F
:10FD8800D1E700BF580F0108171E00200000093DE9
:10FD98000048E8011FB52E4A0446D1689068127CD5
:10FDA80001AB03C31A702B4B20781B78834201D018
:10FDB800FFF7F4FE2378032B26D8DFE803F0023898
:10FDC8003302637AF12B21D14FF6FF70FFF784FCE1
:10FDD80048F20500FFF792FC02236288A188ADF87B
:10FDE800061052BAE188ADF804208DF80B30227A5B
:10FDF800A37A8DF80A20ADF808108DF80C30092286
:10FE080001A98C20FFF7C2FC04B010BDF22BE4D18D
:10FE180041F60F50FFF760FC41F22100FFF76EFC3E
:10FE28000623DAE7237B8DF804300122E8E7E3892B
:10FE3800094A5BBAADF80430237C13708DF806309C
:10FE4800637C8DF80730638AADF808300622D7E75F
:10FE5800580F0108171E0020151E002007B50222A2
:10FE68008DF804008DF805108F2001A9FFF78EFC8E
:10FE780003B05DF804FB000010B51346EFF31084DF
:10FE880072B60A4601460348F6F7F8FC84F3108870
:10FE980010BD00BF4C03002007B5012201A91520A1
:10FEA800FFF7EAFF9DF804004042401003B05DF8F8
:10FEB80004FB000037B505460C46022201A91320B1
:10FEC800FFF7DAFF0A4B1B78012B0DD1094B1B7882
:10FED800012B09D140F20270FFF7A4FB9DF8053011
:10FEE8002870237003B030BD9DF80400F6E700BF0A
:10FEF800171E0020151E0020F7B50D4606460024E3
:10FF08000DF10701284617468DF80740FFF7D2FF85
:10FF18002A78BA4207D89DF807003146FFF726FC31
:10FF2800204603B0F0BD0120FBE7000013B5032213
:10FF3800044601A91420FFF79FFF184B1A78227076
:10FF48004AB1012A17D014220021204600F0D2FA23
:10FF58000F2323700DE09DF8043023719DF80530C0
:10FF6800A2605B425B10A3719DF806305B425B1098
:10FF7800637102B010BD9DF804305B425B102373BF
:10FF88009DF9053002339B1063739DF806305B4280
:10FF98005B10A373024B1B682361EAE7171E00205E
:10FFA800101E0020012908B5034608460ED1012B72
:10FFB80007D10420FFF746FB0220BDE80840F4F70C
:10FFC80047B8022B14BF08460320F6E70120F4E7E0
:10FFD80038B50446F4F75EF850B1022814BF01257D
:10FFE8000225284602222146FFF7EEFD284638BDA5
:08FFF8000F2CCCBF02250125EE
:020000040801F1
:10000000F3E70A2070470000014B01201B681847E6
:10001000181E0020014B02201B681847181E0020E4
:10002000014B40201B681847181E002011B1012900
:1000300004D07047044B1B6880201847024B4FF4D4
:1000400080701B68F9E700BF181E0020024B4FF4B8
:1000500000701B68184700BF181E0020014B2020AD
:100060001B681847181E0020014B04201B68184706
:10007000181E0020014B08201B681847181E00207E
:10008000014B10201B681847181E0020024B4FF42C
:1000900080401B68184700BF181E002068B1084A3E
:1000A000002352F83310814203D902EBC3021079C6
:1000B00070470133162BF4D1FEE71F20704700BFB5
:1000C0001019010873B51D4B0193044640F6070053
:1000D0000D46FFF7ABFAC0F3C10308336B4413F8C6
:1000E000042C00F00703013302FA03F3144AB2FBB5
:1000F000F3F2B2FBF4F007281ED8400003288CBFAF
:10010000022304234FF4D66002FB03F4FFF78EFAB8
:10011000060240F2B160FFF789FA06F470663043D8
:10012000030544BF6FEA00506FEA10506309434370
:10013000DB112B6002B070BD0123E3E704080A0C59
:100140000048E8014FF0FF3070474FF0FF30704734
:100150004FF0FF3070477047002070470020704715
:1001600070474FF0FF3070474FF0FF3070477047D7
:100170007047704770B5EFF3108672B6144B5C8A07
:100180001A8A944213D1C4F5806292B2904206D387
:10019000844218D901229A7000221C805A825A8AFD
:1001A0000A800244C2F309025A8200200DE006D9F7
:1001B000C4F58065ADB28542F1D88242E9E7121BF1
:1001C00092B28242EBD84FF0FF3086F3108870BDB8
:1001D0001C220020EFF3108172B6034AD38A013348
:1001E000D38281F3108870471C220020EFF3108126
:1001F00072B6034AD38A013BD38281F310887047D9
:100200001C22002010B508481822002100F076F9C1
:1002100006484FF48062002100F070F9044B054855
:100220001B68BDE8104018471C2200201C1E00203F
:10023000F80F0108A5030108014B5860704700BF83
:100240001C220020014B1872704700BF1C220020A6
:1002500073B5EFF3108572B61C4CE08A00282FD1DD
:10026000FFF7B8FF218A628A914227D0A378012B39
:1002700012D1238820805B1A9BB20221A382A17035
:1002800063B9A3702382238A9A428BBFD21AC3F523
:100290008063A282A38201E0002BF4D0238A0C4E5B
:1002A0001E4485F31088F2F70BFC0A4BA18ADB6829
:1002B0000193304602B0BDE870401847FFF796FF43
:1002C00085F31088002002B070BD00BF1C22002002
:1002D0001C1E0020F80F010808B4F0B586B00023FA
:1002E000ADF800302C4B0B9C1D7A85424DD3D8685D
:1002F00081434DD15B681BB112B1694602A8984792
:100300000CAB22464FF400712448019300F0F6FB39
:10031000FFF760FFBDF8003018440DF1020180B214
:10032000FFF728FF01302BD00022BDF80030BDF8C8
:1003300002701B480DF1080C164691B217FA82F5AF
:100340008B42ADB216D83B449BB20EB1ADF8023031
:10035000BDF80250019B22464FF40071284400F082
:10036000CDFBFFF743FFFFF773FF06B0BDE8F0409A
:1003700001B070471CF8011B415501320126DCE732
:10038000FFF734FF6FF00200EFE76FF00400ECE7D7
:100390006FF00500E9E700BF1C2200203422002096
:1003A0001C1E002013B5EFF3108472B6204B9A7810
:1003B000588A022A1DBF1A8A998A5218002214BF2D
:1003C000C2F309029A7090421A8228D0D98A012970
:1003D00025D19978012913D119888A1A022192B25C
:1003E000997000219A82198062B99A701A821A8AC9
:1003F00090428BBF801AC2F5806298829A8201E097
:100400000029F4D01A8A0B48104484F310880A4A51
:10041000998AD368019302B0BDE81040184784F36D
:100420001088F2F751FB02B0BDE81040FFF7DEBEC6
:100430001C2200201C1E0020F80F0108024A002385
:100440001360024A136070473824002034240020CF
:1004500010B5EFF3108472B641B1012903D1064AF9
:1004600013680343136084F3108810BD024A1368B5
:1004700023EA0003F6E700BF3824002010B5EFF3AD
:10048000108472B641B1012903D1064A13680343AF
:10049000136084F3108810BD024A136823EA000336
:1004A000F6E700BF3424002038B5EFF3108572B6AC
:1004B0000A4B0B4C1B6833B1236898476368984715
:1004C00085F3108838BD074B1B681BB1A36898479C
:1004D000E368F4E7236998476369F0E7382400206C
:1004E000840F01083424002001380A44914200D1CD
:1004F000704711F8013B00F8013FF7E700F02CBC12
:1005000010B5EFF3108472B6064A13680343136004
:10051000054A52F83130034342F8313084F31088F1
:1005200010BD00BF88240020802400207047704741
:10053000030C1B04C3B90004102310F07F4F02BF4B
:1005400008330002DBB210F0704F08BF00014FEA21
:100550001070064A08BF0433125C08BFDBB2C3F157
:100560001F03981AC0B270470023E6E7C0190108BC
:100570002DE9F84F384D394ED5F80080DFF8E0B05E
:10058000DFF8E0A0DFF8E090D6F800C0374FDBF8E6
:100590000010374CDAF80020D9F8003008EA0000E3
:1005A0002860286800EA020E1EEA0C0F01D01942EA
:1005B0001ED04FF0FF333B60FFF7B8FFEFF310841E
:1005C00072B63368DBF80020DAF800100B402968B7
:1005D0000B4205D1D9F80030134201D1F2F7FEF9F0
:1005E00084F31088FFF7A3FFC5F80080BDE8F88FFB
:1005F000236823680340134062681A4204BF4FF027
:10060000FF32626060681840FFF792FF62683860EE
:10061000012303FA00F022EA00026260EFF3108186
:1006200072B63A689340326822EA03023260226866
:1006300022EA0303236081F310880E4A3B6852F8D4
:1006400023309847D6F800C0DBF80010DAF8002015
:10065000D9F80030A5E700BF44010020882400201D
:100660004024002048010020442400203C24002095
:10067000802400204824002010B51146EFF3108498
:1006800072B6FFF755FF034B43F8201084F3108830
:1006900010BD00BF4824002082B082B00DF1080CCC
:1006A0000CE90600BDF8042003930B44BDF81010BC
:1006B0000A4491B212B2B2F57A7FA2BFA1F57A7262
:1006C000013312B20360828002B002B0704782B080
:1006D00082B00DF1080C0CE90600BDF8042003936C
:1006E000CB1ABDF81010521A91B212B2002ABEBF36
:1006F00001F57A7203F1FF3312B20360828002B017
:1007000002B0704730B585B0114D6B4683E80300E9
:1007100000230293ADF80C3003A82B699847009B87
:10072000BDF804400290181ABDF80C30E41AA3B2C8
:1007300024B2002CBEBF03F57A731CB200F1FF3067
:100740002B689847AB682046984705B030BD00BF7E
:10075000B80F010873B5114E002305460093ADF89C
:10076000043001A833699847F3680090984773688C
:1007700004469847009B1844BDF8043023449AB2BD
:100780001BB2B3F57A7FA2BF0130A2F57A731BB218
:1007900028602846AB8002B070BD00BFB80F0108CA
:1007A00037B500230093ADF80430074B04461B69AE
:1007B00001A898476D46009095E8030084E803007F
:1007C000204603B030BD00BFB80F010837B50F4D4C
:1007D00002AB03E90300EB6898476B68044698474F
:1007E000BDF80430009A1B1B99B21BB2002BA2EB80
:1007F0000002BEBF01F57A7102F1FF320BB24FF475
:100800007A7000FB023003B030BD00BFB80F0108A2
:100810002DE9F0414FF47A75B1FBF5F5C5EB4513C1
:10082000DFF83C8005EB8303A1EBC3039CB2D8F84F
:100830000C3006469847D8F8043007469847E31925
:1008400099B21BB2B3F57A7F2844A2BFA1F57A739F
:1008500001301BB23060B3803046BDE8F08100BF8C
:10086000B80F0108024B00221A60024B1B681847A0
:100870008C240020CC0F0108F8B504461746084622
:100880001E467CB173B1084B00255B6A2560984712
:10089000069B60602581A572E6602361E772656151
:1008A0002846F8BD0120FCE7CC0F010810B5034C29
:1008B000E3699847A36ABDE810401847CC0F0108C8
:1008C00070B5064DEB69064698476B6A044630469C
:1008D0009847AB6A201ABDE870401847CC0F010852
:1008E000054B1B680BB918467047834201D05B6902
:1008F000F8E70120704700BF8C2400202DE9F34168
:100900000B4E336A044698470123B7692372D4F823
:1009100000800546B8472844804502D2B84728449D
:100920002060B3682068019302B0BDE8F041184729
:10093000CC0F010870B520B3EFF3108672B6124DDC
:100940002B680122827253B10022427298425C6984
:100950000ED102723CB120462C60FFF7CFFF86F328
:100960001088002070BD094BDB6898472C60F6E7C3
:100970001A465B69002BF2D09842F9D14369536162
:10098000EDE70120EEE700BF8C240020CC0F01082A
:10099000084B10B51A685369516911B9506141612A
:1009A00010BD046819688C4202D91A465B69F3E7E6
:1009B0001946F3E78C240020044A13680BB1002188
:1009C000197243611060FFF799BF00BF8C240020AB
:1009D0002DE9F041044600282DD0FFF781FF50BBE0
:1009E000657A45BBEFF3108872B6144E6768336AB8
:1009F000984787422CBF27602060114FA5724FF4A3
:100A0000807323813B684BB9336998472046FFF7D1
:100A1000D3FF88F310882846BDE8F081B369984772
:100A2000236818443B6820601B6898422046EED338
:100A3000FFF7AEFFEDE70125EDE700BFCC0F0108A2
:100A40008C24002010B5044608467CB1084B5B6A34
:100A5000984760602046FFF743FF40B12046FFF70C
:100A600069FF2046BDE81040FFF7B2BF012010BD6E
:100A7000CC0F01082DE9F041EFF3108772B61D4E3F
:100A80001D4D736998473369044698472B684BB9E5
:100A90004FF000082B688BB9286828BB87F31088B3
:100AA000BDE8F081011B241A1A688A428CBF121912
:100AB00000221A605B69002BF6D1E9E71C681CB1C3
:100AC000B36998478442E7D22C6863692B60A4F825
:100AD0000880D4E9033098476389B3F5807FD9D182
:100AE0002046FFF775FFD5E7037A002BD6D1FFF735
:100AF00005FFD3E7CC0F01088C2400202DE9F04F2F
:100B000097B000298046039140F30E819A4604462F
:100B100003991378A4EB0800013923B9002323704B
:100B200017B0BDE8F08F8842F8DA252B04D004F81E
:100B3000013B1646721CEBE792F801C0ACF13003A2
:100B4000D3F1000E4EEB030EACF13003092B02F192
:100B5000010629D8324600254FF00A09164612F838
:100B6000013BA3F13000092819D93378692B00F033
:100B70009C801CD8632B28D0642B00F09680582BC7
:100B80005BD0252B19D13378002B00F0928004F82C
:100B9000013BA4EB08038B4280F28980CAE709FB82
:100BA0000533A3F13005D9E74FF0FF35DDE7752BAD
:100BB0007DD0782B43D0732B1ED0252304F8013B26
:100BC000A4EB08038B4272DADDE7002D05F1FF3953
:100BD000D8BF4FF000094A462046202100F0BCF85B
:100BE0005346A144002D53F8042B89F80020D8BFA8
:100BF00001252C449A469DE74C4B5AF8047B002F64
:100C000008BF1F463846F0F7DBFBA5EB000B85421B
:100C1000B8BF4FF0000B5A4681462021204600F015
:100C20009BF8A34400234B4502DB0BEB090481E74F
:100C3000FA5C0BF803200133F5E74EF0400E10206C
:100C4000DFF8EC903B4F1EF0400F08BF4F46534675
:100C5000BCF1300F0197A4EB08020CBF302720270E
:100C60001EF0020FA1EB0202029753F8041B22D0E0
:100C7000002920DA4942013D4FF02D0E05AF0097C3
:100C800000278946DDF804A0B1FBF0F100FB119BC1
:100C900048451AF80BB0DDF800A00AF801BB07F1CF
:100CA0000107CDF800A0ECD90EE04EF0020E0A20AC
:100CB000C6E7013E6DE711B14FF0000EDEE73020D0
:100CC0008DF814008E460127BCF1300FA5EB070507
:100CD00004D02020002D05F1FF3509DCBEF1000F06
:100CE00004D02D21013A04F8011B83D025440AE0E9
:100CF000013A04F8010BEDD17CE7029904F8011BDD
:100D0000013A3FF477AF291B0029F6DC05A93944E5
:100D100022442744A7423FF46DAF11F8010D04F8B7
:100D2000010B9442F6D165E70020F9E6D0190108DD
:100D3000D7190108FC19010810B501390244904285
:100D400001D1002005E0037811F8014FA34201D042
:100D5000181B10BD0130F2E702440346934200D154
:100D6000704703F8011BF9E770B50D4D0D4C641B7E
:100D7000A4100026A64209D10B4D0C4C00F0B0F88F
:100D8000641BA4100026A64205D170BD55F8043B93
:100D900098470136EEE755F8043B98470136F2E7ED
:100DA000041B0108041B0108041B0108081B01089F
:100DB00000F003B8002200F00EB80A44914200F19E
:100DC000FF3300D1704710B511F8014B03F8014F04
:100DD0009142F9D110BD13460A461946FFF7BCBF30
:100DE000C1F30A522DE9F843A2F2FF36132E0B4647
:100DF00007460C46054632DC002E14DA34A3D3E94C
:100E00000023F0F7EBFA00220023F0F71BFD38B1C6
:100E1000002C56DA24F00044254355D02E4C0025F2
:100E200023462F4625E02D4A42FA06F801EA080239
:100E300002431ED026A3D3E90023F0F7CFFA002205
:100E40000023F0F7FFFC0028EAD0002CBEBF4FF4CF
:100E500080133341E41824EA08040025E0E7332E28
:100E60000BDDB6F5806F04D10246F0F7B7FA0746FE
:100E70000B4638461946BDE8F883A2F213424FF0FC
:100E8000FF3828FA02F810EA080FF2D010A3D3E9CD
:100E90000023F0F7A3FA00220023F0F7D3FC002888
:100EA000BED0002C0ADA142E01D1013406E0C6F1BE
:100EB00034060123B3401D44AF42F6D825EA0805A5
:100EC000AEE700252C46ABE74FF00044A8E700BF93
:100ED0009C7500883CE4377E0000F0BFFFFF0F00E8
:100EE000F8B500BFF8BC08BC9E467047F8B500BF17
:080EF000F8BC08BC9E467047E7
:100EF80000000000010000000200000000000000E7
:100F08008813000010270000204E000030750000F4
:100F1800409C000050C3000060EA0000C0D40100FB
:100F280080A903000053070000EA0637000000000C
:100F38005000000040F70937000000005000000092
:100F4800C194C10000000000B227000000000000AA
:100F58000000000000000000000000000000000089
:100F680000000000B5010008F10100086C0F01083D
:100F7800FC7F003F00350113C41200089F270008BA
:100F880081270008652700088527000861270008D1
:100F9800B12700085975336E3148344F3152354EF8
:100FA800395332543653256473253033643A00007C
:100FB8008D2C00082D2D00089D2C0008392D0008C7
:100FC800FD2C0008452D000800000000AD2C00088D
:100FD800652C0008312C0008E92B0008412C00087A
:100FE800552C0008F52B0008F92B00080D2C0008DB
:100FF800ED2F000815300008992F0008852F0008EC
:1010080052464143005056585858002159756E4869
:101018006F726E20535453205265766976652100AD
:1010280001000000030000000500000001000000AE
:1010380001000000060000000A0000002000000077
:10104800020000000400000008000000100000007A
:1010580040000000800000000001000000020000C5
:101068000000000000000000000000000000000078
:10107800010000000200000003000000040000005E
:10108800A0860100400D0300801A060000350C0000
:1010980040420F0080841E0000093D0000127A00C3
:1010A8000024F40000366E010048E801006CDC0200
:1010B8000000000000000000000000000000000028
:1010C800040208001010100410101002101010086C
:1010D800010002000400060008000A000C001000CD
:1010E80020004000800000010804020408010101FA
:1010F80001010103070100006572726F723A205204
:101108006567696F6E206973206E6F742064656609
:10111800696E656420696E20746865204D573A20B1
:10112800736574206C6F726177616E5F636F6E6652
:101138002E68206163636F7264696E676C790D0A4B
:10114800004D414320727854696D654F75740D0ADE
:10115800004D414320747854696D654F75740D0ACC
:10116800004D4143207278446F6E650D0A004D4171
:1011780043207478446F6E650D0A00080A0C0D0E42
:1011880010121415181A1B1D1E212403050205012F
:101198000602020500000600000105040400000024
:1011A80048E8010048E8010048E8010048E8010073
:1011B80048E8010048E8010090D003000000000062
:1011C800030000000201000C0B0A0908070732009F
:1011D80000000000000102010000000000020302FC
:1011E80001000000000304030201000000040504DC
:1011F80003020100000506050403020100060706B4
:10120800050403020107070706050403020707028E
:1012180002020202020202020202020202020302A5
:10122800020202020203040302020202020405048B
:10123800030202020205060504030202020607066B
:10124800050403020207070706050403020707331C
:10125800337373F2F2F2F200000B357DF2F2F233DF
:10126800337373DEDEDEDE52585F2573206F6E2027
:101278006672657120256420487A20617420445282
:101288002025640D0A005258206F6E206672657121
:1012980020256420487A2061742044522025640D5A
:1012A8000A005458206F6E206672657120256420EC
:1012B800487A2061742044522025640D0A003100C8
:1012C80032004D756C74695F43004D756C74695FCD
:1012D80050000000C6120108C81201080B100108CE
:1012E800CA120108D8120108D2120108C6F8EEF68F
:1012F800FFD6DE916002CE56E7B54DEC8F1F89FA16
:10130800EFB28EFB41B35F452353E49B75E13D4C3F
:101318006C7EF5836851D1F9E2AB622A0895469D47
:1013280030370A2F0E241BDFCD4E7FEA121D5834AA
:1013380036DCB45BA476B77D52DD5E13A6B900C176
:1013480040E379B6D48D67729498B085BBC54FEDEC
:10135800869A66118AE904FEA078254BA25D80056D
:101368003F2170F16377AF4220E5FDBF811826C3A6
:10137800BE35882E9355FC7AC8BA32E6C0199EA3AA
:1013880044543B0B8CC76B28A7BC16ADDB647414A4
:10139800920C48B89FBD43C43931D3F2D58B6EDA6D
:1013A80001B19C49D8ACF3CFCAF447106FF04A5C3E
:1013B80038577397CBA1E83E96610D0FE07C71CC4E
:1013C8009006F71CC26AAE6917993A27D9EB2B2207
:1013D800D2A907332D3C15C987AA50A50359091A64
:1013E80065D784D082295A1E7BA86D2CA584998D37
:1013F8000DBDB1545003A97D1962E69A459D4087F9
:1014080015EBC90BEC67FDEABFF7965BC21CAE6A29
:101418005A41024F5CF434089373533F0C52655E93
:1014280028A10FB509369B3D2669CD9F1B9E742EBA
:101438002DB2EEFBF64D61CE7B3E7197F568002C20
:10144800601FC8EDBE46D94BDED4E84A6B2AE516C4
:10145800C5D75594CF100681F044BAE3F3FEC08A8D
:10146800ADBC4804DFC17563301A0E6D4C14352FBE
:10147800E1A2CC3957F28247ACE72B95A098D17FEF
:10148800667EAB83CA29D33C79E21D763B564E1E55
:10149800DB0A6CE45D6EEFA6A8A4378B324359B71C
:1014A8008C64D2E0B4FA0725AF8EE918D5886F723C
:1014B80024F1C751237C9C21DDDC86859042C4AA97
:1014C800D8050112A35FF9D0915827B93813B3335F
:1014D800BB7089A7B622922049FF787A8FF88017C7
:1014E800DA31C6B8C3B07711CBFCD63A637C777BC8
:1014F800F26B6FC53001672BFED7AB76CA82C97D08
:10150800FA5947F0ADD4A2AF9CA472C0B7FD932698
:10151800363FF7CC34A5E5F171D8311504C723C39C
:101528001896059A071280E2EB27B27509832C1AE0
:101538001B6E5AA0523BD6B329E32F8453D100ED3A
:1015480020FCB15B6ACBBE394A4C58CFD0EFAAFB1E
:10155800434D338545F9027F503C9FA851A3408FE6
:10156800929D38F5BCB6DA2110FFF3D2CD0C13ECFE
:101578005F974417C4A77E3D645D197360814FDC93
:10158800222A908846EEB814DE5E0BDBE0323A0A77
:101598004906245CC2D3AC629195E479E7C8376DFB
:1015A8008DD54EA96C56F4EA657AAE08BA78252E20
:1015B8001CA6B4C6E8DD741F4BBD8B8A703EB566A9
:1015C8004803F60E613557B986C11D9EE1F898119A
:1015D80069D98E949B1E87E9CE5528DF8CA1890D89
:1015E800BFE6426841992D0FB054BB16232323232D
:1015F800232320257320253032583A253032583A93
:10160800253032583A253032583A253032583A2562
:101618003032583A253032583A253032583A253047
:1016280032583A253032583A253032583A25303235
:10163800583A253032583A253032583A25303258FF
:101648003A253032580D0A0023232323232320442C
:1016580065764555493A20202020202025303258EB
:101668003A253032583A253032583A253032583AED
:10167800253032583A253032583A253032583A25F2
:101688003032580D0A00232323232323204170706E
:101698004555493A202020202020253032583A2527
:1016A8003032583A253032583A253032583A2530B7
:1016B80032583A253032583A253032583A253032A5
:1016C800580D0A00232323232323204465764164ED
:1016D80064723A2020202020253032583A253032B2
:1016E800583A253032583A253032580D0A004170A0
:1016F800704B65793A2020202020004E776B4B658F
:10170800793A2020202020004E776B534B65793A98
:101718002020202000417070534B65793A2020200A
:1017280020004442496E744B65793A202020004DD0
:1017380043526F6F744B65793A2020004D434B45F7
:101748004B65793A20202020004D43417070534B5F
:1017580065795F303A004D434E776B534B65795F3F
:10176800303A0000000000004150505FF6160108B2
:10177800010000004E574B5F0317010808000000E6
:101788004E574B53101701080900000041505053A1
:101798001D1701080A0000004442495F2A17010882
:1017A8000B0000004D435254371701080C0000008D
:1017B8004D434B45441701080D0000004D434B3085
:1017C800511701080E0000004D4153305117010810
:1017D8000F0000004D4E53305E1701081000000046
:1017E8005A45524F2B180108526164696F53656E50
:1017F80064204F76657273697A650D0A0049525103
:101808005F52585F54585F54494D454F55540D0A1F
:1018180000505245204F4B0D0A0053594E43204F5C
:101828004B0D0A00484452204F4B0D0A00484452C1
:10183800204B4F0D0A004952515F4352435F4552B6
:10184800524F520D0A00040506000000841E0000D5
:10185800093D0000127A000024F4000048E8010065
:1018680090D0030020A1070000000000B12800006C
:1018780061510000C3A2000002010003A9E50008AD
:101888006DE40008A5E60008E9E40008D1EF0008C7
:1018980091E50008FDEC000875EB00084DE3000831
:1018A8000DF200084DF000087DE5000865E4000829
:1018B80015E50008EDE40008A5E400089BE400082D
:1018C8009DE3000899E3000897E4000893E4000802
:1018D8003DE6000869E6000889E4000829F30008E5
:1018E800FDE30008C5E30008F9F20008A1E30008D9
:1018F8006DE90008F1E60008450101084B010108FF
:1019080091E3000895E30008C01200001F000000E2
:10191800A816000017000000841C00000F0000003B
:10192800E42500001E000000B42D00001600000091
:10193800083900000E0000002C4C00001D000000BB
:10194800685B000015000000747200000D000000C4
:10195800589800001C00000034B700001400000074
:10196800E8E400000C000000783101001B000000D2
:10197800686E01001300000034CA01000B0000006B
:10198800286202001A00000040DB0200120000007A
:101998003C9303000A000000C0C2040019000000C4
:1019A80060B305001100000038200700090000009E
:1019B80020A1070000000000040302020101010148
:1019C80000000000000000003C4E554C4C3E00302A
:1019D8003132333435363738396162636465666766
:1019E80068696A6B6C6D6E6F7071727374757677F7
:1019F80078797A00303132333435363738394142E4
:101A0800434445464748494A4B4C4D4E4F50515226
:0C1A1800535455565758595A000000000E
:101A240000000000000000000000000000000000B2
:101A34000000000000000000002B7E151628AED226
:101A4400A6ABF7158809CF4F3C012B7E151628AE9F
:101A5400D2A6ABF7158809CF4F3C082B7E15162864
:101A6400AED2A6ABF7158809CF4F3C092B7E1516CD
:101A740028AED2A6ABF7158809CF4F3C0A00000068
:101A8400000000000000000000000000000B000047
:101A940000000000000000000000000000000C0036
:101AA4000000000000000000000000000000000D25
:101AB4000000000000000000000000000000000022
:101AC4000E00000000000000000000000000000004
:101AD400000F0000000000000000000000000000F3
:101AE40000001000000000000000000000000000E2
:081AF4000000000000000000EA
:081AFC004400FF7F010000001F
:041B04005D01000877
:041B08003901000897
:101B0C000200000000000000D2040020C0D401003C
:101B1C00E1290008112A0008292A0008952A000842
:101B2C00E5320008BD320008513200084B35000880
:101B3C00000000000935000825320008513F00085C
:101B4C000B320008093200085135000859320008E0
:101B5C000D32000819320008D534000800020100CB
:101B6C000000000000000000000000000400000065
:101B7C00401F000010270000005601013053054D96
:101B8C000400002008190F28040A413F00050A012F
:101B9C000000050203FFFFFFFFFFFFFFFFFFFF0F2A
:101BAC000103000200000000000000000000000023
:101BBC00000000000000000000093D0010000000C3
:101BCC00100800200000FF000000000000000000D2
:101BDC00100800200000000000000000FF000000C2
